:020000040800F2
:1000000000C00020F143010891440108D92D0108E6
:100010009144010891440108914401080000000046
:1000200000000000000000000000000091440108F2
:100030009144010800000000914401087581000806
:100040009144010891440108914401089144010838
:100050009144010891440108C5B40008C1B40008E6
:100060009144010891440108914401089144010818
:100070009144010891440108E1B400089144010849
:1000800055CC0008914401089144010891440108AD
:10009000914401089144010891440108BDB400084D
:1000A00091440108ADB2000891440108BDB20008B6
:1000B0009DB200088DB200087DB20008B95A000850
:1000C000BD5A0008B15A0008B55A00089144010809
:1000D00091440108D5B40008C9B40008914401084E
:1000E0008581000891440108914401089144010868
:1000F0009144010891440108914401089144010888
:100100009144010891440108914401089144010877
:100110009144010891440108914401089144010867
:100120009144010891440108914401089144010857
:1001300000000000000000000000000000000000BF
:1001400000000000000000000000000000000000AF
:10015000000000000000000000000000000000009F
:10016000000000000000000000000000000000008F
:10017000000000000000000000000000000000007F
:10018000000000000000000000000000000000006F
:10019000000000000000000000000000000000005F
:1001A000000000000000000000000000000000004F
:1001B000000000000000000000000000000000003F
:1001C000000000000000000000000000000000002F
:1001D000000000000000000000000000000000001F
:0401E0005FF8E0F1F3
:1001E8002DE9F04F684B694FA1B03B6000237B605D
:1001F80011F00CFC18B911F02BFC0AF0FDF80AF00C
:10020800A1F9634A634C1378634E43F001031370FA
:100218000023089309930A934FF4E0130B93236880
:10022800B07B43F480332360A36943F01003A361D8
:10023800236803F400330993089B01330893099B4F
:100248001BB9089BB3F5A06FF2D12368514913F489
:10025800003301D0022315E00A6842F001020A6067
:100268000893236803F002030993089B013308935A
:10027800099B1BB9089BB3F5A06FF2D123689B07B4
:1002880039D501230A93454B45491A6842F01002B3
:100298001A601A6822F003021A601A6842F0020211
:1002A8001A606368636063686360636843F48063CB
:1002B80063603C4B1A68043B22F070425A603A4A29
:1002C8001160616821F47C116160596841F0004156
:1002D8005960D96821F40041D9609B681D0449BF61
:1002E800324B4FF4E01313604FF480130B930A9BC7
:1002F800012B01D117E0FEE7022B18D168B10B9B47
:10030800B3F5801F02D14FF4A01305E00B9BB3F5A2
:10031800E01F02D14FF400130B930B9963680B4352
:1003280043F4803302E0636843F460136360236836
:1003380043F0807323602168164B8901FBD5596807
:1003480021F003015960596841F00201596063685E
:10035800104903F00C03082BF9D14B68DFF85490CF
:1003680003F00C03042B03D0082B03D00C4B29E01B
:10037800136827E04B684868C3F38343C50303F158
:10038800020319D40A4A1CE0E79B0008C8000020B1
:10039800C030002000100240D4110020002002408C
:1003A80000127A000410014034000020001BB7003E
:1003B80000093D005000002049681268880348BFC2
:1003C80052085343C9F800306368DFF888A2C3F3C2
:1003D800031353441A7ED9F80030DFF87CC2D340A7
:1003E800C9F80030854A864B20ADD360A3690492D2
:1003F80043F00103A361636ADFF86082BB60636A4C
:10040800604643F080736362A3694FF0000B43F0CA
:100418001C03A3614FF6FF7325F82C3D2946CDF840
:100428000CC08DF856B00CF007FD404629460CF07C
:1004380003FD744829460CF0FFFC734928464B68B5
:1004480043F000734B600EF015FF159B6F49049A3B
:10045800B3FBF1F36E490B606E4B4FF47A71C3F83E
:1004680000B0D9F80030DFF8F891B3FBF1F36A492E
:10047800013B4B60F02382F823300723C1F808B012
:100488000B60B368DFF898B1C9F800300AF12803A7
:100498000FCB85E80F00A369159843F00803A36103
:1004A800A36916A943F00803A3610823C8F810300C
:1004B8001023C8F8103004930CF0BEFC179818A944
:1004C8000CF0BAFCD9F80020049B12F0080F12D0E7
:1004D8009BF89221012A0ED850499BF893218968EC
:1004E80011F0805B00F0CB8405E04D4B002283F8CF
:1004F80093210AF0EBF9642007F0EBFDA0224948AC
:10050800002116F04AFBE369002243F00703E36188
:10051800A36943F4006343F00C03A3613F4B4FF01E
:10052800000B03F10C0102F801B001320E2AF5D1DB
:10053800FF229A76DA761A775A773B4B3B4A594626
:100548001A603B483022D9F8004016F026FB59467D
:10055800C4F380180423374ADFF8D4E0885C0C22FF
:100568004A4302F80E00B8F1000F08D11E380128DE
:100578009FBFFF2003F1FF3302F80E00DBB2013109
:100588000429E8D12C4A96F805B013702B4B2C4956
:1005980083F800B02B4B214A3B62C0330B602A4BD7
:1005A800A10603EBCB035B7848BF0123536200230A
:1005B80040F2DC51254A22F813100133082BF7D1F9
:1005C8000EA800211C2216F0E8FA14F4007304F4B3
:1005D800006947D0A2040BD4B9F1000F0AD01C4A15
:1005E80096F88601A2F10C01012808BF0A4602E02C
:1005F800184A00E0164A0492149534E000ED00E031
:100608000005FA05001001400000014040420F00BB
:10061800C81A0020CC1A002010E000E0C800002012
:10062800D4110020B02A0020BC280020C8130020C4
:10063800C0280020A8C10108A9110020040A002030
:10064800CC2B0020E81100208CB7010814110020E1
:10065800789101086C91010800080140000C0140E4
:10066800FC2C00200493BBF10E0F04D00BF0EF0B11
:10067800BBF1080F02D101228DF84A200120059311
:1006880007F0FAFA059B18B14088003018BF01201E
:10069800C4F340028DF83E20C4F3403200F001005C
:1006A8008DF83820C4F3C0328DF83D008DF84080B5
:1006B8008DF83B20B9F1000F07D096F8869109F123
:1006C800FF3EDEF1000949EB0E09003318BF012394
:1006D8008DF842307B6AB6F84801003318BF012311
:1006E8008DF84330C4F300538DF84430B6F84A31DE
:1006F800E504ADF84830B6F85631ADF84E0048BFBD
:10070800BA48ADF84630C4F3804348BFB0F850014A
:100718008DF83F30B6F8543148BFADF84E00B3F508
:10072800FA7FADF84C3084BF0023ADF84E3096F810
:10073800D631AF4887F82830002387F8293043702E
:100748009DF84A30C4F30042002B8DF8412004F094
:100758000101C4F3C0028DF83C908DF839108DF872
:100768003A200CBF0023022301B902B101330AEB7E
:10077800830ADAF838304FF00008A3F102091A3377
:1007880005934FF6FF7339F802AF9A4500F0788168
:100798009DF83D205FFA8AF31AB19A1E012A40F2A9
:1007A8006B819DF8402032B192491A018958924ACA
:1007B800914200F061819DF8412032B18D491A01C2
:1007C80089588D4A914200F057819DF83E2052B1D8
:1007D800884A039802EB03125168814203D11289B7
:1007E800102A00F049819DF83B2052B1814A0398B4
:1007F80002EB03125168814203D11289022A00F0E8
:100808003B819DF83C2052B17A4A7C4802EB0312A6
:100818005168814203D11289022A00F02D81149A6D
:100828007AB1744C116804EB03146068884208D1EB
:1008380021899088884200F01F81D2888A4200F07E
:100848001B814FEA1A2ABAF1020F02D19DF838200B
:1008580004E0BAF1010F04D19DF83920002A00F014
:100868000B81DFF890B19DF844101F010BEB0704D2
:100878005A4631B19DF84A1019B9043B032B40F28E
:10088800E380BAF1010F5FFA8AF341D15C4D3A4433
:10089800FF23517B85F8703085F87130506802F17C
:1008A800080312890026ADF854208DF8561002224C
:1008B80015A985F87460C5F8804006938DF857200F
:1008C80085F82C602E636E63AE63EE6685F8726001
:1008D80085F873600CF0B0FA069B5BF8070099780E
:1008E80032460CF05DF92046314652460AF03EFD8C
:1008F800444BC5F88C60C5F88430434B2046C5F896
:10090800883005F1840105F188020AF077FDB3E02B
:10091800022B46D15FFA88F21C2101FB02FC384AFF
:10092800002502EB0C06334A4FF0010A3A44517B8A
:10093800506802F1080B128986F875808DF85610F8
:1009480086F8765015A986F87E5086F874A0C6F801
:100958008040CDF818C0ADF854208DF857300CF011
:100968006BFA244B9BF80210D8592A460CF018F958
:100978002046294652460AF0F9FC244A204BDDF865
:1009880018C0C6F8842003EB0C01214A8431C6F84C
:100998008820C6F88C5020460A1D0AF02FFDD04446
:1009A8006AE0032B4ED19DF83F30154D194E3BB1EF
:1009B80095F82A70204608214FF6FF72002335E08B
:1009C800BDF84C2095F82A70B2F5FA7FBDF84E3084
:1009D80026D911492046B1FBF2F2082192B20CF057
:1009E8001FFB0E4B46F8270025E000BFD41100205E
:1009F800F10000201CB4010800040040000C014074
:100A0800C800002015CA0008F5CA0008E5CB000890
:100A1800EDC90008802A002000127A0015CB0008D2
:100A280067492046B1FBF2F2012192B20CF0F8FAC4
:100A3800644B46F82700C36095F82A30013385F8DF
:100A48002A3019E0042B17D1BDF846205C4B5E4DC7
:100A580093FBF2F22046BDF84830012192B295F896
:100A680029600CF0DDFA95F8293005EB860601338C
:100A7800C6F8540185F82930059B99457FF481AE65
:100A8800514D524B95F82920002485F87421504A7D
:100A98001C7017789846A7F11702022A19D82B6AF2
:100AA8000021185903EB040912F04EFC10B16B6ACF
:100AB80063BB26E0474E99E80F00264486E80F00FE
:100AC80098F8003010340133C02C88F80030E6D193
:100AD800EDE7414B13F8376003EBC703D3F804E0A5
:100AE80088F80060BEF1000FE1D0B442DFDA394A7D
:100AF800230103EB020C73440FCB01348CE80F0085
:100B0800F3E7364E3368DC0424D41DE0344B354A11
:100B180013F8370003EBC7035C681070002CF0D0A3
:100B280000238342EDDAC3EBC3016218D2F800C098
:100B3800DFF8BCE0013341F80EC001EB0E069188E6
:100B4800B1809279B271ECE707F0EF03082B264BDE
:100B580025D126E098F80030012BF5D9234C04EB79
:100B6800031303F1100810344445EDD054F8100C69
:100B78004FF07C5112F054FA4FF07C5144F8100CAD
:100B880054F8140C12F04CFA4FF07C5144F8140C41
:100B980054F80C0C12F044FA44F80C0CE3E70E2F4E
:100BA80008D11A78182F42F010021A7022D10FF0CB
:100BB8004FFC1FE01A78192F22F010021A70F5E77F
:100BC80040420F0005CB0008C80000207F2A002003
:100BD800040A0020400900208CB70108FC2C0020E2
:100BE800249C0108582B0020C8190020480900201F
:100BF800592B00200FF010FC3368DFF81CB35803A2
:100C08005EBFBA4B01221A70B94A0DF15409137824
:100C1800B84F43F004031370B74B4FF0100A93E832
:100C28000300DBF8183089E8030043F00803CBF829
:100C3800183016A915980CF0FFF801200AF004FEE8
:100C48003468524604F400430393384604F40063BE
:100C58000021059315F0A1FF4FF6FF72ADF834207F
:100C680002224FF0000814408DF836208DF83780A6
:100C78000DD020A921F84CADA0480EF06FFC04233C
:100C88003B700124072387F80180BC70FB70039B2D
:100C980073B1022320A921F84C3D98480EF05EFC60
:100CA8000123E2183B71BB7107237C71FB71D4B23D
:100CB800059B7BB1022320A921F84C3D90480EF0FA
:100CC8004DFC092301223B73BA73631C07227C7312
:100CD800FA73DCB2DBF804308A4843F44043CBF8BB
:100CE8000430DBF814304FF0000843F00103CBF870
:100CF8001430DBF81830DFF80CA243F40073CBF89B
:100D080018300EF03FFA804B012C15937F4B494663
:100D1800169394BF434680231A934FF480731B9312
:100D28004FF480631C9320231D9350464FF40053C7
:100D380018941E93CDF85C80CDF86480CDF87C8043
:100D48000EF002FADAF80030714A43F00103CAF8EB
:100D580000305368012C23F4702394BF0021012133
:100D680023F4807343EA012353609168694B013C83
:100D78000B4043F4602343F002039360D36AE4B268
:100D880023F4700343EA0454D462012307EB0802F6
:100D9800917800295CD017F80800591C0928C9B2B5
:100DA800D278DFF86CE111D9A0F10A04DEF80CA0C2
:100DB80004EB44044FF0070C0CFA04FC2AEA0C0C70
:100DC800A2404CEA0202CEF80C200EE0DEF81040F9
:100DD80000EB400C4FF0070A0AFA0CFA24EA0A045E
:100DE80002FA0CF22243CEF81020062B484C0ED8FB
:100DF800013B626B03EB83034FF01F0E0EFA03FEF9
:100E080022EA0E0200FA03F3134363631FE00C2B7C
:100E18000ED8073B226B03EB83034FF01F0E0EFA2D
:100E280003FE22EA0E0200FA03F3134323630EE0E3
:100E3800A3F10D02D4F82CC002EB82021F239340C9
:100E48002CEA030E00FA02F34EEA0303E3620B46B0
:100E580008F10408B8F1100F98D12D4B9A6842F4A4
:100E680080729A609A6842F001029A609A6842F029
:100E780008029A609968264A09074FD5FAE7013AA5
:100E8800092A3FF638ABDAF85400C8F81430294676
:100E98002860039804930BF0CFFF039B3C201A466D
:100EA8000823136107F015F9049BC8F81030D846D9
:100EB80096F893319845BFF618AB114B4FF0080BD5
:100EC800C3F810B00493039B7820C3F814B007F05C
:100ED800F5F8049B7820C3F814B0039B08F10108C7
:100EE800C3F810B007F0EAF8E2E700BF700E002080
:100EF800C03000201C290020B491010800080140DE
:100F0800000C0140080002404C2401402C2900201C
:100F180000240140FDF7F1FF00100240936843F000
:100F280004039360AB4B9A6812F00408FAD1AA4FF5
:100F38009A68B7F85C0142F4A0029A60002841F070
:100F48006882B7F95E31002B41F06382B7F96031EE
:100F5800002B41F05E8233689B031FD5C82007F041
:100F6800B8F8AE200AF06BFC08B10CF0B3F99B4C52
:100F780085F87501C82007F0ACF8994B00210C22C0
:100F88002046C5F8783115F008FE0223E3700CF00E
:100F98003AFC07F077F8934B0344A36097F86B315A
:100FA800B7F864410593904B97F863B11B6897F8BD
:100FB8006C61B3F85630B7F80CA00693FB7B8B4FE7
:100FC80000210C228A48039315F0E7FD0021142222
:100FD800384615F0E2FD874B00221A700793C5F8D2
:100FE8007C2104F017FE079BDFF840921A4648B3AD
:100FF800814BB4F5807F3B60804B7B60804BFB600E
:10100800804B3B61804B01D1002116E0BB2C01D9FC
:10101800012112E0612C01D902210EE0292C01D90D
:1010280003210AE0132C01D9042106E0092C01D977
:10103800052102E0002CE7D0062119700123137066
:10104800022322E00790192007F043F815AB682027
:101058000F21012204F000FA9DF85430DDF81CC07D
:10106800D32B40F01983694B4E2C3B60684B7B6057
:10107800684B3B6100F00A835D2C00F00B83362C33
:1010880000F0028389F880C10123634A634F3B70F3
:10109800136843F0010313600022614BBBF1090F91
:1010A80000F2F680DFE81BF01000F40010000E00DC
:1010B80079000C000E000A000A00EA001A70D3E05A
:1010C8001A70BDE01A7019E01A704FF0000920ABD1
:1010D80003F82C2D53204946012204F0BDF968B1CC
:1010E8009DF85430E52B09D1414B4E4A85F8839140
:1010F8001A604D4A5A60022300F020BC4B4B002274
:10110800C3F87C2104F086FD002847D006210A4652
:1011180015AB682004F0A0F99DF8591001F0010200
:101128009DF8571001F001014B0043EA82019DF838
:10113800552002F001030B430BD05BB2012B01D108
:10114800002202E0022B0FD10122384B83F88421C0
:1011580011E00DAB68200C21012204F07DF99DF807
:10116800343013F00F0303D1032006F0BCFF02E074
:10117800042BE9D1E4E71E4B2D4A1A602D4A5A6028
:101188002A4A92F88421002A0CBF6F226E221A7212
:10119800234B01221A700323D0E31A70002220ABDC
:1011A80003F82C2D1C200D21012204F055F90028EC
:1011B80046D09DF854302A2B01D01A2B40D10C4A26
:1011C8001D4911601D495160184A82F88531042370
:1011D800B4E300BF00240140D4110020D41A002039
:1011E8005E130020404B4C0024110020942700205F
:1011F800C82C0020C4070020315900080D560008EB
:101208007752000890C1793D00000020FD59000880
:10121800EB560008325C8F3DC41900204C000020BA
:10122800E4300020595A000871570008C80000200F
:10123800FD5200084F5600089D59000891560008B5
:10124800002120AB03F82C1D1820012204F004F91A
:1012580050B19DF85430FB2B06D1C04BC04A1A60E0
:10126800C04A5A60052369E304F026FC38B1BB4B39
:10127800BD4A1A60BD4A5A6008235FE31A70B74B2B
:10128800BB4A1A60BB4A5A6000221A72092355E306
:10129800BBF1010F3FF618AF1A70042E00F23B8124
:1012A800DFE816F0050042016700050006010A2084
:1012B80006F00FFF7720A02101220DAB04F0CCF837
:1012C800002856D01E210122772004F0B5FA4FF4E9
:1012D8002F6006F0F3FE0025A5F160010026C9B2D3
:1012E800022215AB77208DF854608DF8556004F014
:1012F800B3F89DF854209DF8553043EA02239E4ADE
:1013080002F5C3716B520235102DE5D1B2F8940184
:10131800334600F00F0500F47F40A2F894013246EE
:101328000127954E22F001013144B1F886110029B8
:1013380018BF002712F0010F03D0C9B24B40082193
:1013480002E083EA1123FAE713F4004F18BF83F48D
:10135800C05301394FEA4303F6D10132102AE0D1D4
:101368002843A6F8940127B9C3F303339D4200F03C
:10137800EC82814D95F89631002B41F06A8014205B
:1013880006F0A7FE7720D02101220DAB04F064F807
:10139800002800F08D809DF834300322552B85F805
:1013A800AF31A5F8B82140F08380D12101220DABDF
:1013B800772004F051F89DF83430772003F00F02BD
:1013C8001B0985F8B02185F8B131162215ABAA2181
:1013D80004F042F89DF854209DF8553043EA022362
:1013E800A5F898319DF856209DF8573043EA022316
:1013F800A5F89A319DF858209DF8593043EA022300
:10140800A5F89C319DF85A209DF85B3043EA0223E9
:10141800A5F89E319DF85C209DF85D3043EA0223D3
:10142800A5F8A0319DF85E209DF85F3043EA0223BD
:10143800A5F8A2319DF860209DF8613043EA0223A7
:10144800A5F8A4319DF862209DF8633043EA022391
:10145800A5F8A6319DF864209DF8653043EA02237B
:10146800A5F8A8319DF866209DF8673043EA022365
:10147800A5F8AA319DF868209DF8693043EA02234F
:1014880041F27072A5F8AC313C4B1A8046F67812DE
:101498005A803B4A5A603B4A9A603B4ADA603B4A68
:1014A8001A613B4A5A61012385F8963100F0D1BF91
:1014B800314D95F8BC61002E40F05882142006F09A
:1014C80008FE05F2BD137620D021012203F0C4FFE7
:1014D80095F8BD31582B27D105F5E07388211822DE
:1014E800762003F0B9FF31227620F42104F0A4F924
:1014F8000123284A85F8BC31204B9A60264A1E8071
:101508005A6045F6D8125A80244ADA60244A1A6189
:10151800244A5A612AE2012E06D0234B234A9E70A0
:10152800136843F004031360204D2B689E0702D50F
:101538000A4B1B689847039BE4B20F4E1C4A002BCA
:1015480056D02B68B4BB40F2596113F0020F40F239
:10155800712318BF0B467D2135E000BFC82C002041
:10156800355A00082B57000865520008B353000885
:1015780001EE00081DEE0008C800002058060020F3
:1015880029590008E555000811590008A555000813
:101598008951000885510008875100080959000839
:1015A80059550008214F00084C000020C41900209C
:1015B800602D0020980759BF4FF47A7319464FF4ED
:1015C800FA634FF47A719A4505DBBAF57A6FA8BFCA
:1015D8004FF47A6A00E09A464B1E5344B3FBF1F38A
:1015E800013BDBB203FB011186F88231116005E093
:1015F8009DF80C30C2F800A086F88231BA4F3B68DB
:101608009847DDF81490B94C0023B9F1020F237004
:1016180006D0B9F1030F1AD0B9F1000F40F0A88134
:10162800002220AB03F82C2DC6F8DC211E200A214D
:10163800012203F011FF50B19DF85430482B06D118
:10164800AB4BAC4A1A60AC4A5A60022395E14FF0A2
:10165800000A20AB03F82CAD0C205146012203F000
:10166800FBFE002800F0F8869DF85430482B08D17E
:101678009F4BA24A1A60A24A5A6007232370032389
:101688007BE1504600F0E8BE402300E0802389F863
:101698008031F9E4C023FAE795F88171002F56D01C
:1016A800984B00221A80002F40F09380964A8021A0
:1016B80013886B2023F040031B041B0C1380138832
:1016C80023F038031B041B0C43F0300313801388EA
:1016D8009BB243F04003138004F08CFA962006F086
:1016E800F8FC0321682004F085FA962006F0F1FC46
:1016F80003216B2004F07EFA012006F0DFFC1021A4
:101708006A2004F077FA012006F0D8FC39466C20EC
:1017180004F070FA012006F0D1FC3946192004F0D3
:1017280069FA012006F0CAFC10211C2004F062FAB4
:10173800012006F0C3FC1B20182104F05BFA0120ED
:1017480006F0BCFC714B012283F8812141E06E4A0E
:101758006B201388802123F040031B041B0C13808B
:1017680013884FF0060923F038031B041B0C43F0C1
:101778003003138013889BB243F04003138004F0B6
:1017880039FA962006F0A5FC752015A9012204F067
:10179800D7F99DF85430682B05D009F1FF3919F0B5
:1017A800FF09EED10FE00C2015A9012204F0C8F9B9
:1017B8009DF85430142B06D3182B7FF671AF543B89
:1017C800062B7FF66DAF04F077F9474B002860D100
:1017D80080E0B4F5807F0ED0BB2C0ED8612C0ED8DB
:1017E800292C0ED8132C0ED8092C0ED8002C14BF77
:1017F800062700270AE0002708E0012706E002275D
:1018080004E0032702E0042700E005273E4A1920E8
:10181800138823F040031B041B0C1380138823F048
:1018280038031B041B0C43F03003138013889BB24E
:1018380043F04003138095F8821104F0DBF901208E
:1018480006F03CFC39461A2004F0D4F9012006F0D1
:1018580035FC15A804F09AF99DF95630294A013348
:1018680003D19DF95430013302D013889BB213B1D0
:1018780000231380A7E71C4B254A64201A60254AD9
:101888005A60254ADA60254A1A6106F022FCFFF7F9
:10189800FBBB234ABB2C1A60224A5A60224ADA60F0
:1018A8001E4A1A61214B01D901220EE0612C01D98F
:1018B80002220AE0292C01D9032206E0132C01D9BF
:1018C800042202E0092C03D905225A70FFF7DCBB79
:1018D8000622FAE7164A1A60164A5A60164A9A60A9
:1018E8000823FFF7D2BB00BF94270020E530002073
:1018F800340600209DB600081DB500082DB6000866
:1019080099B50008EC2C002000380040C8000020E1
:1019180075520008955B0008715B000890C1793D1D
:1019280011540008755300085153000800000020A6
:1019380007EE00082BEE000803EE00082C4A7B7027
:10194800136843F002031360A7E442F21072294BB4
:1019580003261A805A80284A5A60284A9A60284AD8
:10196800DA60284A1A61284A5A61D6E50426D4E57D
:10197800B9F1010F07D9994645E6244AD3702B6877
:1019880043F008032B60224A92F8583191460BB174
:10199800204A137099F859310BB11F4A137099F8FE
:1019A8005A3103B123702B68DFF878A013F0080FC1
:1019B8003AD0BDF918204FF0640B92FBFBF4204697
:1019C800059211F0D9FA059A03900BFB142000B286
:1019D80011F0D2FA114911F023FB039B0146184676
:1019E80011F016FA0E4911F01BFBCAF800001EE0B0
:1019F800C41900205806002001590008495500085C
:101A0800F958000839550008654D00084C000020B9
:101A1800D4110020C4070020E43000208988883CC5
:101A280000002041D82B00200023CAF80030A84C21
:101A3800102223784FF00A0B43F002032370A54BC2
:101A48005A6108221A610394A24C1920E3680BF129
:101A5800FF3B83F01003E360E36883F00803E3606F
:101A680006F037FB192006F034FB1BF0FF0BEBD117
:101A780008234FF0100B2361C4F810B02B68190726
:101A880009D5954BC4F814B01B689847934B0122AD
:101A9800C4F810B01A70924B924C1B68187B11F066
:101AA8006BFA914911F0BCFA08F082FB8346208852
:101AB80011F062FA594611F0B3FA15F07BFA8B4B24
:101AC8001880208811F058FA0146894811F05CFB0B
:101AD800884911F059FB884B83491860386911F01F
:101AE8009FFA864911F09CFA854F864BFF211860B2
:101AF8001B22384615F051F8002139702968824BAD
:101B0800012211F0020F1A701FBF7A7003221A7097
:101B1800022218BFBA704A0748BF1A78384641BF30
:101B2800551C1D700325BD5411F00A0F0CD01A78EE
:101B38000421B954511CC9B205257D54D11C023267
:101B48001970D2B20621B954704A11688F0641BF84
:101B58001A78551C1D70072548BF85540D0608D5F1
:101B68001A7809258554951C01321D70D2B20A25B0
:101B7800855499F80550082D01D00E2D04D11A78F6
:101B8800571C1F700B2787541A78CC0302F10107E2
:101B98004FF00C0E48BF5C4C00F802E0FFB248BFA3
:101BA80002321F7041BF2270554A4FF00E0E02F8E4
:101BB80007E04F0748BF1A784FF0120E41BF571C75
:101BC8001F70102787541A784C0502F10107FFB2DD
:101BD8001F7000F802E00AD599F818423CB14A4C47
:101BE80002322270464A4FF0130E02F807E01A78C4
:101BF8008C0502F101074FF0140E48BF424C00F863
:101C080002E0FFB248BF02321F7041BF22703C4A57
:101C18004FF0150E02F807E0182D0DD11A78162787
:101C28008754571CFFB24FF0170E00F807E0D71C77
:101C38000232D2B21F7085540D0341BF1A78551C69
:101C48001D70192548BF8554CC0541BF1A78511C11
:101C580019701A2348BF8354002198222C4814F085
:101C68009CFF0DF06EF92B4A2B4BB9F852111A60F4
:101C78002A4BB9F898011980294900230B808B70E9
:101C880028490A6081B2284A22F813100133122B1E
:101C9800F9D11E4F3B68D9045CBFB9F89E11118079
:101CA8001B0740F1EC8099F89251062D00F2E18073
:101CB800DFE805F004073E6984A2A20045F2F0526D
:101CC80001E042F6F822194B1A800DF0C3F9CFE073
:101CD800C0300020000C0140340600204C060020D3
:101CE800500800201A00002035FA8E3C6C080020AD
:101CF8000AE81C4100401C4680070020BD37863595
:101D0800ED1000204C080020EC100020FC2C0020D6
:101D1800182800205E130020A40F0020A80F002020
:101D28009430002088300020382D0020AC08002096
:101D380042F6F822784B1A8011F01EF9774911F013
:101D48006FF9774911F062F811F056FB0023754AD4
:101D580042F823000133122BF9D1734A734940200A
:101D68001160734A137006F061F8002800F0818052
:101D780001234FF0070C90F9000040218DE808106E
:101D88006C4A6D4B6FE042F6F822634B40201A8094
:101D98006A4A654B1A60664B10221A7006F046F8BC
:101DA800002866D001234FF0000E90F90000402172
:101DB8008DE80840624A4FF4E13354E042F6F822D5
:101DC800554B40201A805F4A574B1A60584B0822DF
:101DD8001A7006F02BF800284BD00123002590F943
:101DE800000040218DE82800574A4FF4E13306F0FF
:101DF800D0F9C6F8E00138E042F6F822464B4FF039
:101E08000C0E1A804A4B51485149524A83F800E057
:101E1800062D4FF00003504C03700B7013700AD05E
:101E28001B2323704D4B052283F800E04C4B4FF4E5
:101E3800E1351A7007E021232370484B83F800E04E
:101E4800474B1D70474D484A374B40201A6005F0F4
:101E5800EDFF70B10123002490F900008DE818000F
:101E68002B46424A402106F094F9003018BF012061
:101E780028B9082008F08EFA3D4A2B4B1A603B68B7
:101E88002B4A13F4804F1FBF082111703948264987
:101E980018BF086042F20101194099B144F6206068
:101EA8001D490880980441BF0821117032481E4915
:101EB80048BF0860D90741BF0C2111702F481A4943
:101EC80048BF086011781D06A1F10401517040F166
:101ED8009480DFF8BC902A4DC6F8E491002631467C
:101EE8001522284C28486E706E60AE6014F055FEBE
:101EF800A9F105033046236009F051F8234B02206D
:101F08001B68A246EB6005F091FF002842D18020B3
:101F180008F040FA69E000BFAC080020CDCCCC3F07
:101F28000000B044982F002030000020412A01080A
:101F3800B4280020E52B0108A08601002D2A0108FD
:101F4800392B0108192A0108ED2A010884300020DC
:101F5800F1270020F02700201328002083300020DC
:101F68001428002090D0030009EE000839EE00087C
:101F78009D2A0108712A01088D2A01087D2A010875
:101F88009C070020BC070020B0020020202D002064
:101F9800C813002046796B78BA490C2202FB031259
:101FA8005278B24204D00133DBB2042BF4D90023B7
:101FB8006B70DAF800306A781B7890F90000002B13
:101FC8004FF00C0303FB021314BF03260126002263
:101FD8005B7800960192022106F0DBF8AA4B1860A4
:101FE800002894D0012008F0DAFFA84B1868A84B05
:101FF80000F5C5721A6009F079F83B689C056CD544
:10200800A44AA54D049BA5482B6093690DA943F0EC
:1020180001039361049B1B88ADF8343010238DF8BD
:10202800363002238DF837300AF006FF2B689B48BC
:102038005B880DA9ADF8343004238DF836300AF0EA
:10204800FBFE28680F21037A03F0030203F0FC0368
:1020580003F1804303F580339D689200914025EA9F
:10206800010199609968012505FA02F20A439A600C
:1020780042688B4BD1435A611E680E401E605E68F1
:102088000E405E601E6816431E609E680E409E608D
:10209800DE683140D960996811439960D9680A436C
:1020A800DA60437A15A88DF8543003238DF855303B
:1020B80000238DF856308DF8575010F019F8794BE9
:1020C800794A1B683C3B1360784A136843F0100355
:1020D8001360774B4FF0FF321A60764B764A774D94
:1020E8001360774A803313603B680026D8032E704C
:1020F80040F1AA8040F22A3ADFF8F4B1654C0EF0BC
:10210800E9FA4FF0010952465846314685F80090E1
:1021180014F043FDA3696B4843F00403A361402313
:10212800ADF8303018238DF833300CA903238DF81F
:1021380032300DF013FAE369634943F00203E361B7
:10214800624B634D1B68A4F69474B3FBF1F32988C2
:10215800013B21F45C710904090C29809BB21D2103
:10216800A9852B85A5F814902B8C23F001031B045B
:102178001B0C2B842B8CA888298B23F0020321F0BD
:10218800730109041B04090C1B0C41F0600180B2A7
:1021980043EA0903A8802983AE862B842B8B23F07E
:1021A80008031B041B0C43F008032B83B5F84430C9
:1021B8006FEA43436FEA53439BB2A5F84430D4F81F
:1021C800A83F43EA0903C4F8A83F20460CF0DAFF09
:1021D800404BCDF858B0159380231A934FF4807371
:1021E8004FF0100B1B9320464FF4005315A91E9374
:1021F80019961C961D961F96CDF85CB0CDF860A078
:102208000CF0A2FFAB890DA89BB243F40073AB811D
:10221800236843F0020323608DF834B08DF83590BD
:102228008DF836608DF837900FF062FF2A4B1A68E8
:102238002A4B43F8282008F10108B8F1200FF5D1FE
:102248000AF01CFD0AF01AFD3B68590540F1908020
:10225800234D244BD5F828A50420C3F800A005F089
:10226800E5FD0421C5F82C0505F0BCFD1E4B85F8DD
:1022780030050820C3F800A005F0D8FD1B4B082145
:10228800186037E030920108D01A0020241100208D
:10229800001000200010024098070020000C0140A8
:1022A80000040140202D002094070020C4190020BC
:1022B80044110020FC130020181B0020710E002080
:1022C800141B00200008014000366E015000002059
:1022D8000004004034040040BC910108720E002044
:1022E800C8000020B8190020101A00205C1A00202D
:1022F800C502002005F076FD5C4E85F83105002109
:1023080030462C2214F049FC8E2373704FF07C0960
:10231800E0234FF07D08F37086F8009086F82B8054
:10232800534E2C220021304614F037FC8A23737058
:102338001020A023F37086F8009086F82B80C5F84B
:1023480034A505F073FD1021C5F8380505F04AFDE0
:1023580085F83C052020C5F840A505F067FD20213B
:10236800C5F8440505F03EFD85F848050BF022F94F
:102378003B68404A13F4002318BF0123137005F08B
:1023880081FE3D4B18603D4B5A79052A02BF3C4AF5
:102398004FF4C87111803B4A4FF47A7111803A4A60
:1023A800C821118039490A7842F008020A70384970
:1023B8000A7822F002020A7040F6020239680A40DE
:1023C8006AB13448344A1060344A03201070344AE1
:1023D80001201070334800220280334802808A03AB
:1023E80042BF324A042111719B6848BFD1783B60D3
:1023F80048BF41F001012E4B48BFD17001221A702D
:10240800039B039A1B7863F07F03137021B0BDE828
:10241800F08F284B00221A7000B210F0ADFD26494B
:1024280010F0FEFD1590B7F95E0110F0A5FD2249E8
:1024380010F0F6FD1690B7F9600110F09DFD1E49E9
:1024480010F0EEFD1D491790484607F0BBFEFEF759
:1024580082BD0226FFF761B8B9F1010F7FF693AA92
:102468004FF000092070FFF7DBB800BFE01900202B
:10247800151A00205C2D00208C080020D4110020A3
:10248800B60F0020DE300020DC300020C819002004
:10249800E730002050130020B0190020141A002043
:1024A80044000020A0100020A2100020D41A002010
:1024B800700E00203800002035FA8E3CF8280020E5
:1024C800954A2DE9F04F1568944C05F59C43944EB8
:1024D80020332360336889B013F4804F059205D107
:1024E80010F046FC10B92379013323718D4A137813
:1024F8004BB18D4909688D4240F2E58003F1FF3800
:1025080082F80080DFE09846884B5FFA88F51F78EC
:10251800DFF83892AF4231D9D9F80030072D98BF8B
:10252800595D834B88BF29461B6880489847032D0F
:102538001ED8D9F8002005F10E0302EB8303998811
:10254800DA88A8B14FF47A73401A5843531A90FBAB
:10255800F3F040F6C90300F57A70984205DC40F2C2
:10256800EE239842B8BF184601E040F6CA0080B290
:1025780004EB4505E88008F10108C5E794F80480F4
:102588000325B8FBF5F50F2384F82A3094F82B308F
:1025980005EB4505019394F82C30C5EB080503932A
:1025A800D9F80030DFF8ACA10293EBB20493002510
:1025B800BD4255DA5F4B4FEA450933F815B0019B28
:1025C80053B910F0D5FB28B1039B002B08BF4FF07F
:1025D800000B01E0DDF804B0029B988A584502D848
:1025E800D88A58450ED2E8B210F06CFB032D83460A
:1025F800DFBF94F82AE00120A8402EEA0000D8BFE7
:1026080084F82A0010F0B4FB18B14B4829F800B040
:1026180022E0049B94F876002AF813B030B9B8F198
:10262800020F15D93D4B012083F87600BAF8000057
:10263800BAF802300344BAF8040003443F489BB296
:1026480029F800301BB2032093FBF0F39BB200E0A3
:102658005B46394829F8003001350AF1060AA7E730
:1026680094F82A203648A2F10F014A424A4184F8D8
:102678009020344B6AB1344A1268520109D4026876
:10268800D9689A60521AC82A1DD9012283F82120D4
:1026980019E002689868DA605B68121A9A4288BF83
:1026A800284B4FF0000184F82B1088BF83F82110C5
:1026B8000025BD4207DAE8B210F004FB1E4B23F8F0
:1026C80015000135F5E73368DD0405D51E4B1B6899
:1026D800D80701D410F054F9059B1F681B4B1A68E2
:1026E800907A002838D01449137B013831F810004B
:1026F8001BB1C0F53B60083080B200B2A0F57A701B
:10270800B0F57A7FA8BF4FF47A7020EAE07010F035
:1027180033FC0F4955E000BFCC300020F80E0020F4
:10272800FC2C0020903000208C300020B4280020A1
:1027380030000020FE0E0020382D0020700F0020F1
:10274800202D002094300020E81000208830002040
:1027580000007A44260F0020336819043AD5D4F8CB
:102768009430934DFB1A002B34DB07F59C43203340
:10277800C5F894308F4BD27A59798F4B33F8113092
:1027880095F898109BB293FBF2F3013101F00F0218
:1027980085F898202A4482F899300346874A825C53
:1027A8000130134410289BB2F8D11BB293FBF0F010
:1027B80000B26428A8BF642020EAE07010F0DCFBB7
:1027C8007F4910F0E1FC7F4910F02AFC10F014FE5C
:1027D8007D4B188033687D4D13F4807F00F00F81A6
:1027E8007B4BDFF8F0919F4205D999F8022012B986
:1027F800012289F8022099F80220002A00F0FF80BF
:10280800744A95F8008092F82170C8F380087A1EFF
:1028180057425741704A002F9246116818BF4FF02F
:10282800000BC1F38063019308BF4FF0030B99F8C5
:102838002020052A00F2DD80DFE802F0034E5379FC
:1028480088A5B8F1000F3AD0D4F8AC00B4F8B010AD
:1028580005F089FB012809D16049614A09681268B5
:10286800C988642000FB0122C9F81020019B6BB1C4
:102878005A4A126812794AB10CF08AFA032289F886
:1028880020204FF47A72C9F81C20D0E7002F40F0BE
:10289800B080534AD9F8101010684E4A88420AD9B5
:1028A80002920CF075FA029A032182F8201040F681
:1028B800B831D161BBE7012182F82010B7E7019B4D
:1028C8004FF4806013B107F055FD01E007F041FDBA
:1028D8000022C9F810208CE0002F49D10CF058FADA
:1028E800A5E727B1052289F82020012000E0384615
:1028F800B8F1000F0CD0D4F8AC204FF0020BD189FE
:10290800384A118051809180344909684988D180BA
:10291800334A1168D9F81420914202D8B8F1000F4F
:1029280064D147F23052C9F81C20032221E02A78EA
:1029380042F002022A7010F023F8294AD9F81C1034
:1029480012680A44C9F81820042212E0244A9FB1E8
:102958001168D9F8182091424BD9234A12781AB92C
:10296800DAF80020D30744D42A7822F002022A7029
:10297800052289F820205AE71268D9F81C100A4461
:10298800C9F8182035E01549154A09681268C98838
:10299800642000FB01224FF48060C9F81020002257
:1029A80089F8202089F8032007F0D3FC3FE700BF0F
:1029B800F80E00201C2900202C290020910F00204F
:1029C8000000C84200C07F4448110020E7300020C2
:1029D800404B4C0094300020E8100020CC27002009
:1029E800202D0020382D00201800002000287FF41A
:1029F8001EAFBBF1000F02D0584605F009FB934FFC
:102A080007F5C570B7F8521105F0ADFA019783467E
:102A180068B90CF0AFF98E4B0022C3F800B0C3F8C8
:102A280004B0C3F808B08B4B1A605A609A602B78D0
:102A38005F0736D53368D80633D5874B1B78D90658
:102A48002FD4864B1B789BB1019B93F8E231BBF1E5
:102A5800000F15D17BB1824B1A68D4F8B4309B1A99
:102A6800002B08DA0FF08CFF7E4B83F8B8B018E023
:102A7800BBF1000F0DD1102005F0CAFA01230EE0BA
:102A88003BB1774A4FF47A71126801FB0323C4F80B
:102A9800B43094F8B83023B105F0A8FA002384F8CC
:102AA800B830019B93F8E0A193F8E111B3F89AE1EB
:102AB800B3F89CC1002318466B4F800837F91320E0
:102AC80001337245C4BF60F07F00C0B26245B8BF31
:102AD80040F04000042BB946EED194F8B930614A71
:102AE800834205D192F8BA30F92B04D8013300E0BB
:102AF800002382F8BA30594B84F8B9001A785B4F32
:102B08009846E2B93B68DA0708D5BBF1000F16D141
:102B18002B78DB0713D50FF08FFD10E02B785807C3
:102B28000DD5504B93F82B304BB1514BDB7833B963
:102B380011B10FF025FF02E0BBF1000FF9D094F8B6
:102B4800BA30484A142BDFF83CB140F0AD8098F811
:102B580000301AF1000A18BF4FF0010A6BB392F85F
:102B6800B9305F2B11D12B7803F0040303F0FF0178
:102B780013B10FF005FF08E00B200391029205F056
:102B880047FA029A039982F8BA10BAF1000F14D0E2
:102B980094F8B9307D2B10D12B7803F0040303F09F
:102BA800FF0213B10FF0ECFE07E00B20029205F0D4
:102BB8002FFA2C4B029A83F8BA202B7803F00403DF
:102BC80003F0FF01002B6FD194F8B930254A572B39
:102BD80015D1284B4FF47A721A803368190601D53B
:102BE80008F0D4FA244B1B685A0742BF234A0A212B
:102BF800118013F0080357D1214A138054E030683C
:102C0800400717D55A2B15D192F8BB302BB10123A9
:102C180082F8BB1082F8BC3046E092F8BD3083F0F1
:102C2800010382F8BD300BB10C2000E00D2005F047
:102C3800EFF939E05D2B00F018855B2B00F0178564
:102C48005E2B21D1032000F013BD00BFD41100205A
:102C5800E02900205C2A0020C81900201800002064
:102C6800202D0020F80E0020382D0020E81000202C
:102C780094300020DE300020C4190020DC30002011
:102C8800C411002024110020562B03D1029307F011
:102C98001DFE029B98F80020002A00F0FF846F2B8D
:102CA80040F0F6840FF0C8FC3368580736D594F81E
:102CB800BD30B64A93B12B7859070FD5019BB9F9A6
:102CC8000610B3F89A31994208DD3B6813F0010306
:102CD80002BF3221A2F8C01082F8BD303B68DA0387
:102CE8000DD594F8C220A94B2AB993F8BB2012B984
:102CF8003222A3F8C020012384F8C2300EE094F8F1
:102D0800BB30A24A53B12B7803F0040303F0FF0150
:102D180023B9012382F8BB1082F8BC30DBF800909D
:102D280000233B6009F17B0809F1CB0A98F80020E1
:102D380098F8013018F8010C9A420BD2414605F078
:102D4800DDF838B118F8022C012303FA02F23B68C7
:102D580013433B6008F10408D045E7D18C4B1B783E
:102D680053B18C4B8C4F1A68984612F0020FDFF85B
:102D7800409240F032832AE309F1CA0709F58978BD
:102D88003A787B7817F8010C9A4225D2394605F033
:102D9800B5F808B397F804E00C21BB7801FB0E41A5
:102DA8007E4A013B03EB43031344D1F8C82097F84C
:102DB80003909A4275480FD0C1F8C830002390F8A4
:102DC800F420C1F8CC30012303FA0EF322EA0303FE
:102DD80081F8C49080F8F43006374745D0D1704B5D
:102DE800DFF8D0A1D3F800806E4B4FF0000B1B68C2
:102DF800029394F82B300393DAF80030002B00F09C
:102E0800DD8293F80090B9F1000F00F0D782DAF86C
:102E1800042002998A1A002A0CDB01F5FA72CAF812
:102E2800042094F8F410012202FA0BF221EA0202BB
:102E380084F8F420039A002A00F0C0821AF8042CBF
:102E480059780432D2B2002940F07982564931F9D2
:102E58001210564AB2F8982102F1C800814201DDE9
:102E68009F7814E0C83A914202DA99784F420EE00E
:102E780094F8F420012303FA0BF322EA030384F8FD
:102E8800F430029B03F5FA73CAF8043096E294F81A
:102E9800F43043FA0BF3DB0700F19082002FCCBF2C
:102EA8000220012005F0D6F809F1FF32374B132A2A
:102EB80000F27C82DFE812F01400230032004400A4
:102EC80061008000E5004A01AF01E40113027A02C3
:102ED800440055008000E5004A01B7001C0181014B
:102EE80098F8001040460F44FA2FA8BFFA2727EA9F
:102EF800E77788F8007004F0E7FF01201EE098F8F3
:102F0800011040460F44642FA8BF642727EAE777DB
:102F180088F8017004F0D8FF02200FE098F8031039
:102F280040460F44642FA8BF642727EAE77788F84C
:102F38000370D3F8F81004F07FFF03203946CBE183
:102F480098F805100D2039446429A8BF642121EAA6
:102F5800E17188F8051005F035F8B9F10D0F00F0AA
:102F6800258298F804100E2039446429A8BF6421EA
:102F780021EAE17188F80410AEE198F806100520FE
:102F8800394481F3080188F80610A5E1F80E0020FD
:102F9800E8300020E8100020C419002074930108CC
:102FA8004C110020202D0020382D0020D4110020A5
:102FB8008C1A0020C00F0020D3F8FC301A78022A9F
:102FC80022D1384604930FF0D7FFA94910F0DCF856
:102FD800049B596A05930FF01BFF0021049010F021
:102FE800BDF9059B48B9049AA249104610F0D4F9D6
:102FF800049A059B10B19F4A00E000225A620F20F4
:10300800114604F0CBFF0AE099780F203944C8290B
:10301800A8BFC82121EAE171997004F0D3FFB9F182
:103028000F0F00F0C381944BD3F8FC9099F800304F
:10303800022B1AD138460FF09FFF8D4910F0A4F8E3
:10304800D9F820100FF0E4FE0021074610F086F9A9
:1030580030B93846874910F09FF910B1854F00E024
:103068000027C9F82070122059E199F801101220A0
:103078003944C829A8BFC82121EAE17189F801109B
:103088002AE1D3F8FC301A78022A22D13846049370
:103098000FF072FF774910F077F8049B196B0593CE
:1030A8000FF0B6FE0021049010F058F9059B48B9BE
:1030B800049A7049104610F06FF9049A059B10B1F4
:1030C8006C4A00E000221A631020114604F066FFE3
:1030D8000AE0197B10203944C829A8BFC82121EA71
:1030E800E171197304F06EFFB9F1100F00F05E8101
:1030F800614BD3F8FC9099F80030022B1AD138466E
:103108000FF03AFF5B4910F03FF8D9F82C100FF098
:103118007FFE0021074610F021F930B9384655499D
:1031280010F03AF910B1534F00E00027C9F82C709D
:103138001320F4E099F80B1013203944C829A8BFCC
:10314800C82121EAE17189F80B10C5E0D3F8FC30F9
:103158001A78022A22D1384604930FF00DFF474906
:1031680010F012F8049BD96B05930FF051FE002163
:10317800049010F0F3F8059B48B9049A3D491046AD
:1031880010F00AF9049A059B10B13A4A00E00022AF
:10319800DA631120114604F001FF0AE0997D11203D
:1031A8003944C829A8BFC82121EAE171997504F0FA
:1031B80009FFB9F1110F00F0F9802F4BD3F8FC90FB
:1031C80099F80030022B1AD138460FF0D5FE2B495A
:1031D8000FF0DAFFD9F838100FF01AFE0021074671
:1031E80010F0BCF830B93846224910F0D5F810B1C3
:1031F800204F00E00027C9F8387014208FE099F8B4
:10320800151014203944C829A8BFC82121EAE17142
:1032180089F8151060E0D3F8FC9099F80030022B7B
:103228001AD138460FF0A8FE11490FF0ADFFD9F8B2
:1032380028100FF0EDFD0021074610F08FF830B987
:1032480038460C4910F0A8F810B10A4F00E00027E2
:10325800C9F82870092062E099F803100920394458
:10326800C829A8BFC82121EAE17189F8031033E011
:10327800000020410000C842F80E002000007A44F7
:10328800D3F8FC9099F80030022B1AD138460FF089
:1032980073FEB4490FF078FFD9F834100FF0B8FD79
:1032A8000021074610F05AF830B93846AD4910F0F9
:1032B80073F810B1AB4F00E00027C9F834700A204A
:1032C8002DE099F80D100A203944C829A8BFC82153
:1032D80021EAE17189F80D1004F074FE66E0D3F874
:1032E800FC9099F80030022B1DD138460FF044FEAF
:1032F8009D490FF049FFD9F840100FF089FD0021D2
:10330800074610F02BF830B93846964910F044F8C3
:1033180010B1944F00E00027C9F840700B203946DF
:1033280004F03CFE42E099F817100B203944C829F4
:10333800A8BFC82121EAE17189F81710CCE7012953
:1033480034D19878894B33F91230B3F5617F05DBB6
:1033580040F633029342A8BF134601E04FF461736D
:10336800B9F10C0F22D14FF4966292FBF0F0A3F55D
:10337800617393FBF0F37E4ADFB21378BB4215D03A
:10338800042F34BF3B4602231370019A09FB032321
:10339800784A03F2B27313600EF014FB48463946BC
:1033A80004F010FE781CC0B204F054FE94F8F42027
:1033B800012303FA0BF3134384F8F4300BF1010BE8
:1033C800BBF1040F0AF10C0A7FF416ADC9E43368A7
:1033D800D80510D5684BDB786BB13B6899070AD5DF
:1033E800B9F8003013F0010A0AD10BF0C3FC012030
:1033F80006F0C0FF04E0012006F0ABFF012300E067
:103408000023D8F8002052070DD563B1012006F03B
:10341800A0FFB9F800309B0708D40BF0ABFC0220E2
:1034280006F0A8FF02E0022006F093FFB9F800308A
:10343800524A13F0030F4FF0100114BF516111618C
:103448003A6812F00A0F27D0D8F80020D00609D51C
:1034580059070AD4042006F08DFF494B1B88A4F8AD
:10346800003102E0042006F074FFD8F800309A0614
:1034780007D5B9F800305B0606D4402006F07AFF7D
:1034880002E0402006F065FFD8F80030580642BF39
:103498003B4B1B88A4F802313B68990609D4D8F83D
:1034A80000301A0540F1B0804FF4807006F062FFDA
:1034B800AEE0344B1B789B076ED5334B1B78042B3F
:1034C8006AD9D8F8003013F4007A0FD0B9F8003070
:1034D800DF063AD4102006F04DFF202006F039FF11
:1034E8002A48011D07F0BCFD02232AE0B9F8007044
:1034F80007F01007BFB22FB1102006F02AFF0127EE
:1035080084F804A1D8F80030580512D5D4F8083149
:103518001F495A89B1F90030002BB8BF5B4293426A
:1035280007DAB1F90230002BB8BF5B429342C0F210
:103538000581B9F80030990608D5202006F009FF62
:10354800002384F80431012700E0002794F80C31A7
:103558009BBB0E2004F05CFD0E4B012283F80C216E
:103568002BE000BF0000C84200007A44382D00203C
:10357800A82C00204C11002094300020000C0140A1
:10358800C4110020C8190020CE19002054110020B1
:10359800CC110020F80E0020B9F8003003F03003F9
:1035A800002B3FF47CAF102006F0D3FE202006F05D
:1035B800D0FE002384F8043102E0002F3FF46FAFFF
:1035C800002214466A4B002023F81400694B191D89
:1035D80003F10A0721F814000021D151174478603B
:1035E800B96023F8140003F132075A33D151D1508E
:1035F800174413447860B960586099601432002CFD
:103608007FF44DAF0124DDE74FF4807006F0A1FE92
:10361800594B5A791C46082A01D00E2A02D140205B
:1036280006F097FE33685A0540F19E8094F81832E8
:103638001BB92B7813F0040F03E0D8F8003013F40B
:10364800002F0BD04D4B00221A703C200BF04AFD86
:10365800002800F089800DF0BBFEF6E709F0AAFF0C
:1036680009B0BDE8F04F0BF06CBC012000E002206F
:103678005FFA80F8019A08F1FF3382F8B03706F054
:10368800BBFE06F05FFF404604F0E4FCFFF70CBB0E
:10369800BAF1000F02D07E2B3FF404AB972B05D173
:1036A8004FF4C873A4F8BE30FFF7FEBAA72B06D1B3
:1036B800334A137843F004031370FFF7F5BA002276
:1036C800BB2B079201D1022303E0B72B04D14FF69D
:1036D800FE73ADF81E3009E0BE2B01D1022303E0D2
:1036E800BD2B1AD14FF6FE73ADF81C30DBF8003055
:1036F800BDF81C10B3F858200A44A3F85820BDF8A8
:103708001E10B3F85A200A44A3F85A2007F0DEF82E
:10371800002384F8BA30FFF7C7BA792B04D1194AC5
:10372800D37823F0010306E07A2B7FF4BDAA154A6B
:10373800D37843F00103D370FFF7B6BAB9F8003075
:103748009B063FF503AF202006F014FE0E4B0F48F2
:103758001A685B68011D4360026007F081FC0C4B2E
:10376800012783F80471F1E609B0BDE8F08F00BFC6
:10377800E030002006100020D4110020B9280020D5
:10378800C8190020D41A0020D01900205C1100208C
:10379800F80E0020B54B2DE9F04FB3F90610B44BE5
:1037A80085B01F6801937A8991420EDBB1F5FA6FF3
:1037B800FC79BFBF8B1A6343A2F5FA6493FBF4F458
:1037C800ACBFC4F16404643400E06424A94BAA4A81
:1037D800B3F898B193F9623112689BB20292154618
:1037E8000393002240F2E630A04B4FEA420C33F933
:1037F80012E0CBEB0E0303F2F316864203D8002B3C
:10380800B8BF5B4201E04FF4FA73022A2ED0029E41
:1038180096F811611EB1B342CCBF9B1B00236420F4
:1038280093FBF0F8954E6FF0630A36F818900AFB90
:10383800083A08F1010836F918600FFA89F8C8EB58
:10384800060606FB0AF696FBF0F68D484E4420F86D
:103858000C60BE183679642073438A4E93FBF6F3E6
:1038680064339BB2634393FBF0F02CE0029890F82A
:1038780012611EB1B342CCBF9B1B0023642093FB93
:10388800F0F0DFF82C926FF0630808FB003A39F982
:103898001060013039F91000002BA0EB060000FB86
:1038A8000AFA9AFBF8FA0398C6EB0A0A0AFB00FA26
:1038B8007348B8BF5B42A0F804A0B8794343714885
:1038C80093FBF0F064306B784FF06408434393FB4C
:1038D800F8F36D4E022AB354EB7A6C4E00FB03F3F7
:1038E80093FBF8F3B3546B7D654E00FB03F090FB3C
:1038F800F8F0674B9854674B0ED1DE4583F8028089
:103908000DDB5C4CB4F89A21914214DBB1F5FA6FE7
:10391800A8BF4FF4FA610FE0DE459C5404DA36F88C
:103928000C305B4226F80C300132032A05F1010500
:103938007FF458AFE5E71146891A4FF47A73594373
:10394800C2F5FA62B1FBF2F1642391FBF3F2DFF8FE
:1039580074E16FF063073EF8120007FB02110132B1
:103968003EF9122007B2D21B514391FBF3F30344F3
:10397800F380494B424D1B885F063BD5474A484B6D
:1039880010881B88181A00B20FF0F6FA45490FF094
:1039980047FB074606F00CFC8046384606F095FBC8
:1039A8000746B5F902000FF0E7FA8146B5F90000BD
:1039B8000FF0E2FA414682460FF032FB3946834661
:1039C80048460FF02DFB014658460FF01FFA0FF03E
:1039D800EDFC4146288048460FF022FB39468046D8
:1039E80050460FF01DFB014640460FF011FA0FF04C
:1039F800DDFC68802C4D2B68980740F19E8045F2CD
:103A080007212A4B2A4F1A687B69D31A8B4240F345
:103A180094807A610BF010FF264BDFF8AC901A788F
:103A28009846032AB9F8003050D10A2B58D90023F8
:103A3800282088F8003004F04CFB0BF0FDFE1E4BEC
:103A480018880BF0E3FE1D4B1A68D37890FBF3F04F
:103A5800013008281A4BA8BF08201870537980B283
:103A680043433B8313795843788339E0382D00204A
:103A78004C110020D411002024110020AA1A002083
:103A8800CC1100200CFEFFFF682A002096100020B1
:103A98007C2A0020C02900208C1A0020FA0F002060
:103AA800C411002035FA8E3CFC2C0020CC300020BC
:103AB80088100020141A002034290020B019002092
:103AC80044000020921A0020B41900200A2B07D8BD
:103AD8000323964A88F80030002313703B837B83C6
:103AE80098F80030924A012B0CD002D3022B1BD03D
:103AF80023E03A8BB9F800309A421EDD012388F89A
:103B080000300FE0B9F800107B8B8B4202DD0223F6
:103B180013700FE0874B1B8B0133994202DD0023A2
:103B280013700AE0082006E07B8BB9F80020013307
:103B38009A42E3DC072004F06BFA2D68290577D553
:103B48007D4B7C4F1A68FB69C3EB020845F20723DB
:103B580098456DDD794BB6F906B0D3F800904FF46F
:103B68007A7099F80A30FA61012B98FBF0F8B4F8EA
:103B78005211ABF57A7B724E03D042D3022B20D080
:103B880041E0704B396A5A7B6F4B4FF0080E33F89F
:103B9800122091FBFEF392B2C91A8B183B6293FB79
:103BA800FEF3BA8440F6E4429BB25343B9F80820C6
:103BB800C2EB13335843B9F9063090FBF3F0306089
:103BC80021E0624BB9F808A01B78C6F800A05A0794
:103BD80019D55F4804F0C7F920B915F0100F18BFC0
:103BE8004FF0000B0BFB0BF3322293FBF2F3B9F906
:103BF80006205B445A434FF47A7392FBF3F3534421
:103C080000E0002333603368D7E90A0103FB08F8B2
:103C18004FF47A7398FBF3F810EB080041EBE87166
:103C28000023C7E90A014B4A0FF006FC4A4B18600B
:103C38004A4E3368DB0427D52F0622D5484B1B781C
:103C48009D071ED5474B187804281AD90022464BE1
:103C58000521D718951C4FF00A0E122AD154E9B243
:103C680087F801E004D0B0EB510F2A46EFD800E006
:103C780014215A18322002F8010CFF225A540F203E
:103C880000E00A2004F0C4F9384D2A68002A45D01B
:103C9800374B384F18683968984681423ED8364BBA
:103CA800DFF8E09018785168B0B901221A70B9F8B5
:103CB8000030CB5CD3B1314B1A700FF065F8B9F80E
:103CC80000309BB92B681B78053B012B0ED804F0FC
:103CD800D9F92B4B186009E000221A70B9F80030A6
:103CE800CB5C1BB1254B1A700FF04EF82B68B9F856
:103CF80000205B6823499B5CFE2B02D100230B80CC
:103D08000CE0FF2B02D104F071F907E0D8F80000AD
:103D18000A2505FB030301323B600A800B4D2B7813
:103D2800580733D5184B08225A616DE0440000202B
:103D3800141A002088100020CC300020B019002070
:103D4800BC1900201C2900202C290020E730002065
:103D58005E130020407E0500C0190020E8100020F6
:103D6800C8190020CE190020D42C0020C41A002025
:103D7800202D0020BC1A0020B81A0020B8300020DE
:103D8800182F0020C01A0020000C01403268D1070B
:103D98005CBF43F001032B70984B1B781F075EBF75
:103DA8002B7823F001032B70D60248BF2B78944A56
:103DB80044BF23F001032B70924B1B6813F0040FD0
:103DC80002D09149098851B99049098809B19807E1
:103DD80005D48F4B1B88003318BF012333B102234E
:103DE80013702B7823F001032B7004E02978C9079E
:103DF80058BF0223137004F045F9864B1B68C01A9C
:103E0800002801DB0EF0C0FF09F0D4FB824B1E78BE
:103E18009846002E00F0AB80804E3368002B00F0EF
:103E2800EC8630680CF052F9002800F0E6867B4BEF
:103E38007B4C18680CF047F9092801D03F2850D16D
:103E48004FF0000A5746D4F80090764DB9F1000FAC
:103E580005D0754829684A4612F0ECFE10B9AA4602
:103E680007B92F46714B10359D42EFD3C7B1D7F82C
:103E780000E0DAF800C023681EF803501CF80300BD
:103E8800A8420DD15A1C684938B92D2B05D8644D64
:103E98002A602025CD54885402E0CD542260EAE7F8
:103EA80023680BB1574511D061480DF081FB574588
:103EB80007D857F8100B0DF07BFB09200DF070FBAD
:103EC800F5E75C480DF074FB4FF00009236899454D
:103ED800A7D2554B13F809000DF062FB09F101094F
:103EE800F4E72368002B40F06D86042840F0AB8689
:103EF8004D4804F0F3FA00F080BED9F80000DFF86E
:103F080044A10CF0E3F840B3DAF800000CF0DBF859
:103F1800DBF80030024693F84810002935D12428F0
:103F280040F09280012283F84820DBF80030DFF867
:103F380010A193F84820062ADFD193F8490001F030
:103F48007FFE8146002800F0AA803B6898790DF032
:103F58007CFA3B68002283F84820374B93F83530C9
:103F6800002B40F01D864C36982E00F04686334BC9
:103F7800F21892F84A100129F5D1314FF3583A60F6
:103F8800304ABB4613609146B7E7012904D14D2852
:103F980014BF00220222C6E7022904D13C2814BF1C
:103FA80000220322BFE703290CD140284FF000016B
:103FB80002D983F84810B8E758711971D971987106
:103FC8000422B0E7042906D1997983F849004A40C8
:103FD8009A710522A7E70529A7D158791979884246
:103FE800987906D950409871481C18710B441A7278
:103FF8009BE790420CBF0622002294E7C8190020D4
:10400800B8300020C4190020DC300020B60F002092
:10401800DE300020BC300020E8300020C42C002016
:10402800101B00201C9A0108E01A0020CC9B0108F4
:10403800FBB5010800B601088810002018280020E8
:104048006C1A0020701A00202B78D84958073FF5C1
:104058006CAF232ADAF8003014D1012088F8000068
:10406800D34803910360D34802920363D2480DF00A
:104078009FFAD2480DF09CFA0399029A0B7843F004
:1040880002030B70CE4B1B681B78934201BFCD4ACD
:10409800CD4B1A60CD4A04BFCD4BDA6045E7DAF85C
:1040A800002092F849304C2B00F069845DD8332BFE
:1040B80000F0A08421D8292B00F02D8409D8252BC5
:1040C80000F00484272B00F00884232B40F0B785E8
:1040D8002FE22D2B00F0308407D82B2B40F0AF8532
:1040E8000DF096F9607100F03EBD2F2B00F0EE84C4
:1040F800312B00F0008500F0A2BD3E2B00F0F280CD
:104108001DD8372B00F0AA8404D8352B00F04A823A
:1041180000F095BD392B00F0ED833C2B40F08F85E6
:10412800DFF8B092D9F800A00DF072F98AF8000013
:10413800D9F8003018780CF039FA00F014BD432B88
:1041480000F0698406D8412B40F079854FF00009CA
:1041580000F055BC442B00F002854A2B40F06F85D7
:104168000DF060F9A08100F0FEBCD02B00F01083A8
:1041780055D8CA2B00F0C08009D8C82B00F085801C
:1041880000F23E834E2B00F0078400F058BDCD2B83
:1041980000F0098304D8CC2B00F02C8200F04FBD2E
:1041A800CE2B00F00983CF2B40F049850DF03AF96A
:1041B8006FF4AF6283189BB2C62B98BFA4F898011E
:1041C8000DF030F9A4F844010DF02CF9A4F84601DB
:1041D8000DF028F9A4F848010DF024F9A4F8DA0143
:1041E8000DF016F984F8EF010DF012F90DF010F941
:1041F80084F8F0010DF00CF984F887010DF008F946
:1042080084F894010DF004F9724BD3F800900DF086
:1042180009F900EB80004000A9F856006AE3D62BA4
:1042280000F03B820AD8D22B19D0C0F01083D32BD0
:1042380025D0D42B00F03C8200F001BDEF2B41D0FB
:1042480005D8D82B40F0FB844FF0000904E1F22B8D
:1042580000F07682FA2B00F0B88200F0F0BC2B78E0
:10426800590700F180840DF0D3F8022884F8B007CC
:1042780040F29482584B002283F8B0278EE20DF06A
:10428800D1F8564B188000F06EBC92F805904FEAB2
:104298005909B9F1120F03D90AF020FF00F063BCE5
:1042A8004FF0000ACA4507D20DF0BCF84C4B23F872
:1042B8001A000AF1010AF5E73E4B012283F834207F
:1042C80000F051BCDFF80C91D9F800A00DF0AAF865
:1042D800AAF85A00D9F800900DF0A4F8A9F85800E7
:1042E80000F041BC0DF094F884F8E2010DF090F86C
:1042F80084F8E10100F037BC364B1A689A46127808
:10430800022A40F08E80DAF8003009F1080B029397
:104318000DF07EF80EF02CFE32490EF035FF029BB0
:1043280043F82B00DAF800B00DF072F809F10A032F
:104338000BEB830B0EF01CFE2B490EF025FFDAF871
:104348000030CBF8040002930DF062F80EF010FE76
:1043580026490EF019FF09F10E0B029B09F101091C
:10436800B9F1030F43F82B00CDD1B9F1070FDAF8F3
:1043780000B03DD10DF04CF80EF0FAFD19490EF0E1
:1043880003FFCBF84400DAF800B00DF041F80EF066
:10439800EFFD14490EF0F8FECBF84800DAF800B04B
:1043A8000DF036F88BF84C0035E000BFE730002000
:1043B800C42C00208810002030B6010800B601087F
:1043C800BC280020EFBEADDEF04F00200400FA0547
:1043D80000ED00E024110020D4110020F80F002087
:1043E800382D0020000020410000C84200007A4417
:1043F8000DF00EF8CB448BF80100DAF800B00DF0A0
:1044080007F8CB448BF80B00DAF800B00DF000F891
:10441800CB448BF8150009F10109B9F10A0FA4D1B1
:10442800A1E3DAF800B00CF0F3FFCB448BF80100FD
:10443800DAF800B00CF0ECFFCB448BF80B00DAF89C
:1044480000B00CF0E5FFCB4409F10109B9F10A0FFE
:104458008BF81500E5D186E3DFF890A309F1080B86
:10446800DAF8003002930CF0DDFF0EF081FDD94937
:104478000EF08AFE029B43F82B00DAF800B00CF02D
:10448800D1FF09F10A030BEB830B0EF071FDD14943
:104498000EF07AFEDAF80030CBF8040002930CF044
:1044A800C1FF0EF065FDCB490EF06EFE09F10E0B53
:1044B800029B09F10109B9F1030F43F82B00CBD195
:1044C800B9F1070FDAF800B01AD10CF0ABFF0EF013
:1044D8004FFDC0490EF058FECBF84400DAF800B0A2
:1044E8000CF0A0FF0EF044FDBA490EF04DFECBF8DB
:1044F8004800DAF800B00CF095FF8BF84C0012E099
:104508000CF090FFCB448BF80100DAF800B00CF007
:1045180089FFCB448BF80B00DAF800B00CF082FF6F
:10452800CB448BF8150009F10109B9F10A0FC7D17D
:1045380019E30CF06DFF132883463FF6ADAEDFF8A4
:10454800ACA2DAF800900CF063FF0023A2490C2219
:1045580002FB0312117A814220D1137809EB8B09EF
:1045680089F879300CF054FF89F87A000CF050FF84
:1045780089F87B000CF04CFF984A994B89F87C002D
:104588001A60DAF80000974B00211860793003F0C0
:10459800D9FC954B80F001001870E4E201331C2B24
:1045A800D4D179E60CF034FF0B2882463FF674AE7E
:1045B8008E4BD3F800900CF02BFF03283FF66CAE1F
:1045C800062303FB0A9989F8CE000CF021FF89F82D
:1045D800C9000CF01DFF89F8CA000CF019FF89F812
:1045E800CB000CF015FF89F8CC000CF011FF89F80E
:1045F800CD00B8E25379092B7FF64EAE019BD3F874
:1046080000900CF005FF019B89F80000D3F800909A
:104618000CF0FEFE89F801000CF0FAFE019B6428FC
:104628001B68A8BF642018710CF0F2FE019B642877
:104638001B68A8BF642058710CF0EAFE019BFF2894
:104648001B68A8BFFF2098710CF0E2FE019B64284C
:10465800D3F8009028BF642089F807000CF0D8FE32
:10466800019B89F80200D3F800900CF0D1FE019B61
:1046780089F80300D3F800900CF0D4FE3B68A9F841
:104688000A005B790A2B40F26E82594BD3F80090EE
:104698000CF0BEFE89F8080065E20CF0C3FE554B2D
:1046A80023F8190009F10109B9F1080FF5D15AE207
:1046B80053790F2B7FF4F0AD0CF0AAFE0728814642
:1046C8003FF6EAADDFF824A1DAF800B00CF0AAFE54
:1046D8000E2303FB09F9CB44ABF81901DAF800B053
:1046E8000CF0A0FECB44ABF81B01DAF800B00CF0DC
:1046F80099FECB44ABF81D01DAF800B00CF088FE47
:10470800CB448BF81F01DAF800B00CF081FECB44E3
:104718008BF82001DAF800B00CF07AFECB448BF865
:104728002101DAF800B00CF073FECB448BF82201BB
:10473800DAF800A00CF080FED144C9F8230112E297
:104748000CF066FE0F2881463FF6A6AD0CF060FE21
:10475800C9EBC909A14489F8D4000CF059FE89F8BD
:10476800D5000CF055FE89F8D6000CF051FE89F8FA
:10477800D7000CF04DFE89F8D8000CF049FE89F8F6
:10478800D9000CF045FE89F8DA000BF061FEEAE189
:104798002B785B0700F1E7810DF05AF905F02CFE44
:1047A80005F0D0FEDFE12B78580700F1DC81124BD1
:1047B8004FF4C8721A80D6E12B78590700F1D381DB
:1047C8000E4A137843F004033FE02B785A07E5D5E7
:1047D80035E200BF00007A44E09301081813002076
:1047E800F00F0020F40F00201800002024110020F2
:1047F8004C110020AA2C0020B60F0020C819002058
:104808000CF006FEDA4B1A7810B142F0020201E011
:1048180022F002021A700CF0FBFDD64BDFF87893F9
:1048280018700CF009FEC9F800000CF005FEC9F874
:1048380004000CF0F7FDD04B18800CF0F3FDCF4BC3
:10484800CF4A1880137843F0020313708BE10CF001
:10485800DFFD02900CF0F0FD83460CF0EDFD824682
:104868000CF0EAFD81460CF0DDFD0CF0DBFD0CF0F0
:10487800CFFD029BA3B9C34B1020C3F800B0C3F807
:1048880004A005F066FDBA4A137843F001031370DB
:10489800B9F1000F00F06781BB4BC3F8009062E1EB
:1048A800102B40F06081B94BC3F800B0C3F804A0E6
:1048B800B9F1000F02D0B44BC3F80090B348B44B21
:1048C8000222011D1A7006F0CBFB4CE1A0600CF02F
:1048D800B3FDA3681843A06045E10CF0A3FDA4F85C
:1048E8005C010CF09FFDA4F85E010CF09BFDA4F8A0
:1048F800600138E10CF08CFD84F87C010CF088FD37
:1049080084F880010CF084FD84F87F010CF080FDB0
:1049180084F8810127E10CF085FDA4F882010CF0F0
:1049280081FDA4F884010CF073FD84F886010CF075
:1049380079FDA4F8880116E10CF06AFD84F892016B
:104948000CF070FDA4F89C010CF06CFDA4F8980123
:104958000CF068FDA4F89A010CF05AFDDAF8003062
:1049680084F893015B79082B40F2FD800CF05AFD26
:10497800A4F89E010CF056FDA4F8A001F3E00CF099
:1049880047FD84F8D8010CF043FD84F8D9010CF0F8
:1049980049FDA4F8DA01E6E092F805900323B9FB93
:1049A800F3F9B9F1120F3FF677ACDFF8F0A14FF049
:1049B800000BCB4580F0D7800CF02AFD8AF8A201C5
:1049C8000CF030FD40F2ED23984205DD40F6CA03B5
:1049D8009842A8BF184601E040F2EE20A0F2EE206F
:1049E800192390FBF3F00BF1010B8AF8A3010AF1EC
:1049F800020ADEE70CF00CFD84F89401B3E00CF039
:104A080007FD04EB090309F10109B9F1080F83F85F
:104A18008A01F4D1A7E00CF0FBFCC4F8089060719F
:104A28000CF00AFDA3681843A0600CF0F1FC84F8B0
:104A380092010CF0F7FCA4F85C010CF0F3FCA4F86C
:104A48005E010CF0EFFCA4F860010CF0EBFCA4F89C
:104A580082010CF0E7FCA4F8840184E053794FF05C
:104A6800070AB3FBFAF2C2EBC2029A1A12F0FF0F5E
:104A78007FF412ACB3FBFAFA0AF1FF3A5FFA8AFA4A
:104A8800BAF1FF0F6FD00CF0C3FC5FFA80FB4FFA4E
:104A98008BF003F0F1F8814600283FF4FDAB80F875
:104AA80000B00CF0BFFCA9F802000CF0B1FC89F8CA
:104AB80004000CF0ADFC89F805000CF0A9FC89F89D
:104AC80007000CF0A5FC89F80600D5E7DFF8CC90C4
:104AD80009F1400A0CF0A6FCA9F8A8020CF098FC11
:104AE80089F8AA020CF094FC09F1040989F8A702D4
:104AF800D145EFD137E00CF08BFC1F2881463FF6FB
:104B0800CBAB3B685B79082B7FF4C6AB0CF08AFC17
:104B180009F18A0904EB890A00F03F00AAF80200AB
:104B28000CF080FCBAF80230800100F4FE50184303
:104B3800AAF802000CF06CFC000104F829000CF043
:104B480067FC14F8293000F00F00184304F8290016
:104B58000CF05EFC8AF801000BF0BCFD03E00D4B85
:104B6800012283F8352000200CF09EFCFFF7EDB9F8
:104B7800C8190020CE190020CC190020CA1900201D
:104B88005211002054110020641100205C110020F3
:104B9800FC0F002088100020D0190020D41100201C
:104BA8005B4B985903F03EFB18B9322003F091FA99
:104BB800F6E70BF00DFC05F0F5FB564A564BDA60AC
:104BC800FFF7D1B90C2840D00A2847D1534D544893
:104BD8000CF0EEFC2846232112F015F808B1401B12
:104BE80020602368002B5CD14C48002130222360D0
:104BF80011F0D3FF98F8003053BB4A4B1B689B0653
:104C080014D5494B49491B688A6B9A1A002A0DDB4F
:104C1800474A1278042A09D903F5123303F5F873C1
:104C2800444A8B63D36883F01003D360424B9B687C
:104C3800002B69D0414805B0BDE8F04F18470AF08D
:104C48004DFAFFF782B90C2804D13D480CF0B0FCAE
:104C58003C480DE07F2812D1FFF7E3B80D28B5D006
:104C68007F2809D12D4A013B002137482360D154C0
:104C78000CF09EFCFFF7D5B82F2B3FF6D2A8A0F179
:104C88002002D2B25E2A3FF6CCA813B920283FF4FE
:104C9800C8A85A1C2260214AD0540CF081FCFFF7A6
:104CA800C0B85A1EA95C202901D113469AE71B4AAD
:104CB80000212360D154254B254DD3F800A0D5F809
:104CC80000B0DFF85890584611F0ABFF0746594638
:104CD8003A46484611F0AEFF1E4A28B919F807307F
:104CE80053445B785B0703D010359542E7D306E061
:104CF800954204D2781CEB684844984702E016486D
:104D08000CF056FC00236FE705B0BDE8F08F00BF3C
:104D1800182800200400FA0500ED00E0E01A002041
:104D2800E6C40108C4190020CC30002088100020F7
:104D3800CE190020000C014094270020C410002048
:104D480005B6010800B601082CB601085800002075
:104D58001C9A0108CC9B010810B601086B4B6C4AE1
:104D68002DE9F04F5E8914684FEA062AB4EB0A0A67
:104D78009C884FF000054FEA04481C894FF0000B4F
:104D8800A4FB0A6765EB0B0B04FB0B77F40944EAF9
:104D9800476418EB04065C884FF000094FEAE715F2
:104DA8004FEAC438DC8849EB050787B0CDE90467CA
:104DB800A4FB0A6704FB0B77340A44EA076418EB80
:104DC80004064FEA27259C894FF0000949EB05079F
:104DD800CDE90067AAFB046704FB0B77F40D44EAEE
:104DE800472414F5FA664FEAE75545F10007B6F58A
:104DF800FA6F77F10003CDE90267964666DADDE9D6
:104E08000489A4FB046704FB05F34FF0050C07EBCA
:104E18004307A6FB0C230CFB07335F104FEA32064F
:104E2800B8EB06084FEA920646EA837669EB07096B
:104E38009F10DDE90023921B63EB0703CDE90023F4
:104E4800DDE90267334A4FF0FF33964277EB0303FD
:104E5800CDE9048927DA40F6AC520023A4185D4155
:104E680004FB05F3A4FB04456FF0060205EB4305BC
:104E7800664202FB0566A4FB0223334418EB0206D4
:104E880049EB0307CDE904670B26A4FB062306FBC1
:104E98000533DDE900455B104FEA3202A41A65EBE1
:104EA8000305CDE90045DDE902450AFB0BF3AAFB42
:104EB8000AAB0BEB430B4FEADA7242EA4B02A41A35
:104EC8004FEAEB7365EB0305CDE90245DEF80440D4
:104ED800009B019DA4FB032304FB05334FEA5258B2
:104EE80048EAC3284FEA6359DDE90423B8EB020214
:104EF80069EB03039946D30B43EA494300B10360C6
:104F080009B1029B0B6007B0BDE8F08F4E0200208C
:104F1800C810002024FAFFFF2DE9F04FDFF858925F
:104F280085B00746D9F808000E460EF025F88E4CD5
:104F3800804620880EF01CF84FF05C51054640462C
:104F48000EF06EF84FF06451824628460EF068F86D
:104F5800014650460DF05AFF4FF0625182464046D6
:104F68000EF05EF84FF06A51804628460EF058F869
:104F7800014640460DF04AFF0546B4F902000DF01F
:104F8800FBFF014628460EF04BF8514605465046B1
:104F98000EF046F88046B4F904000DF0EDFF014626
:104FA80040460EF03DF8014628460DF031FF804698
:104FB8000EF0FCF96D490546A06140460EF0E4F894
:104FC800D9F80C308046284601930DF0D5FF4FF0F4
:104FD8007C510EF025F866490DF018FF0546E38967
:104FE800B4F90A0002930DF0C7FF29460EF018F82D
:104FF80029460EF015F84FF058510EF011F8814679
:10500800B4F90800B4F810B0B4F80CA00DF0B4FF6F
:1050180029460EF005F8014648460DF0F9FE4FF016
:1050280058510DF0FDFF4FF060510DF0F9FF4FF0B2
:105038007E510DF0EDFE8146E0880DF099FF0146A6
:1050480048460DF0EDFF002181460EF07DF900285D
:105058007BD1294628460DF0E3FF03900FFA8BF029
:105068000DF08AFF039B014618460DF0D9FF4FF05B
:1050780060510DF0D5FF8346BDF908000DF07CFFA7
:10508800014628460DF0CCFF01460DF0C1FE014651
:1050980058460DF0BDFE4FF07A510DF0C1FF834622
:1050A80001980DF069FF01464FF093400DF0AEFEF8
:1050B80005460FFA8AF00DF05FFF4FF08F410DF0B3
:1050C800AFFF014658460DF0A3FE4FF066510DF0B4
:1050D800A7FF014628460DF099FE26490DF0A0FFCE
:1050E80049460EF051F80546B4F916000DF044FF94
:1050F80029460DF095FF29460DF092FF4FF04051DB
:105108000DF08EFF8146B4F914000DF035FF01460D
:1051180028460DF085FF4FF060510DF081FF0146E4
:1051280048460DF075FE8146B4F912000DF024FFD3
:10513800014648460DF06CFE4FF076510DF070FFB9
:10514800014628460DF064FE00E0002017B10EF07D
:105158002DF938602EB140460EF028F964235843E3
:10516800306005B0BDE8F08F880200200000A0453F
:1051780000007A470050C345C810002070477047A8
:105188002DE9F041324C334D62892B8AB4F9048001
:105198009A1A2389B4F902E05A43B4F91230D613A3
:1051A800B4F91420DB02324493FBF2F232440A26AB
:1051B800E2615643A2F57A6202FB02F3B4F90EC02B
:1051C80002FB0EFE02FB08F2B4F90C801B130CFB69
:1051D80003FC03FB08F31B1403EB62320232E3887F
:1051E800921002F5004253434CF25032B4F9207049
:1051F8004FEAEE2EB4F900400EEBEC2C0CEB8404D5
:10520800BC406D690234A5EBA4043A4162434FEAFD
:10521800D3384EBFB2FBF8F35400B4FBF8F340F6B2
:10522800DE3448BF5B001A12524362430A4C083608
:105238005C43241404EB224202F6CF62361103EBDE
:10524800221300B1036001B10E60BDE8F08100BF18
:1052580060020020C810002043E3FFFF024B4FF418
:1052680080521A80704700BF1A0000207047054A14
:10527800137E23B101230370002313767047037054
:10528800704700BFC8100020054A08B513880133CD
:105298009BB21380034B187806F0D6FA002008BD9D
:1052A800E61000206C1D00200F4B13B55A7E1C46DB
:1052B800C2B90E4B1B68ABB11A681AB10C498869A0
:1052C80002438A619A889868ADF8042002228DF812
:1052D800072004220DEB02018DF8062007F0ACFD33
:1052E8000123637602B010BDC810002044020020DC
:1052F8000010024008B5FFF7D7FF074B1B7813B122
:10530800012B03D008BD4FF4006201E04FF4805236
:10531800024B1A8008BD00BF4C0200201A00002072
:10532800F8B50F461646074C4FF48055656140F0B6
:1053380080000CF0FBFE384631460CF01DFF25615D
:10534800F8BD00BF000C014013B501220DF10701A3
:1053580004463820FFF7E4FF052002F0AFFE9DF871
:10536800073003B10123237002B010BD13B5044602
:10537800694643200622FFF7D3FF9DF800209DF8D9
:105388000130012043EA022323809DF802209DF882
:10539800033043EA022363809DF804209DF805301A
:1053A80043EA0223A38002B010BD13B50446694640
:1053B8003B200622FFF7B4FF9DF800209DF801303E
:1053C800012043EA022323809DF802209DF8033040
:1053D80043EA022363809DF804209DF8053043EAE0
:1053E8000223A38002B010BD70B50E46054C4FF4E1
:1053F800805565610CF09AFE30460CF097FE2561E9
:1054080070BD00BF000C014008B580216B20FFF77C
:10541800EBFF642002F05DFE00216B20FFF7E4FF44
:10542800642002F056FE6B200121FFF7DDFF1B20F0
:105438001821FFF7D9FF1C201021FFF7D5FF054BD6
:105448001A201978FFF7D0FFBDE80840192000217D
:10545800CAE700BF0100002010B54000204CC0B2D0
:1054680020702048204C0170204800210170012044
:1054780020701F4C23601F4C23601F4B1A701F4A5B
:105488001F4B107019701F49086811461A4630B32F
:1054980083889C0515D40388DB050DD447F2305367
:1054A8000488A40502D5013BFAD112E08BB1038828
:1054B8009BB243F48073038083889BB243F44073A8
:1054C800838047F23053087810B1013BFBD100E0EC
:1054D80013B9BDE81040D7E6107880F0010010BD80
:1054E800721D0020701D00206E1D0020781D0020F8
:1054F800741D00207C1D0020711D0020801D0020CF
:10550800811D0020681D002007B5002101AB032282
:105518007720FFF7A1FF9DF805309DF804001B02D6
:1055280043EA00439DF80600184303B05DF804FB06
:1055380008B5FFF7E9FF014B586008BDC810002007
:1055480008B5FFF7E1FF014B186008BDC81000203F
:1055580007B5F7216B4606227620FFF77DFF9DF8F9
:1055680000309DF801101B0343EA01139DF8021057
:10557800094A43EA1113D3609DF803309DF80410DB
:105588001B0343EA01139DF8051043EA11139360C6
:1055980003B05DF804FB00BFC810002007B5F62172
:1055A80001AB03227720FFF757FF9DF805309DF8E0
:1055B80004201B0243EA02439DF806201343054AD0
:1055C800B2F92020C2F10802D340034A536103B064
:1055D8005DF804FB60020020C810002007B5F62122
:1055E80001AB02227720FFF737FF9DF804209DF8D2
:1055F800053043EA0223024A138203B05DF804FB34
:10560800C810002013B506220446432168206B46C3
:10561800FFF722FFA8B19DF800209DF80130012076
:1056280043EA022323809DF802209DF8033043EAD1
:10563800022363809DF804209DF8053043EA022385
:10564800A38002B010BD13B5062204463B21682092
:105658006B46FFF701FFA8B19DF800209DF80130C7
:10566800012043EA022323809DF802209DF803309D
:1056780043EA022363809DF804209DF8053043EA3D
:105688000223A38002B010BD13B5062204460121EF
:105698001C206B46FFF7E0FE08B39DF801309DF82B
:1056A8000020042143EA022242F38D0292FBF1F228
:1056B8009DF8023022809DF8032042EA032242F33B
:1056C8008D0292FBF1F29DF8043062809DF805206E
:1056D80042EA032343F38D0393FBF1F3A38002B063
:1056E80010BD13B506220446A82168206B46FFF7B3
:1056F800B3FEA0B19DF800209DF8013043EA0223D3
:1057080023809DF802209DF8033043EA022363803A
:105718009DF804209DF8053043EA0223A38002B0D7
:1057280010BD13B506220446022118206B46FFF768
:1057380093FEB8B19DF800309DF801209B0803EB5B
:10574800022323809DF802309DF803209B0803EB79
:10575800022363809DF804309DF805209B0803EB25
:105768000223A38002B010BD314B2DE9F3411B7811
:105778000546002B3BD0002426462746A046013488
:105788005320322108226B46E4B2FFF765FE08B9C0
:10579800002049E09DF801209DF80030202C03EB03
:1057A80002231BB29DF8032098449DF8023003EBB6
:1057B80002231BB21F449DF805209DF8043003EB1B
:1057C80002231BB21E449DF8073003F07F0301D06B
:1057D800002BD4D198FBF4F897FBF4F796FBF4F67A
:1057E800144BA5F800806F80AE809C761CE0532097
:1057F800322106226B46FFF72FFE0028C8D09DF8FD
:1058080001209DF8003003EB02232B809DF8032034
:105818009DF8023003EB02236B809DF805209DF86C
:10582800043003EB0223AB8002B0BDE8F08100BF77
:105838004B020020C810002013B502AB03F8012D5D
:105848004000214AC0B21070204A0020117020493F
:1058580001220A701F4908701F490B601F490B601D
:105868001F4B20491A700A701F4B204A1870106885
:105878001A4630B383889C0515D40388DB050DD4FC
:1058880047F230530488A40502D5013BFAD112E04F
:105898008BB103889BB243F48073038083889BB2E7
:1058A80043F44073838047F23053087810B1013BCA
:1058B800FBD100E013B9FFF7E7FC02E0107880F0B5
:1058C800010002B010BD00BF721D0020701D002035
:1058D800781D00206E1D00207C1D0020741D0020F6
:1058E800711D0020801D0020811D0020681D0020E2
:1058F8007720482101229FE77720582101229BE742
:105908007620F421312297E7044B772093F8202062
:10591800F4219201343202F0FC028DE7600200208B
:105928007720F4212E2287E708B5FFF7BDFC6B210D
:1059380080226820FFF780FF642002F0CAFB6B21F9
:1059480003226820FFF778FF0F2002F0C2FB0F4BFD
:1059580019211A786820FFF76FFF0F2002F0B9FBB2
:105968000B4B1A211A786820FFF766FF1B211822B3
:105978006820FFF761FF1C2110226820FFF75CFFF9
:10598800BDE8084068203721002255E74A02002078
:105998000000002008B52A2100221C20FFF74CFF38
:1059A8000E2102221C20FFF747FF0F2103221C2093
:1059B800FFF742FF2B2112221C20FFF73DFF2C216D
:1059C80002221C20FFF738FF2D2101221C20FFF79F
:1059D80033FF2E2100221C20FFF72EFF05221C205A
:1059E8002A21FFF729FF024B4FF480721A8008BD65
:1059F8001A00002008B5642002F06BFB6820232100
:105A0800F022FFF719FF10B9022002F06CFB052005
:105A180002F05FFB044B68201A78202142F00F0245
:105A2800BDE8084008E700BF4802002008B50F217C
:105A380008221820FFF700FF0E2218201021FFF778
:105A4800FBFE024B4FF480521A8008BD1A0000205A
:105A580008B5134B53201B782D2108227BB1FFF783
:105A6800EBFE31210A225320FFF7E6FE2C210C22FF
:105A78005320FFF7E1FE53203821902209E0FFF779
:105A8800DBFE31210A225320FFF7D6FE53202C21BA
:105A98000A22FFF7D1FE40F20912024B1A8008BD14
:105AA8004B0200201A00002005F0C6BF06F0EAB835
:105AB80005F0C2BF06F0E6B873B51D4CE37E53BBD4
:105AC8001C4A1D4D93694FF4805643F008039361B7
:105AD80010238DF806302846032301A98DF80730D6
:105AE800ADF8046007F0A8F9144A2E61138823F072
:105AF80040031B041B0C1380138823F038031B047A
:105B08001B0C43F00803138013889BB243F0400337
:105B180013800123E376752001A90122FFF700FC19
:105B28009DF80400A0F170035842584102B070BDBE
:105B3800C810002000100240000C0140003800404E
:105B4800F8B50F461646074C4FF48055656140F08E
:105B580080000CF0EBFA384631460CF00DFB25615D
:105B6800F8BD00BF000C014013B501220DF107017B
:105B780004463A20FFF7E4FF052002F09FFA9DF85B
:105B8800073003B10123237002B010BD184A13B5C2
:105B98001388044623F040031B041B0C138013884E
:105BA800432023F038031B041B0C13801388694619
:105BB8009BB243F0400313800622FFF7C1FF9DF814
:105BC80000209DF80130012043EA022323809DF83C
:105BD80002209DF8033043EA022363809DF80420E5
:105BE8009DF8053043EA0223A38002B010BD00BF30
:105BF8000038004070B50E46054C4FF4805565617D
:105C08000CF094FA30460CF091FA256170BD00BF93
:105C1800000C014007B5232002F05BFA68207521CB
:105C280001220DF10703FFF717FC28B19DF80700C3
:105C3800A0F168035842584103B05DF804FB00BF67
:105C48004D282DE9F047044600F0548600F2B9804B
:105C5800302800F0B48651D8222800F0908423D848
:105C6800032800F0058214D8012800F0F5810228E5
:105C780040F0F48604200BF017FC43200BF0E5FB02
:105C88004C200BF0E2FB46200BF0DFFB4C2000F031
:105C980056BE042800F0F581052840F0DF861A205A
:105CA8000BF002FC0024FCE1282800F0E28515D85E
:105CB800242800F0C985262840F0D086DA4C062032
:105CC8000BF0F2FBB4F85C010BF0F1FBB4F85E01E9
:105CD8000BF0EDFBB4F8600100F0B3BD2C2800F028
:105CE800DB852E2800F055862A2840F0B78601204B
:105CF8000BF0DAFBCC4B587900F021BE3D2800F0C0
:105D0800F8821ED8362800F02B860BD8322800F0EF
:105D18001086342840F0A28648200BF0C5FB0025E9
:105D280000F04FBC3A2800F0B9823B2800F02084EC
:105D3800382840F0938604200BF0B6FBBA4C00F0EC
:105D480089BD452800F0768627D8402800F0FA85D6
:105D5800422840F08386B44C10200BF0A5FB6079F4
:105D68000BF073FBA0680BF0ABFB94F892010BF0FF
:105D78006CFBB4F85C010BF09AFBB4F85E010BF015
:105D880096FBB4F860010BF092FBB4F882010BF0BB
:105D98008EFBB4F8840100F054BD492800F0B482A9
:105DA8004B2800F09885462840F058860D200BF0C7
:105DB8007BFB00200BF049FB00200BF081FB00F07F
:105DC80044BE702800F0F08200F2E180692800F0FB
:105DD800458200F2B280662800F0A08100F2A2801D
:105DE800642800F07781652840F038868F4C0B20B6
:105DF8000BF05AFB20880BF05AFB608880B20BF03E
:105E080056FB8B4B1B68C3F3C000C3F380028000B2
:105E180040EA4200C3F340021043C3F3401240EA91
:105E2800C20003F0100318430BF041FB814B1A88A2
:105E3800636802F0080103F4475949EA010903F4C9
:105E4800804149EA010903F4004149EA010903F4E0
:105E5800803149EA010903F4003149EA010903F4F0
:105E6800802149EA010903F4002149EA010903F400
:105E7800801149EA010903F0007349EA0303DFF8D6
:105E8800D49112F0010F99F8009018BF4FF0020852
:105E9800C9F3800908BF4FF0000843EA090312F06C
:105EA800020F43EA080314BF4FF0040C4FF0000C34
:105EB80012F0040F43EA0C0C14BF4FF0100E4FF011
:105EC800000E12F0400F14BF202700274CEA0E0ED8
:105ED80012F0100F14BF4FF4007600264EEA0707A1
:105EE80012F0200F14BF4FF4806500253E4312F4D2
:105EF800807F14BF4FF400600020354312F4007F08
:105F080014BF4FF400110021284312F4806F41EAB6
:105F1800000114BF4FF08063002300201943247A46
:105F28000346E7E0672800F02181682840F096855D
:105F380010200BF0B9FA002488E16C2800F0A18148
:105F480017D86A2800F003846B2840F0878505205D
:105F58000BF0AAFA384B18880BF0A9FA374B1888B7
:105F68000BF0A5FA314B93F86E0000F0010000F039
:105F7800E6BC6E282D4D00F0978100F2CB810620FB
:105F88000BF092FAE86D0BF09BFA2D4B84E1782820
:105F980000F0F98018D8742800F034830AD87228E1
:105FA80000F09583732840F0598508200BF07CFA9F
:105FB8000124C5E3762800F0EA8300F25C832F20F1
:105FC8000BF072FA1F4CCBE2A42800F0068414D818
:105FD8007B2800F06B82A02840F040850C200BF055
:105FE80063FA194B18680BF06BFA184B18680BF02A
:105FF80067FA174B186800F02CBDF12800F0FF80F5
:10600800FE2800F01184F02840F02885074C042071
:106018000BF04AFA236CB3F85A000BF048FA236CD9
:10602800B3F8580000F00DBCD4110020E410002093
:10603800C41900208C1A0020421A0020441A00209B
:10604800BC110020AF930108E8F7FF1FECF7FF1F12
:10605800F0F7FF1FE730002003200BF025FA00209F
:106068000BF0F3F920460BF0F0F90D2000F067BCB7
:106078000BF01AFA01200BF0E8F90A200BF0E5F909
:10608800A9E306200BF010FA45200BF0DEF95520A5
:106098000BF0DBF946200BF0D8F931200BF0D5F9DD
:1060A800CEE3B04B185D01340BF0CFF90B2CF8D1CF
:1060B8000024AD4B185D01340BF0C7F9082CF8D15A
:1060C8000024AA4B185D01340BF0BFF9072CF8D156
:1060D80000F0C1BC07200BF0E7F9E7200BF0B5F999
:1060E800A34B58790BF0B1F900200BF0AEF904205E
:1060F80000F0AFBCA3420AD29E4A9D5C012202FA7C
:1061080005F50D421CBF9A4010430133F2E70BF02E
:10611800D7F9974B93F8B00700F011BC12200BF099
:10612800C3F9954B00241B88B3F5806F8CBF0825F5
:106138000125924B33F91400013490FBF5F080B23D
:106148000BF0B5F9032CF4D18D4CA08C0BF0AFF902
:10615800E08C0BF0ACF9208D0BF0A9F9608D0BF0F9
:10616800A6F9A08D0BF0A3F9E08D6AE310200BF0DF
:106178009BF90024834B185D01340BF066F9102C51
:10618800F8D100F068BC70200BF08EF900260E24C0
:1061980074437B4D01362B6C2344B3F819010BF083
:1061A80086F92B6C2344B3F81B010BF080F92B6C98
:1061B8002344B3F81D010BF07AF92B6C234493F8B0
:1061C8001F010BF042F92B6C234493F820010BF0CC
:1061D8003CF92B6C234493F821010BF036F92B6C16
:1061E800234493F822010BF030F92B6C1C44D4F8AB
:1061F80023010BF065F9082EC9D100F02CBC7020E2
:106208000BF052F95A4C04F1700594F8D4000BF0D5
:106218001CF994F8D5000BF018F994F8D6000BF097
:1062280014F994F8D7000BF010F994F8D8000BF093
:106238000CF994F8D9000BF008F9073494F8D30056
:106248000BF003F9AC42E0D100F005BC4E4B185DF1
:1062580001340BF0FAF8102CF8D1FCE34B4D002474
:106268002878400000F0FE000BF01EF92B789C42C5
:1062780080F0F183464B33F814000BF018F9013421
:10628800F4E7444C06200BF00FF920880BF00FF9C7
:1062980060880BF00CF9404B1888D2E204200BF010
:1062A80003F9374B186ED4E307200BF0FDF83B4B8E
:1062B8001888FF28A8BFFF20C0B20BF0C6F8384BDB
:1062C800186880F3100080B20BF0F1F8B5F864009C
:1062D8000BF0EDF8264B93F88721324B186822B162
:1062E8000A23584380F3100001E000F30F0080B246
:1062F800A7E21F4C02200BF0D7F894F8E2010BF04C
:10630800A4F894F8E1011AE302200BF0CDF8184B39
:10631800988996E20B200BF0C7F8AB6E0026187828
:106328000BF093F8AB6E58780BF08FF8AB6E144CFB
:106338003344187901360BF088F8032EF6D1A36E92
:10634800D8790BF082F8A36E98780BF07EF8A36EDC
:10635800D8780BF07AF8A36E58890BF0A8F8A36EDA
:10636800187AECE268B6010874B601087DB601082F
:10637800D4110020ED1000201A000020B6110020D2
:10638800E41000201411002028110020B428002057
:10639800382D0020F42C0020C4110020B41900204E
:1063A800C0190020BC190020C04C1E200BF07CF83E
:1063B800236C00251B78022B65D1236C05F108029C
:1063C80053F82200BA490CF02BFE10F0F3FD80F3CD
:1063D8000800C0B20BF039F8236CB64903EB85030B
:1063E800D86A0CF01DFE10F0E5FD80F30800C0B27D
:1063F8000BF02BF8236C05F10E0253F82200AE497E
:106408000CF00EFE10F0D6FD80F30800C0B2013586
:106418000BF01BF8032DD0D1072D236C21D1586C1C
:10642800A3490CF0FDFD10F0C5FD80F30800C0B2D3
:106438000BF00BF8236C9E49986C0CF0F1FD10F0F2
:10644800B9FD80F30800C0B20AF0FFFF236C93F88F
:106458004C000CF08DFD10F0ADFD80F30800C0B2CB
:106468000BE02B4458780AF0F0FF236C2B44D87AC1
:106478000AF0EBFF236C2B44587D01350AF0E5FF49
:106488000A2DC9D1E7E2236C2B4458780AF0DDFFC6
:10649800236C2B44D87A0AF0D8FF236C2B44587D00
:1064A80001350AF0D2FF0A2DEDD1D4E23C200AF0E2
:1064B800FBFF00247D4D04F108022B6C7E4953F844
:1064C80022000CF0ADFD10F075FD80B20AF0EFFF70
:1064D8002B6C794903EB8403D86A0CF0A1FD10F00A
:1064E80069FD80B20AF0E3FF2B6C04F10E0253F849
:1064F800220071490CF094FD10F05CFD013480B26B
:106508000AF0D5FF032CD5D1072C2B6C16D1586C6B
:1065180069490CF085FD10F04DFD80B20AF0C7FF07
:106528002B6C6549986C0CF07BFD10F043FD80B234
:106538000AF0BDFF2B6C93F84C000BE0234458780D
:106548000AF0B5FF2B6C2344D87A0AF0B0FF2B6C05
:106558002344587D01340AF0AAFF0A2CD4D17AE2E8
:1065680014F8010F002800F076820AF06EFFF7E7B2
:1065780001200AF099FF4D4B1B6C1878DFE1502081
:106588000AF092FF0025494B0C211C6C4B4B04EB85
:10659800850494F87920013501FB023393F838001B
:1065A8000AF053FF94F87A000AF04FFF94F87B0042
:1065B8000AF04BFF94F87C000AF047FF142DE2D153
:1065C80049E23A4B1C6C062303FB054494F8CE00C1
:1065D8000AF03BFF94F8C9000AF037FF94F8CA00A4
:1065E8000AF033FF94F8CB000AF02FFF94F8CC00A0
:1065F8000AF02BFF013594F8CD000AF026FF0C2D88
:10660800DFD128E24FF0000801260027274B1A7A2D
:10661800974227DA0933FA5C00240C236343274D99
:1066280005F13001595C914207D12B44586B10F0A9
:10663800F8FA82462EB9B14605E001341C2CECD19B
:106648000EE080440CE0D1450ADA0C2303FB045326
:106658005B6B13F809000AF0F8FE09F10109F2E78B
:106668000137D3E7002E00F0F6815FFA88F00AF0D0
:106678001BFF0026C9E70D4D0024287A0AF014FFF5
:106688002B7A9C4280F0E7810D4B0021E65C0C22BE
:1066980002FB01F3094800F13007DA5DB24211D17B
:1066A800034493F838000AF0D0FE0EE0E41000200E
:1066B800000020410000C84200007A44B09301085D
:1066C800ED10002001311C29E1D10134D8E7CE4C6E
:1066D80016200AF0E9FEB4F898010AF0E8FEB4F8CA
:1066E80044010AF0E4FEB4F846010AF0E0FEB4F80A
:1066F80048010AF0DCFEB4F8DA010AF0D8FE94F892
:10670800EF010AF0A2FE00200AF09FFE94F8F001C3
:106718000AF09BFE94F887010AF097FE94F894011A
:106728000AF093FE00200AF090FEB84B0A201B6C7A
:10673800B3F9563093FBF0F080B20AF0B8FE89E066
:10674800E0B201340AF081FE092CF9D183E110206E
:106758000AF0AAFEAE4BAF4C187800F002000AF01F
:1067680074FEAD4B18780AF070FE20680AF0A8FE97
:1067780060680AF0A5FEA94B18880AF098FEA84B95
:1067880018880AF094FEA14BB3F86C0059E00AF09F
:106798003FFE074612200AF087FE9C4C17B9266F69
:1067A800656F05E0102F19BF00252E46A66FE56F0F
:1067B80038460AF04AFE30460AF082FE28460AF0B9
:1067C8007FFED4F880000AF07BFE00200AF06FFEFE
:1067D80000200AF06CFE0020B1E08C4D002495F8F2
:1067E80084002E4680000130C0B20AF05DFE95F8A4
:1067F80084000AF02AFE96F884309C4280F02B81AF
:10680800884D285D0AF021FE05F11003185D0AF095
:106818001CFE05F12003185D30350AF016FE285DD0
:106828000AF013FE0134E6E708200AF03DFE0020D6
:106838000AF03DFE00200AF03AFE00200AF037FE7A
:1068480000200AF034FE06E104200AF02DFE6E4B0B
:106858009868FEE094F87C010AF0F7FD94F880014E
:106868000AF0F3FD94F87F010AF0EFFD94F8810136
:1068780065E0654C07200AF017FEB4F882010AF0BB
:1068880016FEB4F884010AF012FE94F886010AF0A4
:10689800DCFDB4F88801D4E75B4C0C200AF004FE58
:1068A80094F892010AF0D1FDB4F89C010AF0FFFDBA
:1068B800B4F898010AF0FBFDB4F89A010AF0F7FD64
:1068C80094F893010AF0C1FDB4F89E010AF0EFFDB7
:1068D800B4F8A001B5E74C4C04200AF0E5FD94F8A3
:1068E800D8010AF0B2FD94F8D9010AF0AEFDB4F867
:1068F800DA01A6E74C4C4D4D2078002600EB40000D
:10690800C0B20AF0D1FD237802359E4280F0A38000
:1069180015F8020C0AF099FD15F8010C013600EB88
:10692800800000EB800000F2EE2080B20AF0BFFD8C
:10693800E9E701200AF0B8FD334B93F894010AF017
:1069480084FD88E008200AF0AFFD00242E4B234484
:1069580093F88A0101340AF078FD082CF6D17AE020
:106968002A4B294C93F8C50004F12005C0EBC00060
:10697800C0B20AF099FD94F8F60100232C4AD25CC3
:1069880090426ED00C33302BF8D10834AC42F2D19F
:1069980061E040200AF088FD1B4C04F14005B4F882
:1069A800A8020AF084FD94F8AA020AF04EFD043405
:1069B80094F8A7020AF049FDAC42F0D14BE0E02080
:1069C8000AF072FD104C04F18005B4F82A02043470
:1069D80000F03F000AF06BFDB4F82602C0F3861001
:1069E8000AF065FD94F8240200090AF02EFD94F8D7
:1069F800240200F00F000AF028FD94F825020AF09E
:106A080024FDAC42E1D126E0D4110020E41000209E
:106A1800C8190020D0190020CE190020CC19002058
:106A2800CA19002069110020B4280020761300201C
:106A3800C028002013200AF037FD0024144B185DED
:106A480001340AF002FD0B2CF8D100200AF038FDC1
:106A580000200AF035FD0120BDE8F0870020BDE8E0
:106A6800F0870AF0F2FCB4F8F8010AF020FD94F877
:106A7800FA010AF0EAFC94F8FB010AF0E6FC94F843
:106A8800FD010AF0E2FC94F8FC010AF0DEFC7CE768
:106A980068B601082DE9FF47CB4C07462378CB4E53
:106AA800002B00F0E78132686368D31A7C2B40F230
:106AB800E181237A6260013323724FF0000808F104
:106AC8002400C14DC0B206F029FD05F10A0333F9CF
:106AD80018000CF051FABE4B814618880CF04CFA9D
:106AE800014648460CF050FBBA490CF099FA0CF0F4
:106AF8005DFC08F1010800B206F0FEFCB8F1030FD6
:106B0800DDD1302006F00AFDB5F9100006F0F4FCDE
:106B180006F0FCFC2B7A9A072CD141F288336A687C
:106B28009A4218D9102006F0F9FC68694FF06408F9
:106B380090FBF8F000B206F0DFFC212006F0EEFC36
:106B4800686990FBF8F308FB13000028B8BF4042BF
:106B580000B206F0D1FC142006F0E0FCB4F91800ED
:106B680006F0CAFC1C2006F0D9FC002006F0C4FC84
:106B780006F0CCFC237ADFF850825B0740F057819F
:106B8800022006F0CBFCD8F81C006423323090FBBE
:106B9800F3F000B206F0B0FCB8F926504FF0050A41
:106BA80095FBFAF5032006F0B9FC8B4BADB21B78C8
:106BB800DFF8389213F0040F0DD008F5D970394674
:106BC80001F0D1F928B9D9F8003013F0100F18BF27
:106BD800002528B205E0D8F804389889B0FBFAF007
:106BE80000B206F089FCD9F800309F076ED5DFF8AF
:106BF8000092B4F8082899F800304FF0640808FBB0
:106C080002325B00B2FBF3F3B4F80A7806203F01C6
:106C1800BFB247EA0327BFB2C3F303231F4306F0FB
:106C28007DFC38B206F068FCB4F80A3899F8001010
:106C380001339BB293FBF1F201FB1233A4F80A383B
:106C4800D4F80C38604D9B7B012B05D1392006F018
:106C580065FCB5F908081AE0B5F808586E235D43D5
:106C6800152795FBF7F53A20AFB206F057FCB7FBAE
:106C7800F8F528B208FB157506F03EFC3B2006F037
:106C88004DFCA8B2451D0A2095FBF0F000B206F0B5
:106C980033FC282006F042FCD4F810380A2093FB75
:106CA800F0F000B206F028FC042006F037FCD4F817
:106CB80004389B8913B108F083FD04E0424BD3F8F4
:106CC800140880F3100000B206F016FCD4F8183847
:106CD8003D4F9D0640F1A08097F81C3898071DD5B8
:106CE800112006F01BFCB7F81E084FF4F365684343
:106CF8003A4B90FBF3F000B206F0FEFB192006F0C9
:106D08000DFCB7F81E084543642095FBF0F595FB8C
:106D1800F0F300FB135000B206F0EEFB94F81C38B9
:106D2800B4F8205813F0020F08BF0025012006F020
:106D3800F5FB28B206F0E0FB092006F0EFFB002087
:106D480006F0DAFB264B94F822581A88B2F5967F9B
:106D58000AD91D4B1B7A03F00F03072B04D842F204
:106D68000F75954228BF1546052006F0D7FBD4F8C5
:106D78000C385B7B0BB928B216E0A5F120000CF0AB
:106D8800FBF818490CF000FA002105460CF0E6FA69
:106D980010B94FF07C5101E04FF03F4128460CF00C
:106DA80037F80CF003FB00B206F0A6FB94F81C2899
:106DB800054B910703D493F82328012A1AD10123FC
:106DC80084F8233808482EE0AC110020202D00203C
:106DD8001A00002000007A44E7300020A086010055
:106DE800460000206666E63FD0190020FC2C0020F3
:106DF80044000020D3F80C58C04968680CF010F91A
:106E08000CF0D4FABD490290A8680CF009F90CF00E
:106E1800CDFA039002A806E0B94A02AB92E8030053
:106E280083E80300184606F089FB06F06FFB237A17
:106E3800282B1FD1B34B00221A7233684FF47A7093
:106E4800B3FBF0F83C27172006F068FBB8FBF7F512
:106E5800B5FBF7F007FB1050000200B206F04CFB40
:106E6800182006F05BFB07FB158000B206F044FB18
:106E780006F04CFB94F82C38A24D002B00F06181F1
:106E880001F000F9D5F830389F4AC31A93420746F3
:106E980040F2C780002385F8363885F83838B5F8C9
:106EA8000838DAB21B0A85F8522885F8533885F86D
:106EB800482885F84938D5F8602833689A1AD5F8EB
:106EC8006438D97B4FF47A734B439A420ED38F4B75
:106ED8001B68C5F8603895F86838013B012B9FBFDF
:106EE800102385F83638022385F83838D4F8102866
:106EF8000A20D4F8143892FBF0F293FBF0F384F8EC
:106F08005028121284F8512884F8543894F81C2810
:106F18001B1284F8553894F822389207794984F876
:106F2800833803D42D2381F8843878E0D4F8249862
:106F38007748DFF8E8C199FBF0FA0CFB0A924FF0AA
:106F4800060E042B0EFB02F28CBF3323322381F88A
:106F58008438704BD4F8286892FBF3F196FBF0F074
:106F680003FB1122642592FBF5F20CFB006C0EFB6F
:106F78000CFE84F87528121284F876289EFBF3F22A
:106F880003FB12E393FBF5F30AEB8A0A4FFA81F845
:106F98000AEB8A0A08EB8A0189B284F8731800EBB5
:106FA8008000090A84F8741800EB800051B201EBE4
:106FB800800292B284F87828120A84F8792884F832
:106FC8007A38B4F81E281B1284F87B3824235343DC
:106FD80093FBF5F5B4F896380A2284F87C381B0A36
:106FE80084F87D38B4F820384FEAD979B3FBF2F346
:106FF80003F5FA739BB284F87E381B0A84F87F384D
:10700800B4F89838F60F84F87058C5F3072584F853
:10701800729884F8776884F8715884F88538C4F8C9
:10702800307894F89A88374DB8F1000F0DD1D5F81B
:10703800A00809F04BF8012807D90228364E00F0BD
:107048005E8202F041FD0123B370D4F8A4282D4DCF
:10705800002A76D095F89A683EB140F6B731D5F84F
:10706800AC38FB1A8B4219D86BE00123D5F8A0087D
:1070780085F89A3800F0ECFDD5F8B038082193F976
:10708800000002238DE8480032464FF4964301F091
:1070980080F885F8B468C5F8A00850E095F8A868A5
:1070A800CEB9D5F8A008C5F8A46885F89A6800F0A4
:1070B800CFFDD5F8B038082193F9000001238DE8F9
:1070C800480032464FF4964301F063F8C5F8A0082B
:1070D80002F0FAFC33E0013EF6B285F8A86895F8AC
:1070E800B41895F8B538DEB94A1C013385F8B428C8
:1070F80085F8B538D5F8A0081FE000BF8096184B72
:107108003C950108AC1100203F0D0300202D002004
:107118008096980040420F001A000020806967FF9F
:1071280012F8016B01337018314685F8B408D5F8A8
:10713800A008C5F8A42885F8B53808F0CAFFC4F82F
:10714800AC7894F8B638A14DF3B1D5F8B838DBB1BE
:10715800D5F8BC38C3B1C5F8C0381B689C4AC5F817
:10716800C438D5F8C8381344187AFEF769FDD5F83D
:10717800C03898790AF069F9D5F8C8380133092B6D
:1071880088BF0023C5F8C838924D94F8CC282E68DB
:107198008E4B002A00F0EE81D3F8D028002A00F0A8
:1071A800E98193F8D438013B012B00F2E381D4F84C
:1071B800D008864F08F08AFFE0B1D7F8D00808F069
:1071C80082FF97F8D53880467E2BD5F800900ED1EF
:1071D80002231B2887F8D43809D1D7F8D00808F03B
:1071E80075FF20B90123C7F8D89887F8DC3884F8E8
:1071F800D588DCE7D7F8D8282B689B1A41F658328F
:1072080093421ED9032387F8D438B3E1724A32F87F
:10721800130010B903464FF403600133B0F5C06F93
:10722800DBB279D01ED9B0F5006F7FD032D9B0F576
:10723800036F3FD184F8DD38D4F81838634F9906C6
:107248003FD494F8DC1894F8DD38002900F0548114
:107258002A68921B012AD9D984F8DD38002384F8DA
:10726800DC3887E1B0F5007F43D007D8B0F5807FE0
:1072780049D0B0F5887F00F08B80E6E7B0F5806FE5
:1072880000F0AE80B0F5826F00F0F380B0F5047FB7
:10729800DBD123E0B0F5E26F00F08B80B0F5E46F4E
:1072A80000F08C80B0F5E06FCFD184F8DD38B4F908
:1072B8000A1087E0B0F5046F74D0B0F5026FC4D13E
:1072C80003E197F81C389A07BBD5B7F81E18242392
:1072D8004B436421123393FBF1F107E184F8DD3865
:1072E8003E4B3A4F1B689B07ABD5B7F808380A21C5
:1072F800FBE084F8DD38394B344F1B681905A0D5FD
:10730800D7F81018F2E084F8DD38D4F818382F4F81
:107318005A0796D57969E9E084F8DD382F4B2B4F69
:107328001B681B058DD5D7F81418DFE0D4F818189A
:10733800264A8F0684F8DD3883D592F81C1888070A
:107348007FF57FAFD90711D5D2F82838192283EAFB
:10735800E371A1EBE37101EB5101B1FBF2F1002BF9
:10736800ACBF41F0004141F040410EE0D2F8243872
:10737800192283EAE371A1EBE37101EB5101B1FB3F
:10738800F2F1002BB8BF41F080414FF400608BE070
:1073980084F8DD38D4F818380C4F5B077FF551AF07
:1073A8003969A3E084F8DD38B4F918306421594309
:1073B8007AE084F8DD38B4F90C1003E0B4F90E1063
:1073C80084F8DD382C2391FBF3F16DE0AC1100203B
:1073D8003C950108202D00206AB70108FC2C0020EC
:1073E80084F8DD3894F8DE38644A0133DBB2032BC5
:1073F80088BF012382F8DE3842F2107394F8DE1851
:1074080059435F4B1B78D80748BF01319A0748BFDB
:1074180002315F07B4F8E03848BF0431D80748BFE5
:107428000A319A0748BF14311F0648BF2831D805CA
:1074380048BF28315A0748BF64311F0748BFC831C1
:10744800980548BF01F5C8719A0648BF01F57A71D9
:10745800DF0648BF01F5FA61580648BF01F57A61B1
:107468004FF4806002F0FCFA444B002283F8DC28D9
:10747800E7E6D4F81818DFF8048111F0200784F83B
:10748800DD3817D098F81C2812F0020F14BF4FF4FB
:107498007A71002112F0010F14BF4FF4FA63002330
:1074A8000B4494F82218194402F0DAFA002384F8FD
:1074B800DC38C6E6334B1B6819067FF5C2AE394681
:1074C80002F0CEFA88F8DC78BBE684F8DD38D4F828
:1074D80018382A4F9A067FF5B4AE97F81C389B07E0
:1074E8007FF5AFAEB7F820386421594302F0B8FAF7
:1074F800002387F8DC38A4E684F8DD383AE0B3786E
:1075080023B1C5F89C7886F802809EE5D5F89C38AA
:10751800FB1AB3F57A6FFFF498AD0123D5F8A008EC
:10752800B37008F0D0FD0646D5F8A00808F0CBFDEA
:1075380076067FF48AAD8A2802D08E280DD084E59D
:10754800D5F8183898067FF580AD95F89A38002B4D
:107558007FF47BAD05F6690306E095F89A38002BB1
:107568007FF473AD05F63403C5F8A4382D2385F8E8
:10757800A8386AE504B0BDE8F08700BFAC11002068
:10758800E7300020FC2C0020F8B504460E461746CC
:107598000025204620210FF036FB0446D0B10134E7
:1075A80020460FF093FBB0F5617F05DB40F634030E
:1075B8009842A8BF184601E04FF46170A0F56170C9
:1075C800192390FBF3F00DB9307000E070703B7830
:1075D80001333B700DB90125DBE72046F8BD30B516
:1075E80005460C46134629462246BDE83040014868
:1075F80002F03CBD5CB801087FB504780646E4B9E2
:10760800354B1921186800EB840090F87B5090F8EE
:1076180079204D4305F5617590F87A30009590F81A
:107628007C00414301F5617101912C4821460134E8
:1076380002F01CFD142CE3D14BE00FF047FB13289C
:10764800054641DC244B701C1C68202100238DF862
:107658000F300FF0D8FA1E35064670B101363046A5
:107668000FF034FB1A289FBF04EB850358709DF870
:107678000F30013398BF8DF80F30304620210FF0BE
:10768800C2FA064670B1013630460FF01FFB0D28CE
:107698009FBF04EB850398709DF80F30013398BFA6
:1076A8008DF80F3004EB85043046E11C0DF10F0214
:1076B800FFF76AFF9DF80F30042B0AD0601C0021E9
:1076C80004220FF06AFA04E0054800211322FFF7AC
:1076D80086FF04B070BD00BF241100207BB80108EC
:1076E80090B80108014809F063BF00BF96B80108C7
:1076F800F8B50478064674B9304D2146B5F8C62168
:10770800B5F8C8312E48013402F0B0FC042C05F15C
:107718000405F2D1F8BD2B490FF048FAA8B9274B58
:107728004FF47A714FF4FA62A3F8C611A3F8C8218E
:10773800A3F8CA11A3F8CC21A3F8CE11A3F8D0213D
:10774800A3F8D211A3F8D421F8BD30460FF0BEFA41
:10775800032805462BD8304620210FF054FA04465A
:1077680030B1013420460FF0B1FA0126074600E097
:107778000646204620210FF046FA10B9BDE8F84029
:10778800B0E701300FF0A2FA012EF7D140F2DC5336
:10779800A7F2EE229A42F1D8A0F2EE229A42EDD850
:1077A800064B703503EB8503DF801881F8BD06486A
:1077B80000210322BDE8F84011E700BFD4110020E2
:1077C800A4B80108B7B801080EC701082DE9FF41A0
:1077D80004780546002C34D16D4809F0E9FE6D4D5A
:1077E800686900210BF0B0FD002840F0CE802146EA
:1077F800694802F03BFC6869694602F0BDFA014637
:10780800664802F033FCA869694602F0B5FA0146F9
:10781800624802F02BFCE869694602F0ADFA0146BD
:107828005E4802F023FC286A694602F0A5FA013492
:1078380001465B4802F01AFC0C2C05F11005CFD16B
:10784800A3E0584905220FF0F5F938B9514B002249
:1078580003441030C0285A61F8D196E028465249AE
:1078680004220FF0E7F904462846002C3FD12021D6
:107878000FF0C9F9002800F08880451C28460FF051
:10788800D0F90746494B53F824601EB9484809F017
:107898008FFE7AE028463146FAB20FF0CBF9013470
:1078A8000028EFD13B4B0021C2181030C02851618D
:1078B8009E46F7D13F4B03EBC402D2F804C098466A
:1078C800BCF1000F04D131463B4802F0CFFB53E036
:1078D800002718F834309F42F5DA3B010EEB030518
:1078E800143563440FCB013785E80F00F1E70FF03B
:1078F800EDF90B28064643DC284620210FF083F9D2
:10790800054648B10135284602F0A0F9214B01246B
:1079180003EB0613586100E00446284620210FF0C7
:1079280072F9054640B10135284602F08FF9194B26
:10793800013403EB06139861284620210FF063F900
:10794800054640B10135284602F080F9114B013453
:1079580003EB0613D861284620210FF054F910B91B
:10796800FFF7C0FE11E0013002F070F9094B032C5B
:1079780003EB06163062F3D11048FFF727FF04E047
:107988000F4801210C22FFF72AFE04B0BDE8F08160
:10799800BDB80108D4110020D8B80108DEB8010824
:1079A80028C40108B7B80108E2B801087CB2010888
:1079B800E7B801088CB70108F6B801082FB6010826
:1079C80090B80108F0B5047887B0064614BB514B4F
:1079D80019201968062303FB041191F8CA5091F87D
:1079E800CE20454305F5617591F8C930009591F8A9
:1079F800CB50C831684300F5617001900879029056
:107A08004979454803912146013402F02FFB0C2C9B
:107A1800DDD17CE00FF05AF90B28044672DC3D4BAF
:107A2800701C1D68202100238DF817300FF0EBF82B
:107A3800064680B1013630460FF048F903289FBF4B
:107A4800062303FB045383F8CE009DF817309CBF30
:107A580001338DF81730304620210FF0D4F807464F
:107A680080B1013738460FF031F90D289FBF062342
:107A780003FB045383F8C9009DF817309CBF0133FA
:107A88008DF8173006266643A9193846CA310DF114
:107A98001702FFF779FD20210FF0B5F8074670B1FE
:107AA800013738460FF012F914289FBF9DF8173098
:107AB8007619013386F8CC0098BF8DF81730384610
:107AC80020210FF0A0F878B101300FF0FFF80D2851
:107AD8009FBF062303FB045383F8CD009DF817309E
:107AE8009CBF01338DF817309DF81730062B0ED048
:107AF800062202FB04500021C9300FF04EF8FFF7B0
:107B0800F1FD04E0054800210B22FFF768FD07B0EE
:107B1800F0BD00BF2411002002B9010890B8010887
:107B28002DE9F347047806464CB9204601A90AF026
:107B380071FD0134FFF7F4FF122CF6D17AE00FF053
:107B4800C5F8C5B2112D70D83C4C05F1D00704EB2F
:107B58004703701C202193F802800FF054F8384E28
:107B6800034630B9A8F10202D2F1000848EB020836
:107B780045E000F1010A597830460FF044F860B149
:107B8800032D8CBF03230023801BC0B23344184449
:107B980090F80490B9F1030F02D1FFF7A3FD49E073
:107BA800A9F10203D3F1000850464FF0200148EB39
:107BB80003080FF028F8D8B1B8F1000FEDD0013064
:107BC8000FF084F840F2ED2380B2984205DD40F6CC
:107BD800CA039842A8BF184601E040F2EE20A0F27E
:107BE800EE20192290FBF2F004EB4703D87002E074
:107BF800B8F1000FD1D104EB470383F8029004EBEE
:107C08004704A378F25CB8F1000F09D0E178192392
:107C18004B430C48294603F2EE2302F027FA09E009
:107C28002946094802F022FA04E0084800211122F6
:107C3800FFF7D5FC02B0BDE8F08700BFD4110020E3
:107C48005095010822B9010834B901080EC7010886
:107C5800002208490C2303FB02135968814204D10E
:107C68000022C2621A725A6070470132042AF0D1A7
:107C7800704700BFC028002010B5084B00221968C3
:107C880001EBC20393F90240844201D1981C10BD54
:107C98000132042AF4D1002010BD00BFBC28002006
:107CA800F0B5027887B08AB94A4C04F1200694F8F6
:107CB800F6210023484950B2595681426DD00C3301
:107CC800302BF7D10834B442F1D180E0002204927D
:107CD8000592451C0EF0FAFFC4B260B2FFF7CCFF64
:107CE800074618B18DF81040012400E004462846E4
:107CF80020210EF088FF054638B1013528460EF0E0
:107D0800E5FF0134ADF81200E4B200262846202130
:107D18000EF079FFB0B3451C28460EF0D7FF0022BD
:107D28002E495FFA82FE51F82230834204D0013294
:107D3800082AF5D1002300E0734651F82320824237
:107D480020D1022E0FD0032E12D05A1E012ED2B2ED
:107D580004D0042A13D88DF814300EE0042A0ED863
:107D68008DF8153009E0052B09D88DF8173004E097
:107D78009A1E052A03D88DF816300134E4B201366C
:107D8800042EC3D1052C03D807B0BDE8F040A9E400
:107D980004AB03CB3860796019E094F8FB010F4B12
:107DA80094F8FA5153F82000B4F8F821009094F8A8
:107DB800FD0153F82000019094F8FC0153F82000CD
:107DC80053F825300290064802F050F97AE707B0D8
:107DD800F0BD00BFD4110020C028002034A1010844
:107DE80043B9010838B1438811EA030003D08B4234
:107DF8000CBF01200220704730B50A4B0A491C68A5
:107E08000A78032A0AD81346551C04EBC303EAB2BE
:107E18009D882842F5D00A70981C30BD0A70002051
:107E280030BD00BFBC280020901A0020014B002262
:107E38001A70E1E7901A00202DE9F047877890F84A
:107E480003C0BBB2C7F1640E03EB83065C42C3F107
:107E580078001C4D5FFA8EFE7600CCF16408A4B25F
:107E680080B2A3B20FFA83F9B9F1000F04DC002B3A
:107E780014BF3B46012300E0734609FB09F25B434C
:107E880002FB0CF292FBF3F3434403FB09F30A22CF
:107E980093FBF2F333449BB225F8023FB1F800900C
:107EA8004A880A34C9EB020A1AB202FB0AF24FF4F2
:107EB8007A7392FBF3F3A4B24B4484422B80D0D163
:107EC800BDE8F087901A002010B5447800780022A9
:107ED80040F6C41102FB02F3193B634303F6C413D3
:107EE8005343434393FBF1F3034921F81230013222
:107EF800072AEDD110BD00BFAA1A0020104B04308C
:107F080033F91000B0F5617F05DB40F63303984282
:107F1800A8BF184601E04FF461700A7819235A4344
:107F280002F28332824208DA4A78534303F28333F7
:107F38008342B4BF0020012070470020704700BF73
:107F4800382D002010B500F1500302788A4203D181
:107F58008478C278944204D304309842F5D1002042
:107F680010BD012010BD0B4B1B6813F4805F0A4B3A
:107F7800B3F9063005D0C089421A934207DD084498
:107F880000E0008A8342B4BF00200120704701202E
:107F9800704700BFFC2C0020382D00201FB5084B6F
:107FA8001B681B0309D58DF80400039101230D20DC
:107FB80001A98DF8053001F0AFF905B05DF804FBB3
:107FC800FC2C00201FB5084B1B681B0309D58DF836
:107FD8000400029100230D2001A98DF8053001F05D
:107FE8009BF905B05DF804FBFC2C002010B5064B8E
:107FF80000241C700AF0C8FE044B83F82840DC6299
:108008001C865C6310BD00BFB8300020901A0020A9
:1080180010B510B9BDE81040E8E700230C225A4318
:108028000A4C1119125D824203D00133102BF5D18D
:1080380010BD074B586B18B14A784078824203D27A
:10804800002259631A86DA6210BD00BF20A4010815
:10805800901A002010B540001428A8BF142000234F
:10806800074A022199540B4499181424834201F8B1
:10807800014CF5DBFF21D1540F20BDE81040C7E7C4
:10808800D42C002010B50A4A0A4B11689B6800BF1F
:1080980012689142F7D1084A4FF47A70946B00FB4A
:1080A80004F2D31AB3FBF4F300FB013010BD00BF98
:1080B800202D002010E000E0901A002038B504467A
:1080C800FFF7E0FF0546FFF7DDFF401BA042FAD3AC
:1080D80038BD10B504462CB14FF47A70FFF7EEFFA7
:1080E800013CF8E710BD2DE9F84381460B26013E17
:1080F80031D01B4B10225A6108221A6109F101077D
:108108004FF032080525164C4046E36883F010030B
:10811800E360E36883F00803E360FFF7DAFFE368EE
:10812800404683F01003E360E36883F00803E360EC
:10813800FFF7CFFF45B1013DE5D14FF4FA70FFF7E6
:10814800C8FF4FF0FA08DEE7013FDCD14FF47A7040
:10815800FFF7BFFFCBE7034A034BDA60BDE8F883BC
:10816800000C01400400FA0500ED00E0024A136823
:1081780001331360704700BF202D0020024BDB6BDA
:1081880003B11847704700BF901A002003685B6965
:1081980018472DE9F743064689469DF82880114679
:1081A8001A469DF82C3000250C2068431A4FC41934
:1081B800C057B04202D1207A20B126E00135042D03
:1081C800F2D122E0012E0AD003DCF6B9009313485D
:1081D80007E01E2E0AD01F2E17D1012006E01048F6
:1081E8000093434604F0B9FA044605E004F056FE4D
:1081F80041460446FFF7CAFF4CB10C2303FB057543
:10820800267185F808906C6001E0002000E02046A7
:1082180003B0BDE8F08300BFC0280020003801404B
:108228000044004003681B69184710B504462046FF
:10823800FFF7F8FF18B90A20FFF74BFFF7E710BD63
:1082480038B500240B4D6059254409F0B1F9696827
:1082580011B1094801F00AFFA96811B1074801F0F6
:1082680005FF0748103409F0A3F9B4F5D87FE9D120
:1082780038BD00BF1C9A010862B9010868B9010835
:10828800E6C40108F0B585B004460EF0CAFC08281B
:1082980026D1621EE01D1F4912F8013F09681944E2
:1082A800497801F00301022908BF203B824213707C
:1082B800F1D1254604F1080715F8016B1648314637
:1082C8000EF0A1FC20B1284631460EF09CFC10B1FE
:1082D800FFF708FA1CE0BD42EED1204606F09CFEEE
:1082E8000E4809F065F900230D4A04A91A4492F8CA
:1082F8008A210A440849595C0133082B02F80C1CEE
:10830800F2D10023074801A98DF80C3001F0AEFE28
:1083180005B0F0BD580000203AD001086EB9010838
:10832800D411002028C401082A4B2B4C1E6880B5A4
:108338002068FFF77AFF3046FFF777FF206841791A
:108348008D0703D441F00201FFF720FF234B0822D9
:108358001A61234D10221A612B689A0341BF062324
:108368006371E37923F0010344BF43F00203E3712F
:10837800206807F0ABFE90B1184F08237B61164BBD
:10838800186807F0A0FE804602F032FB08B108F03A
:10839800FBF93046414607F09CFE08233B61304616
:1083A80007F094FE78B10D4F4FF01008C7F814800D
:1083B8003046D4F8009007F086FE0146484607F09C
:1083C80088FEC7F810802B689B03D1D505F01BFAEF
:1083D800CEE700BFC42C0020D01A0020000C0140BA
:1083E800FC2C00202DE9F04705460EF01AFC2F4E14
:1083F8000446D6F8088090B92D4809F0D9F82D4BD5
:1084080053F8241049B10123A34013EA080F02D0FE
:10841800294801F02BFE0134F1E7284822E02846DC
:10842800274922460EF006FC58B9264809F0C0F83C
:10843800254C54F8041F0029EFD01F4801F016FE00
:10844800F7E72B784FF000092D2B03BF013504F116
:10845800FF344FF0010A4FF0000A164B53F8297009
:1084680027B91A48BDE8F04709F0A2B828463946A6
:1084780022460EF0DFFBA8B9012000FA09F0BAF194
:10848800000F03D001F086FF114803E040EA08001E
:10849800B060104809F08CF83946BDE8F0470E483E
:1084A80001F0E4BD09F10109D7E700BFD4110020AC
:1084B80074B90108CC9B01087EB90108E6C401081B
:1084C80082B9010887B90108C89B0108E7B8010803
:1084D80093B901089CB9010827C4010810B50848D8
:1084E80009F066F8074B00241C741C64064B1C70CA
:1084F80007F092FF09F034FA044B1C6010BD00BF6E
:10850800A4B90108D01A0020E8300020C42C0020AB
:1085180070B5064600240B4BE518AA8816420AD007
:10852800E158094801F0A2FD2846002108F0D1FFD2
:10853800064809F03DF840F6BC4314349C42EAD1A1
:1085480070BD00BFC0A50108D0B90108E6C4010884
:10855800F0B504788BB005460CB1002436E04B4BDF
:1085680019680E2303FB0411B1F91D51B1F9192142
:10857800B1F91B31009591F8205101F58C700195E6
:1085880091F8215101F59071029590F90700039037
:1085980091F902103E4804912146013401F066FD2C
:1085A800082CDCD170E02D2B14D1072C1BDC2846BD
:1085B8000EF08CFB0AAB661C03EB440424F8100C89
:1085C80015F8013F303B092BFAD934462B78002B9C
:1085D800E9D104E0A3F13002092A09D8E5E7082C1B
:1085E800BDF8182009D00BB0BDE8F040FFF77AB805
:1085F800202BF8D101352646E7E7072AF3D840F2C1
:10860800DC55BDF81A00214BA0F2EE2189B2A9422F
:108618001B68E8D8BDF81C10A1F2EE24A4B2AC4245
:10862800E1D8BDF81E6004B237B2A742DBDB0DB259
:10863800AF42D8DCA542D6DBBDF8247007F164044C
:10864800A4B2C82CCFD8BDF826E00FFA8EF4112CAE
:10865800C9DCBDF82050B42DC5D8BDF82240B42CD3
:10866800C1D812B24FF00E0C0CFB0233A3F819015B
:10867800A3F81B11A3F81D6183F8205183F8214149
:1086880083F81F7183F822E10BB0F0BD241100209C
:10869800DAB90108F0B504468FB020460EF0C1FAE9
:1086A800C5B21DBBAB4808F083FFAB4C94F8D6109D
:1086B80009B9AA4853E049B294F8D42094F8D530BF
:1086C800009194F8D710A648019194F9D81007346E
:1086D800029194F9D210039194F8D3100491294689
:1086E800013501F0C3FC102DE0D1E2E720469D4999
:1086F80005220EF09FFA0546B8B929469A48702215
:108708000EF04BFA2846994B19680E2303FB001309
:1087180001300022082883F8232183F8242183F8D4
:10872800252183F82621F0D112E120469049042220
:108738000EF080FA05462046002D4AD120210EF081
:1087480062FA002800F00481461C30460EF069FAEF
:108758002C460746874B53F824502DB986480FB04E
:10876800BDE8F04001F082BC30462946FAB20EF06E
:1087780061FA01340028EDD1774A164602F17001FA
:10878800002382F8DA3082F8D63082F8D53082F8C1
:10879800D43007328A42F3D1784901EBC40191F809
:1087A8000822934210DAD1F80C72C3EBC302B01856
:1087B8003A44176800F1D401C0F8D47090880133A6
:1087C800888092798A71E7E729466D4801F04EFC66
:1087D8008FE06C4907220EF02DFA05462046002D41
:1087E80049D120210EF00FFA06460EF01AFAC4B24B
:1087F8006CBB654801F03AFC21466448013401F03D
:1088080035FC0E2CF8D1554801F030FC00246048A6
:10881800214601F02BFC0025544A012311680E2241
:1088280002FB0412D2F82321AB401342594B5A4998
:108838005A4808BF1946013501F018FC0E2DEBD136
:108848004648013401F012FC082CE0D180E03046A3
:1088580053490EF03FFA2C4600284CD0022C4FD03A
:108868000EF034FA06AB43F824004D4900200EF010
:1088780031FA0134F0E74A490EF02CFA002460B1CD
:10888800082C38D00EF022FA06AB43F824004449ED
:1088980000200EF01FFA0134F1E7082C2BD1069BBB
:1088A8000F2B28D8DDF81CE0BEF1070F23D8089F4E
:1088B8000D2F20D8099E06F16402C82A1BD80A9DEC
:1088C800FF2D18D80B98642815D80C99642912D84C
:1088D800884210DA0D9C032C0DD8324AC3EBC3032F
:1088E800134483F804E05F719E71DD711872597248
:1088F8009C722D4CD1E60FB0BDE8F040FEF7F2BEF9
:10890800069B072B20D807990D291DD80278722AB3
:108918000DD06E2A18D1154A0E20126800FB0323C9
:1089280001228A40D3F8231121EA020209E00F4A02
:108938000E20126800FB032301228A40D3F823117A
:108948000A43C3F8232101E0FEF7CCFE0D4CA4E650
:108958000FB0F0BD02BA0108D4110020E6C4010826
:108968002DBA0108B7B80108A81200202411002068
:10897800E2B801087CB20108E7B801081C9A0108AE
:10898800F6B80108FAB901086CB9010849BA010832
:1089980059C10108FBC8010841C801084EBA0108BD
:1089A80052BA0108A41200202FB601082DE9F74396
:1089B800047805468CB9324D95F8AB12B5F8A82263
:1089C80095F8AA322F4800912146013401F04EFB58
:1089D800102C05F10405EFD14EE00EF077F90F28C1
:1089E800044636DC284620210EF00DF9264EE4B266
:1089F800D6F84480451CA400002728460EF066F9E6
:108A08005FFA87F9B9F1010F83B208D0B9F1020F03
:108A18000BD0B3F5B47F24D2726C13530AE0FF2B4A
:108A28001FD8736C2344987004E0FF2B19D8736C1B
:108A38002344D87028462C210EF0E5F8054608B1E5
:108A4800013502E0B9F1020F0BD10137032FD4D160
:108A580012E00E4800210F2203B0BDE8F043FEF7F4
:108A6800BEBD08EB0400002104220EF096F803B006
:108A7800BDE8F043FEF736BE03B0BDE8F08300BFA3
:108A8800D411002054BA0108D01A002090B8010867
:108A98002DE9F04304788FB00546002C59D17C4B62
:108AA8000021142209A807AED3F848800EF075F803
:108AB8000722304600210EF070F800231A46A7005E
:108AC80005A8059308EB070583807249B5F802E00D
:108AD80031F813C01CEA0E0F0AD00E310DF1380C14
:108AE800595C02F1010E624402F81C1C5FFA8EF216
:108AF8000133072BE9D100210B46674AB5F802E09C
:108B080011F802C01CEA0E0F0AD006320DF1380C1B
:108B18008A5C03F1010E634403F8242C5FFA8EF398
:108B280001310629E9D118F807308DE841006A7843
:108B38005A49029209A81A0903F00F0301F081FAB1
:108B48002146574809AA013401F090FA202CA6D1F1
:108B58009BE00EF0BBF81F28044600F389802846E6
:108B68002021E4B20EF04FF81F2C02D9FEF7BAFD0F
:108B78008BE0474B451C9B6C002103EB840420468B
:108B880004220EF00AF80027464B09AE30460021B1
:108B98000A2217F803905FFA87F80DF0FEFF00230A
:108BA80015F8012B32B10A2B04D04A4502D0F254F1
:108BB8000133F5E74A4561D108F1FF33032B09D8A2
:108BC800DFE803F0100502420DF1230037E00DF154
:108BD80023011FE030460EF079F82378C0B243EA4B
:108BE800001006E030460EF071F8237800F00F0010
:108BF8001843207034E00133062B0BD02A4800F2CA
:108C0800F3269E5D9642F6D1034493F8ED226388DD
:108C18001343638011F8012F12B30023EEE70133E9
:108C2800072B0CD0204A02F2E6269E5D8E42F6D132
:108C380002EB4303B3F8D82263881343638010F828
:108C4800011F69B10023EDE730460EF03FF80F2809
:108C580004DC30460EF03AF8607001E000236370DF
:108C68000137052F90D1012407F034FD6CB97DE759
:108C78000E4800211F22FEF7B2FC06E02046002124
:108C880004220DF08AFF0024EEE70FB0BDE8F08360
:108C9800D01A0020F49C0108099D010868BA01084F
:108CA80077BA0108159D01081C9A010890B80108B7
:108CB8002DE9F04FAB498BB004460DF077FFAA4978
:108CC800002820460CBF012507250DF06FFFA74996
:108CD8000028204608BF02250DF068FF002808BFBD
:108CE8000425E90740F1E680A14808F061FC00206E
:108CF80008F06EFA9F4CA04808F05AFC9F4808F00C
:108D080057FC63799E4A013B52F823109D4801F0B5
:108D1800ADF99D4801F0AAF926460027D6F8148037
:108D2800002140460AF010FB20B1984801F09EF956
:108D3800002669E039469648D6F818B0D6F81CA03F
:108D4800D6F8209001F092F9404600210AF006FB7F
:108D580010B1202008F024FC06A9404601F00CF8C8
:108D680001468C4801F082F9584600210AF0F6FACB
:108D780010B1202008F014FC06A9584600F0FCFFAA
:108D88000146844801F072F9504600210AF0E6FADB
:108D980010B1202008F004FC06A9504600F0ECFFB2
:108DA80001467C4801F062F9484600210AF0D6FAEB
:108DB80010B1202008F0F4FB06A9484600F0DCFFBB
:108DC80001370146744801F051F90C2F06F11006DD
:108DD800A4D1AAE749B294F8D42094F8D5300091E8
:108DE80094F8D7106D48019194F9D810073402917E
:108DF80094F9D210039194F8D310049131460136B6
:108E080001F034F9102E03D094F8D6100029E1D1DE
:108E1800634808F0CDFB574B624C9F6854F8041F19
:108E280019B1614801F022F9F8E70E465F4B53F893
:108E380026404CB10123B3403B4203D05C48214655
:108E480001F014F90136F1E75A4808F0B1FB214660
:108E5800484B0AAA0B4493F88A311344564A8A5C51
:108E68000131082903F8102CF2D1002306A9534830
:108E78008DF8203001F0FAF8514808F099FB514874
:108E8800FEF70EFF504808F093FB4E48FFF700FE30
:108E98004E4808F08DFB4B48FFF788FD4C4801F021
:108EA800E5F84020FFF734FB4A4808F081FB4548C5
:108EB800FEF736FEAA0739D5474808F079FB474838
:108EC80008F076FB3F4808F0C3F9454808F070FB06
:108ED8003C48FEF791FB434808F06AFB3948FEF727
:108EE80071FD414801F0C2F83648FEF701FC3F48E1
:108EF80008F05EFB3348FFF72BFB00260E2777436D
:108F080000243B4A0123D26CA3403A44D2F80A20F9
:108F180013421ED101340E2CF3D10136082EEDD1A7
:108F28002B4801F0A3F88020FFF7F2FA6B0716D55B
:108F3800304808F03DFB304808F03AFB214808F07B
:108F480061F9234801F092F84FF48070FFF7E0FAD6
:108F580005E031462246294801F088F8DAE70BB0E7
:108F6800BDE8F08F83BA010893BE01088ABA0108E8
:108F780090BA0108D41100209EBA0108B0BA0108BD
:108F88007CB20108BCBA0108C7BA0108D4BA010802
:108F9800E1BA01086BB9010828C40108F9BA010847
:108FA800E9BA0108C89B010818BB0108CC9B010855
:108FB80026BB010833BB01083AD001083FBB0108B2
:108FC80048BB01082FB6010857BB010863BB01085D
:108FD800E6C4010871BB01087EBB010891BB01080A
:108FE8009FBB0108A9BB0108B8BB0108C6BB0108A3
:108FF800D01A0020D2BB0108E3BB0108F5BB010869
:10900800344B354A1B68126810B51A60334A116828
:109018005960516892689960DA60314A116819613B
:109028005168926859619A612E4A1168D9615168EC
:10903800926819625A622C4A118819855188598593
:109048009188D2889985DA85284A118819865188A5
:10905800598692889A86264A1188D9865188928894
:109068001987194621F83A2F224A1078002282429D
:1090780006DA214C34F81240013221F8024FF6E7A3
:109088001E4A1288A3F864201D4A1288A3F8662095
:109098001C4A1188A3F86C1051889288A3F86E10A6
:1090A800A3F87020184A3B2112689A66174A12687A
:1090B80092FBF1F2B2F5967FC8BF4FF0FF325A67C4
:1090C800134A1288A3F87820124A5289A3F85E201E
:1090D80010BD00BF802D0020CC300020302A002099
:1090E8003C2A0020482A0020CC110020081100202A
:1090F800B61100207F2A00202811002034290020E2
:10910800AC1000200E110020C01100200400002027
:1091180048110020141100202DE9F84305460E4699
:109128000D4B002493E88003B44213DA7B1933F91A
:10913800140008EB050333F9142009EB050333F990
:10914800143001341344022293FBF2F3C01A08F0DE
:10915800C9FFE9E7BDE8F883802D002070B54720F6
:1091680008F010FF174B1B681B0307D5164B174A4F
:109178005B6810681B68C01A08F0A5FF144E154CF0
:10918800154D307808F09FFF23682868C01A08F04A
:10919800A9FF63686868C01A08F0A4FF0F4B188815
:1091A80008F091FF0E4B188808F08DFF0D4B1888BA
:1091B80008F089FF337823742B68A3606B68E36039
:1091C80070BD00BF042F0020802D0020CC3000206F
:1091D800CE1900206C2D0020D0190020CC190020B9
:1091E800CA190020501100207FB5264C264E274D65
:1091F8002749284A284B20B128480088B0F5805FC5
:1092080031D2308891F820101278ADF8040028780F
:109218001C4D1B788DF806008DF807108DF8082076
:1092280001A8294606228DF809300DF09BFC30B3C1
:109238000198BDF808302860AB80532008F0A2FEE2
:10924800208808F040FFA07808F03DFFE37801A8E7
:109258000193237902936379039308F09BFE0F4BE4
:1092680000221A800BE0308891F8201020801278B4
:1092780028781B78A070E17022716371DDE704B073
:1092880070BD00BF201B00208C1A0020C8190020C8
:1092980094300020230F0020880F0020242F002066
:1092A800A0F17D03012B70B504460D460A4E05D882
:1092B80030687D2106F00DFF84F0200430682146D7
:1092C80006F007FF35B12B881C4404EB142404F086
:1092D800FF042C8070BD00BF7C1A00200A4A138846
:1092E80001331380094A136801331360084A13884D
:1092F80001339BB2202B01BF00231380054A13883A
:1093080008BF013313807047242F00200C2F002042
:10931800102F0020122F002038B53A4B05461B7835
:109328000C46083B012B6BD8452008F02BFE28463D
:1093380008F028FE0C2D23D004D80A2D0AD014D802
:1093480035B138BD0E2D4BD02ED3FF2D50D038BDA2
:10935800206849E0207808F015FE62796378002AD1
:1093680014BF80200020184300E0207808F00AFE8F
:10937800A07808F007FEE07808F004FE20793BE0CA
:10938800B4F9000008F095FEA07808F0FBFDE0783D
:1093980008F0F8FDB4F9040008F08BFEB4F90600F3
:1093A800BDE8384008F085BE637820788BB180F03E
:1093B800800008F0E7FDA468E0B208F0E3FDC4F31C
:1093C800072008F0DFFDC4F3074008F0DBFD200E9E
:1093D80012E008F0D7FD6068BDE8384008F082BEAA
:1093E800206808F070FE6068BDE8384008F06BBE81
:1093F800054808F0A5FD0020BDE8384008F0C2BDCA
:1094080038BD00BF5C2D002004C001082DE9F04FD5
:10941800BE4B8BB01A880193BD4F002A40F0A9803B
:1094280042F20103B7F8D607BA4EC21A5042504169
:10943800FFF7DAFEFFF7E4FD34684920254608F017
:10944800A1FDB54B04F11C09186808F03CFE55F85D
:10945800040B08F038FE284605F066FD04F11000FC
:1094680005F062FD4FF01008AC4D01232A6803FA9D
:1094780008F3134203D0D9F8000008F033FE08F1CE
:109488000108B8F1130F09F10409EDD104F128001E
:1094980005F03AFDB7F84431B4F92E00C01A08F0C7
:1094A80012FE2B68DB0408D59D4BB4F864001B88BA
:1094B800181AC0F30D0008F006FE2B68980403D5AF
:1094C800B4F8660008F0FFFD2B68590503D504F1D0
:1094D8006C0005F019FD2B681A0502D5A06E08F07E
:1094E80001FE2B685B0402D5606F08F0FBFD2B685A
:1094F800180403D5B4F8780008F0E5FDA04604F197
:10950800300005F001FD04F1360005F0FDFCB7F868
:10951800443138F93C0F0127C01A08F0D4FD814BBB
:109528001B789F4208DA38F9020FB4F93C3001374A
:10953800C01A08F0D7FDF2E72B68990505D5B4F9EC
:109548005E00A0F2DC5008F0CDFD3268764872600B
:10955800B260121A9110754A4A43531C032293FBB6
:10956800F2F202EB42029A1A7C2303FB02033360F5
:10957800D6E16F4B6F4A1B6811688B4206D00AA967
:1095880041F8203D00201360FFF7C6FE019B97F8C5
:10959800D6171B8897F8D7070B44013BB3FBF0F2AB
:1095A80000FB12338B4280F086815A4F0120FFF76F
:1095B8001BFEFFF725FD50203E687D6808F0E2FCA1
:1095C800BA683B6810681B687A680344106806F13B
:1095D8001C0BA3EB400008F085FD6A68736802A8BD
:1095E8009B1A0293AA68B36805F11C089B1A039397
:1095F800EA68F36810249B1A049305F095FC2A691D
:10960800336902A89B1A02936A6973699B1A0393C8
:10961800B369AA699B1A049308F0BCFC3F4901226C
:109628000B68A2401A428A4606D0DBF80000D8F838
:109638000030C01A08F056FD0134132C0BF1040B4E
:1096480008F10408EAD106F1260005F126010023F5
:1096580031F9024F30F9022F121B02AC44F82320D3
:109668000133042BF4D103214FF000094FEA890399
:109678005FFA83F902AB53F821206AB102F10800BE
:109688000F2802D849F0010906E08032FF2A94BF6A
:1096980049F0020949F0030911F1FF31E6D24846C1
:1096A800002408F06FFCA0460DF1080B09F0030236
:1096B800022A16D0032A1DD0012A4ED1B8F1000F74
:1096C80005D1DBF8004090462401E4B245E0DBF820
:1096D80000004FF0000800F00F00204308F052FC93
:1096E8003BE0B8F1000F0CD0DBF80000C0F303102A
:1096F80020432CE0B8F1000F1ED19BF8010008F0C0
:1097080041FC9BF8000008F03DFC26E0102F0020EB
:10971800D4110020802D00200C2F0020042F0020C1
:10972800002F00207F2A00208C2D0020DF7BEFBD3A
:10973800182F0020142F0020DBF80000C0F303309E
:10974800204308F01FFCDBF80000C0F3071008F006
:1097580019FCDBF800402401E4B20BF1040B06AB62
:109768009B454FEA9909A1D1B8F1010F02D12046D2
:1097780008F008FCDAF8003013F480541FBFB6F87C
:109788006420B5F864100124521A18BF02929A0492
:109798000AD50AAA02EB8401B5F86600B6F8662075
:1097A8000134121A41F8202C580513D502AA02EBED
:1097B800840C06F16A0E05F16A0000223EF9021FC8
:1097C80030F9028FC8EB01014CF822100132032A4C
:1097D800F4D10334190508D50AAA02EB8400A96E4E
:1097E800B26E0134521A40F8202C5A0408D50AAA3D
:1097F80002EB8400696F726F0134521A40F8202C12
:1098080018040BD50AAB03EB8402B5F87810B6F848
:10981800783001345B1A42F8203C00E0FCB1012C9E
:1098280003D1029808F05EFC19E0631E002002AA2A
:1098380052F823204000C0B20AB140F00100013BB9
:10984800F5D508F09FFB4FF0000802AB53F828004D
:1098580008B108F047FC08F10108A045F5DB302005
:109868000321FFF759FC36200321FFF755FC2F4B46
:109878003C201978FFF750FCDAF80030990506D536
:10988800B6F95E00B5F95E30C01A08F02BFC3A68EC
:1098980027487B687A60121A9110264ABB604A43AF
:1098A800531C032293FBF2F202EB42029A1A7C2326
:1098B80003FB02033B60204B1B681A0630D51F4C84
:1098C8001F4D22682B689A420BD162686B689A42D6
:1098D80007D1019B1B88102B11D11A4B1B885B06E3
:1098E8000DD1482008F04EFB206808F0FBFB6068AB
:1098F80008F0F8FB23682B6063686B600EE0124A7F
:109908000F4B11782A7C914208D1104A9968106847
:10991800884203D15268DB689A4201D0FFF71EFCE7
:1099280008F000FB0BB0BDE8F08F00BF7F2A0020D5
:109938008C2D0020DF7BEFBDFC2C00205411002073
:109948006C2D0020122F0020CE190020D0190020E5
:109958002DE9F84F0C9EC2EB030B394C0B9B0029E9
:1099680014BF4FF0060A4FF0040AF61A636805465A
:109978000133904613D1236853455ED2314A032BF5
:1099880098BF294652F823202F4808F0E9FA63685F
:109998000022013363602D4B05469A7113E00025C0
:1099A80011E02B4A1278954240DA0B9BE3B109FB90
:1099B80006F2995C01228A40264909680A4213D1B5
:1099C800636801336360D4F804900A9B1C4F99457F
:1099D800E7DB2BD10A2008F0D5FA3B6801333B605E
:1099E8004FF0FF337B6021E0184A917921B12C2098
:1099F80008F0C8FA013501E00121917109FB0BF368
:109A0800226808EB030752B958F8030008F098FADF
:109A180097F9041005444B1CD2D00F4802E03A4491
:109A28000E48117908F09CFA0544C9E720685045AA
:109A38002CBF00200120BDE8F88F0020BDE8F88F7A
:109A48001C2F0020D89D01080FC00108201B0020F2
:109A580054000020042F00201EC0010859C101082D
:109A680030B585B004AC002524F8025D0091ADF84E
:109A7800060021461020FFF713FC9DF8060021463A
:109A8800FFF70EFC9DF807002146FFF709FC9DF83B
:109A980000002146FFF704FC9DF801002146FFF76E
:109AA800FFFB9DF802002146FFF7FAFB9DF8030033
:109AB8002146FFF7F5FB9DF80E002946C043C0B2CA
:109AC800FFF7EEFB05B030BD10B5054C206806F079
:109AD800FDFA18B1206806F0F6FAF6E710BD00BFE7
:109AE8004C1A0020F0B50124B0FBF4F58D4201D3E7
:109AF8004C43F9E70026D4B1B0FBF4F504FB15009C
:109B0800B4FBF1F41EB9002D01DC002CF3D1092DB2
:109B180003F1010EEFB204DD002A14BF37255725E3
:109B280000E030253D441D7001367346E3E71C70A4
:109B3800F0BDF0B50124B0FBF4F58D4201D34C43E0
:109B4800F9E70026D4B1B0FBF4F504FB1500B4FB2B
:109B5800F1F41EB9002D01DC002CF3D1092D03F11D
:109B6800010EEFB204DD002A14BF3725572500E0A7
:109B780030253D441D7001367346E3E71C70F0BD87
:109B880003685A1C0260197070472DE9F843089E53
:109B9800002B074688461446334614BF4FF0300959
:109BA8004FF0200913F8012B0AB9254603E0002CD1
:109BB800FBDD013CF6E7002D04DD38464946C04789
:109BC800013DF8E7354624EAE474A01B284415F85B
:109BD800011B11B13846C047F7E7BDE8F883024BCF
:109BE800186806F076BA00BFB8100020F8B5074626
:109BF8000C464868002115461E4609F0A5FB58B1D9
:109C0800284609F0B9F9104909F00AFA01464FF057
:109C18007E5009F0B9FA60606168304609F0F8F8DA
:109C28000146304609F0B0FA256806462946384606
:109C380009F0ECF80146304609F0F2F901462846E9
:109C480009F0E6F82060F8BDDB0FC9402DE9F041C6
:109C580002780346202A00F10100F9D0092AF7D03A
:109C68002D2A02D10346414D04E02B2A08BF0346A2
:109C78004FF07E551C460026234614F8012BA2F10E
:109C88003007F9B209290DD83949304609F0C8F921
:109C98000646384609F070F90146304609F0B8F82A
:109CA8000646E9E72E2A17D1314F234614F8010B4F
:109CB8003038C2B2092A0FD809F05EF9394609F0DE
:109CC80063FA0146304609F0A3F8294906463846A2
:109CD80009F0A6F90746E8E71A7802F0DF02452AF4
:109CE80039D15A782D2A02D10233012704E02B2AD0
:109CF80014BF013302330027013B002413F8012F5E
:109D0800303AD1B2092903D80A2101FB0424F5E726
:109D1800B4F59A7F28BF4FF49A74A0464FF07E534B
:109D2800B8F1070F07D91846124909F079F9A8F1CF
:109D380008080346F4E704F0070434B118460C4950
:109D480009F06EF9013C0346F7E719462FB1304692
:109D580009F01AFA04E04FF07E51304609F060F934
:109D68000146284609F05CF9BDE8F081000080BF93
:109D78000000204120BCBE4C30B5054687B00C46DB
:109D880003A800210C220CF008FF2846002109F046
:109D980003FB20B12846284909F03AF803E0284691
:109DA800254909F033F8254909F03AF909F0FEFA8E
:109DB800054680EAE0706946A0EBE57008F02AFCE9
:109DC800002DACBF20232D2368468DF80C300CF0F5
:109DD80028FF012807D130238DF80D308DF80E307B
:109DE8008DF80F300CE0022805D130238DF80D30A6
:109DF8008DF80E3004E0032804BF30238DF80D30B1
:109E0800694603A80CF0F0FE03A80CF00AFF03381B
:109E1800C5B22A4603A920460CF02EFF002363553D
:109E2800204607490CF0E0FE03AB204659190CF018
:109E3800DBFE204607B030BD6F12033A00007A44BB
:109E480042C0010870B50646B6FBF2F4084615464E
:109E580014B12046FFF7F6FF05FB1464024B1B5DA7
:109E680000F8013B70BD00BF44C001082DE9F04F68
:109E780081468A4616461C4689B000253178002955
:109E880000F0DB80252902D00136484674E072785C
:109E98004FF00008302A0CBFB278B71CA2F130038B
:109EA80012BF4FF0000BF71C4FF0010B092B19D80C
:109EB800A2F13003D9B2092905D80A2202FB0838D1
:109EC80017F8012BF4E7A2F16103052B02D8A2F1E0
:109ED800570305E0A2F14103052B03D8A2F137038C
:109EE8000A2BEADD6C2A30D13A787E1C642A00F00D
:109EF80083800BD8252A3DD003D8002A00F09D8006
:109F0800BCE7582A0CD0632A19D0B7E7732A22D0A5
:109F180002D86E2A37D0B1E7752A5CD0782AADD13D
:109F2800271D2068A2F1580462424FF010016241D7
:109F380055E02CD9582A32D0632A2AD13E464846C1
:109F48002178271DD04701350FE0642A63D00ED948
:109F5800732A14D13E462368484600935146424628
:109F68000023FFF712FE271D05443C4686E7252AF5
:109F7800DFD13E4648462521D04701357EE70AD83D
:109F88006E2A06D13E46236804341D6076E7002A0F
:109F980053D03E4672E7752A26D0782AF9D1A2F125
:109FA800580304F1040C5A422068CDF80CC04FF055
:109FB80010015A4105ABFFF795FDDDF80CC03E4690
:109FC800644605AB00934846514642465B46FFF758
:109FD800DCFD054452E72068271D0A21002205AB55
:109FE800FFF7A7FD3C46ECE704F1040CCDF80CC0E4
:109FF80020680A210022DDE72068271D002808DAEA
:10A008002D238DF8143040420DF115030A2100224A
:10A01800E6E705ABFAE7206804F1040C00280ADA41
:10A028002D238DF8143040420DF11503CDF80CC0E6
:10A038000A210022BFE705ABF8E7284609B0BDE8CA
:10A04800F08F0EB40FB505AB53F8042B01900649F9
:10A0580001A80393FFF70AFF019B00221A7004B0BE
:10A068005DF804EB03B07047899B00080FB413B583
:10A078000B4904AB08680B4953F8042B0968019392
:10A08800FFF7F4FE0446084B1868FEF7CBF80028E3
:10A09800F9D0204602B0BDE8104004B0704700BFB8
:10A0A800CC000020C8000020B810002080EAE0732F
:10A0B800A3EBE0738B4206DB002801DD401A7047F2
:10A0C80002D0084470470020704770B5044609F074
:10A0D8006DF92030402857D820462C4909F05CF902
:10A0E80028B120462A4908F091FE0446F4E72046A4
:10A0F800284909F033F928B12046254908F088FE97
:10A108000446F4E72046244909F046F930B12249CB
:10A11800204608F07BFE01461F480AE020461F49FA
:10A1280009F01CF940B11C49204608F071FE0146AF
:10A138001A4808F06BFE04462146204608F070FFD6
:10A1480005462046294608F06BFF1549064628466D
:10A1580008F066FF134908F059FE0146284608F042
:10A168005FFF114908F054FE0146284608F058FFE1
:10A178000E4908F04BFE0146304608F051FF0146F3
:10A18800204608F045FE70BD002070BDDB0F494039
:10A19800DB0FC940DB0F49C0DB0FC93FDB0FC9BF6D
:10A1A8009A7C2E36FAAF4F393587083CA4AA2A3E46
:10A1B80008B5034908F02CFEBDE8084085E700BF54
:10A1C800DB0FC93F2DE9F04F056885B08146284669
:10A1D8000C46FFF7EDFF80462846FFF776FFD9F8D3
:10A1E800045006462846FFF7E3FF07462846FFF7D0
:10A1F8006CFFD9F8089005464846FFF7D9FF824614
:10A208004846FFF762FF41468146504608F008FF7E
:10A2180041468346484608F003FF514601903046C0
:10A2280008F0FEFE49460290304608F0F9FE39462D
:10A238000390504608F0F4FE4946206007F10040BC
:10A2480008F0EEFE29466060A560029808F0E8FE76
:10A258000146019808F0DCFD2946E060039808F003
:10A26800DFFE0146584608F0D1FD3946206106F167
:10A27800004008F0D5FE29466061584608F0D0FE37
:10A288000146039808F0C2FD2946A061019808F02C
:10A29800C7FE0146029808F0BBFD4146E06138461A
:10A2A80008F0BEFE206205B0BDE8F08F2DE9F04150
:10A2B80007688AB0466885680446084601A9FFF71A
:10A2C80081FF0199384608F0ABFE04998046304674
:10A2D80008F0A6FE0146404608F09AFD0799804618
:10A2E800284608F09DFE0146404608F091FD029977
:10A2F8002060384608F094FE05998046304608F0FC
:10A308008FFE0146404608F083FD0899804628469E
:10A3180008F086FE0146404608F07AFD0399606021
:10A32800384608F07DFE06990746304608F078FE64
:10A338000146384608F06CFD09990646284608F09B
:10A348006FFE0146304608F063FDA0600AB0BDE824
:10A35800F081074B10B51A881C4622EA000090428B
:10A36800188002D00120FDF775FE208810BD00BFBF
:10A378008C1A0020064B10B51A881C4610439042D0
:10A38800188002D00120FDF765FE208810BD00BFAF
:10A398008C1A0020024A936823EA000090607047F4
:10A3A800D411002008B5104B1A780023D9B2914275
:10A3B80007D20E49002051F823100133096808809C
:10A3C800F4E73220FDF785FE094B1B685A0309D5CF
:10A3D800084B9B685B0305D4BDE8084040F2DC509D
:10A3E800FDF777BE08BD00BF7F2A0020802A002025
:10A3F800FC2C0020D41100202DE9F34108F0A2FC28
:10A408004B4A6923137040F2DC735380BE231371E7
:10A41800EF2382F8D93700231946164682F8DA372F
:10A42800F25C0133514040F2DC729342F8D1404B68
:10A43800404A83F8DA17404B04275A6002F1883201
:10A448005A600020013F17F0FF075FD03A4B3422D3
:10A45800DA60002454B100234FF4005056F8048009
:10A46800019304F057FF0428ECD11DE04FF430208D
:10A4780004F050FF0428E5D12F4D4FF430202B690C
:10A4880043F002032B612D4B6B612B6943F04003B2
:10A498002B6104F03FFF41F6FD732A69042803EAA3
:10A4A80002032B61D7D0CDE7234D1FFA88F22B6921
:10A4B8004FF4005043F001032B6104F1006303F5EE
:10A4C8007E331A8004F026FF042814D11C4B4FEA6F
:10A4D800184823440193019B4FF40050A3F80080CF
:10A4E80004F018FF41F6FE732A69042803EA020300
:10A4F8002B6106D0A6E741F6FE732A6913402B614B
:10A50800A0E740F2DC7304349C42A3D10A4A042831
:10A51800136943F08003136102D107F077FA10B989
:10A528000520FDF7E0FD08F0F7FB02B0BDE8F0817B
:10A53800D4110020230167450020024000F80308D9
:10A5480002F803082DE9F04107F060FA10B9042079
:10A55800FDF7C9FDB84C08F0F5FBB84940F2DC72CC
:10A5680020460CF00FFB94F8B0374FF4CC71022B57
:10A5780084BF002384F8B03794F8B027B04D01FBAE
:10A5880002F303F53A7020442344286093F83C030F
:10A5980001FB0242022803F54E7384BF00201871A4
:10A5A80092F83C33A74A13700C2202FB0343A64AD5
:10A5B80003F2B273136046F20902A3681A401AB98B
:10A5C8009D4A43F400539360A368DE0703D54FF414
:10A5D8000050FFF7DFFEA368580409D50820FFF7ED
:10A5E800D9FE4FF40050FFF7D5FE0120FFF7D2FE49
:10A5F800A368190706D54FF40050FFF7CBFE0120DA
:10A60800FFF7C8FEA3689A0413D54FF40040FFF77C
:10A61800C1FE894B93F88631012B03D14FF40060BA
:10A62800FFF7B8FE4FF48030FFF7B4FE4020FFF785
:10A63800B1FEA3685B0603D54FF48030FFF7AAFE8E
:10A6480094F8E0217C4B2AB193F8E42112B100225E
:10A6580083F8E4214FF0000C67467C4E7C4B1E606B
:10A6680004EB0C03B3F8F8E14FEA5E0101F077312F
:10A678004FEA9E0303F03333C1EB0E00C11A4FEAD1
:10A68800DE0303F01133CB1A03EB231303F00F326D
:10A69800FF2392FBF3F31EF00108C3EB032318BF5B
:10A6A8000137A2EB030318BFFFB2012B0ADD022B0F
:10A6B80040F0BE80B8F1000F00F0BA801EF0BC0F69
:10A6C80000F0B6800CF1080CBCF1200FC8D1013F96
:10A6D800012F00F2AD8007F075F9302200215D48A6
:10A6E8000CF05BFA5C4F5D4BD5F800801F605C4B4B
:10A6F800002108F17900C3F80080FDF723FC594BCD
:10A7080080F001001870584B07F126021A60574B69
:10A7180007F1D4021A6098F8000005F047FF28688E
:10A72800534B00F5C5721A6000F0E0FC514B94F8E9
:10A73800D81107F194021A6064224A434E4BC8327A
:10A748005A6000229A60DA601A615A619A61DA6185
:10A7580083F8202083F82120484B2D6807F12C022C
:10A768001A60474B05F219121A60464B05F2891216
:10A778001A60454B07F108021A60444BDFF848811C
:10A788001F60434B07F1A0021A6007F1AA03C8F83B
:10A798000030404BB4F866011E6008F0E9FBC8F8C9
:10A7A8000800B4F8680108F0E3FB95F85C3008F19C
:10A7B800040288F8043095F87830C8F80C0088F856
:10A7C800053094F8E331286E88F81030324BC8F819
:10A7D80014501A60314B05F164021A60304908F0D0
:10A7E8001FFC01464FF07C5008F0CEFCB5F816412E
:10A7F8002C4B1860204608F0BFFB01462A4808F099
:10A80800C3FC2A4908F00CFC294A2A4B15602A4A3D
:10A81800186005F168031360284A05F211151560E0
:10A82800274A1760274ABDE8F041136008F074BA58
:10A8380004F0C8FB4FE700BFD411002000F803085C
:10A8480024110020A82C00204C1100205E130020A9
:10A8580088300020BC0F002018130020F00F0020C3
:10A86800F40F002018000020C8070020F005002081
:10A8780000100020CC270020943000202008002061
:10A888001C1B0020280A0020502B0020542B0020DD
:10A898003C090020000A00205008002088080020F9
:10A8A800DB0F494084080020000061444C3D0F4400
:10A8B800900700203809002084070020280900207C
:10A8C800300900207C060020281B002008B5FFF76F
:10A8D80093FDFFF737FEBDE808400120FDF7BABB3E
:10A8E80010B508F049FB0021044608F055FD08B1F1
:10A8F800204601E004F10040054908F045FC0549FF
:10A9080008F08EFBFFF754FC034B186010BD00BF26
:10A918008096184B35FA8E3C3C0000202DE9F0411A
:10A9280005460E46078A83899BB21F40002F37D001
:10A93800B7FA87F24FF00043D340DB4399B21F4088
:10A94800A2F11B032982042BF0D8DFE803F0221FB1
:10A958001C190300746A24B1013C0023A4B2736279
:10A9680001E0AC8DA4B2D6F82080B8F1000FDDD09C
:10A97800D8F80030404621469847D8F80480F4E7D4
:10A988003068A98E08E07068298F05E0B068A98F43
:10A9980002E0F068B5F84010036889B29847C5E747
:10A9A800BDE8F08138B50D4B0D4D99680D4B1A680F
:10A9B8001C465288114203D0FDF764FB286007E06B
:10A9C800FDF760FB2B68984282BFC01A064B1860DF
:10A9D80023685A68054B5A6138BD00BF000C014016
:10A9E800401B0020980700200400002000040140BC
:10A9F800F8B59C4B04461B68187818B1012800F07C
:10AA08006A819AE2242C984D0CD006D80A2C00F0C2
:10AA1800D9800D2C00F0D68048E12A2C06D02C2CA9
:10AA280004D043E128716871A87150E18F4B6979AE
:10AA38002F7900208C4A58542FBB1978D771472991
:10AA480021D1597850291ED19978472907D1D97829
:10AA5800472904D11979412901D10121D171997866
:10AA6800824A522903D1D1784D2900F06882997819
:10AA78007E4A472907D1D178532904D11279562A19
:10AA880004BF0322EA71EA79774E022A39D0032AF1
:10AA98004CD0012A40F08580BA1E072A00F2818036
:10AAA800DFE802F004080F131A257F2A07F006FDD5
:10AAB800A86076E01B78532B73D1AB685B42AB6020
:10AAC8006FE007F0FBFCE8606BE01B78572B68D160
:10AAD800EB685B42EB6064E01B78302B644B1A78C0
:10AAE8008CBF42F0020222F002021A7059E00020E4
:10AAF80007F044FD287454E0002007F03FFD688209
:10AB08004FE0072F06D0082F4BD1012007F036FD64
:10AB1800F08246E0012007F031FD41F21843584326
:10AB28004FF47A73B0FBF3F0B0823AE0022F07D00B
:10AB3800032F0AD1002007F021FD4E4B187030E09A
:10AB4800002007F01BFD30762BE02AD93A1F92101F
:10AB5800337E0132D2B2013B02EB8303DBB2102B0E
:10AB68001FD8F91EC2F1010201EB8202D2B2012AFA
:10AB78000BD0042A11D100205E1E07F0FFFC3E4BCB
:10AB8800002298553D4B9A5507E03D4A5E1E00202D
:10AB9800935507F0F3FC3B4B98553B4A1368013338
:10ABA8001360314B2A2C18BF9A7907F101074FF02F
:10ABB80000000CBF012254402F7168710CBF5A76F7
:10ABC8009C7184E0687E002848D0304B13F8012D32
:10ABD8002F495A708B42F9D1244A234C1378527862
:10ABE800402B85BF373B1B011B01DBB298BF03F02D
:10ABF800F003402A8CBF373A303AD2B21344AA79CC
:10AC0800DBB29A4227D121230B702249E0790B68E5
:10AC1800012803F101031E4A0B600AD002281CD147
:10AC280072231370A28A1C4B1A80E28A1B4B1A806B
:10AC380013E0672313700E4B1B789F070ED5184B34
:10AC4800A2681A60E2685A60227C164B1A70628AFF
:10AC5800154B1A8002E03F230B70002000236B760F
:10AC680035E000BFBC070020401B0020282D002035
:10AC7800C8190020681100209911002089110020AE
:10AC8800691100207911002030270020C40200201B
:10AC9800B00200203C270020CA19002050110020D3
:10ACA800D0190020CE190020CC1900206B79687EBD
:10ACB8000E2B9FBFA54A591C5171A54A98BFD45461
:10ACC800A24A18B993795C40947100E000200030E2
:10ACD80018BF0120F8BD9D4B0022997E082900F27B
:10ACE8002C81DFE801F0050B0F15202B475D67006D
:10ACF800B52C40F02281DA76012239E0622C08BFB7
:10AD0800022235E003229A761C775C779C7714E15F
:10AD180004229A765A7F997F2244D2B25A770A44FB
:10AD28009A77DC7709E105229A765A7F997F22443F
:10AD3800D2B25A770A449A771C84FEE006229A76A1
:10AD48005A7F997F2244D2B25A770A449A771A8C4A
:10AD580002EB0424A4B2B4F5AC7F82BF7B4A012184
:10AD6800D17600221C845A84002C40F0E680072209
:10AD78009A76E2E05A7F997F2244D2B25A770A44FF
:10AD88009A775A8CB2F5AC7F3EBF7049891881F822
:10AD980024400132198C92B291425A84E7D9CCE00E
:10ADA80008229A765B7FA34200F0C780674B012296
:10ADB800DA760DE0674D9A7615F8012D6A70664AC5
:10ADC8009542F9D1997F614AA14206D03F232B7061
:10ADD800624A536801335360AFE06148016801314A
:10ADE8000160D07E10B13E232B70A6E0212129708E
:10ADF800D17F062941D004D8022907D0032923D0BE
:10AE0800F8BD122959D0302967D0F8BD5021946A6D
:10AE1800297054494C60D46A0C60516B4FF47A74B1
:10AE280091FBF4F1504C218092F87C114F4A19B1F2
:10AE3800117841F0020102E0117821F0020111704D
:10AE4800012283F87D2169E05321297092F82910A5
:10AE5800CE0705D592F82820D51E6A426A4100E03F
:10AE6800024602F0010183F87C11002A56D13F49BD
:10AE78000A7822F002020A7050E04F21297092F8F5
:10AE88002F10CC0705D592F82E20D11E4A424A41F0
:10AE980000E0024602F0010183F87C1122B933492F
:10AEA8000A7822F002020A7093F85310304A11709F
:10AEB800B3F850102F4A118030E05621946B297056
:10AEC8002D490C8042F21074D16B91FBF4F12B4C9C
:10AED8002180012182F87E1120E04921297092F811
:10AEE8002810274A102988BF102111702549147885
:10AEF8000022A2420ED20E7A234D56554E7A234D89
:10AF08005655CE7A224D565511F80C6F214D56558F
:10AF18000132EEE720490A6801320A6093F87D3170
:10AF28000A4A002B3AD092F87E31BBB3002182F84E
:10AF38007D1182F87E111846F8BD0020F8BD1279FF
:10AF4800432A7FF494AD0222EA7190E5401B002069
:10AF5800282D0020C4020020B00200209C070020F9
:10AF68003C270020D0190020CC190020C819002047
:10AF7800CE19002046000020CA19002050110020D8
:10AF880068110020641B002069110020791100203D
:10AF9800891100209911002030270020F8BD0449AC
:10AFA800044B0968002218705A6199611A77704732
:10AFB800202D00209C070020F8B5101A0D461F46CA
:10AFC80007F0DAFF0446781B07F0D6FF174B079EF9
:10AFD800196808F025F821460546204608F020F8AB
:10AFE80029460746284608F01BF80146384607F068
:10AFF8000FFF0CF043FA0E4908F012F808F0FCF9BC
:10B00800069B2946186004F100400CF0ABF809498A
:10B0180008F006F8084907F0FBFE08F0C7F9002811
:10B02800BCBF00F50C40A0303060F8BD3C000020EB
:10B038002C7D8E3FA00CB34500A00C4644F2506313
:10B04800984203DDA0F50C40A0387047034B9842A6
:10B05800BCBF00F50C40A030704700BFB0B9FFFF7F
:10B06800F7B50368174C184D23600B68174E6360DB
:10B078000068FFF735FC95E80300154B019600932F
:10B0880094E80C00FFF798FF3668124B60681E6062
:10B098006B68114FC01A07F06FFF104B196807F063
:10B0A800BFFF08F083F92A68236878609B1A3B6021
:10B0B8000B4B1E600B4B1B68DA880B4B1A8003B0D6
:10B0C800F0BD00BF482C0020D0190020542C0020CF
:10B0D800502C0020902C0020582C00203C000020F0
:10B0E800882C002000100020842C002070B5044615
:10B0F800407907F03DFF1E4908F046F81D4D1E4EE9
:10B108002860E07B07F034FF194908F03DF8EE604D
:10B118006860A07907F02CFF184908F035F8184D39
:10B128002860207C07F024FF114908F02DF868609A
:10B13800A07E07F01DFF134908F026F8EE60A8600E
:10B14800E07907F015FF0D4908F01EF80E4D28604C
:10B15800607C07F00DFF064908F016F86860E07E8D
:10B1680007F006FF074908F00FF8EE60A86070BD09
:10B178000000C842602C00200000FA440000204172
:10B18800702C002000007A44942C002010B50C4C40
:10B1980023789B0713D50B4B1B78042B0FD90A4A2E
:10B1A8000A4B1068526818605A60FFF799FB084B01
:10B1B8001A88084B1A80237843F00103237010BDC6
:10B1C800C8190020CE190020D019002054110020E1
:10B1D800C4110020A42C0020164B13B51B681B03B8
:10B1E80025D5154B154C1B7815498DF80030154B96
:10B1F80020681B788DF8013007F012FF08F0FCF882
:10B2080011498DF80200606807F00AFF08F0F4F8A9
:10B218008DF80300A06808F0EFF80C4B8DF80400D7
:10B228001B780A2069468DF80530FEF775F802B0DC
:10B2380010BD00BFFC2C0020EE2C0020102D00209B
:10B24800000020410C2D002000007A44F22C002040
:10B25800054A137883F001031370044A002313602E
:10B26800034A1360B8E700BFF22C0020082D002025
:10B27800042D002001480249FFF750BB0008004098
:10B28800282B002001480249FFF748BB0004004072
:10B29800002B00204FF080400149FFF73FBB00BF63
:10B2A800D82A002001480249FFF738BB002C01408A
:10B2B800B02A002001480249FFF730BB002C0140AA
:10B2C800B02A0020254B10B55A43254B254C1B6846
:10B2D8000139B3FBF2F20388013AA04289B292B273
:10B2E8009BB212D004F50064A0420ED0B0F1804F9A
:10B2F8000BD0A4F59834A04207D004F58064A0428E
:10B3080003D004F58064A04202D123F070039BB2FD
:10B31800154CA04206D004F58064A0421CBF23F45B
:10B3280040739BB203800F4B8185984202850FD0F2
:10B3380003F5006398420BD003F54063984207D0A9
:10B3480003F58063984203D003F58063984201D1E6
:10B35800002303860123838210BD00BF40420F00F3
:10B3680050000020002C01400010004073B5054635
:10B378000068FFF7A7FF2A680124138800269BB2FC
:10B3880043F001031380EB7A01A88DF804308DF89F
:10B3980005408DF806608DF8074006F0A9FEEB7AA7
:10B3A8001B2B0BD1192301A88DF804308DF805400B
:10B3B8008DF806608DF8074006F09AFE02B070BD61
:10B3C8000C4B800A98420CD004D8B0F5801F0CD1E1
:10B3D80001207047084B984205D04933984206D05F
:10B3E80003E00220704703207047FE2070470020CA
:10B3F800704700BF01001000020010002DE9F8435B
:10B4080004680746204688469146FFF7D9FF032877
:10B418004BD8BA7A9108B8F1000F06D1A589AEB217
:10B4280002258D4026EA0505A5810A2303FB0013A2
:10B438001F4A42F82380043342F82390B8F1000FE2
:10B4480007D0BD7AA189AD080223AB400B439BB25C
:10B45800A3812823434303F120011144EFF312860B
:10B46800502585F3128803F10C051C331544134449
:10B4780055F8047F17B10F60296804319D42F7D150
:10B4880000230B60F3B283F31188282303FB002009
:10B49800036A23B1A3899BB243F0010304E0A389A3
:10B4A80023F001031B041B0CA381BDE8F88300BF34
:10B4B800B02A0020FFF776BAFFF774BAFFF772BA1E
:10B4C800014801F0E7B800BFC01C0020014801F0A6
:10B4D800E1B800BF141D00200C4B4FF400525A6015
:10B4E8004FF6FE730A48D0F8082211680B40136023
:10B4F800D0F8F821D0F8FC319A4203D000F5EA7070
:10B5080001F0FAB8012380F81832704700000240B1
:10B51800401B002037B5044603211E2006226B4637
:10B52800F9F79AFF78BB9DF801309DF80000174D98
:10B5380043EA002000B207F01FFD296807F070FDFC
:10B5480007F034FF9DF8033020809DF8020043EA9D
:10B55800002000B207F010FDA96807F061FD07F0B0
:10B5680025FF9DF80530A0809DF8040043EA0020DF
:10B5780000B207F001FD696807F052FD07F016FFF9
:10B588006080012000E0002003B030BD20000020D2
:10B598001FB5044602210C2001220DF10703F9F71B
:10B5A8005BFF08B900203BE09DF80730DB07F9D5C1
:10B5B8000321062202AB0C20F9F74EFF0C200921CB
:10B5C80001220DF10703F9F747FF0028EAD09DF89B
:10B5D800073013F00C0FE5D19DF809209DF80830CD
:10B5E8000C2043EA0223C3EB83339B009DF80B2016
:10B5F80023809DF80A300A2143EA0223C3EB8333F0
:10B608009B009DF80D2063809DF80C3043EA0223CF
:10B61800C3EB83339B00A3800122FAF70DF90120C5
:10B6280004B010BD07B50A2100220C20FAF704F96E
:10B638001420FCF74EFD0A210F220C20FAF7FCF823
:10B648000A20FCF746FD01AB102103220C20F9F774
:10B6580003FF0A20FCF73DFD0A2100220C20FAF71F
:10B66800EBF80A20FCF735FD0DF103030221012256
:10B678000C20F9F7F1FE0DF10303092101220C203A
:10B68800F9F7EAFE0A2101220C20FAF7D5F803B0EF
:10B698005DF804FB2DE9FF41604B1B689BB11A68FC
:10B6A8001AB15F49886902438A619A889868ADF837
:10B6B800042002228DF8072004220DEB02018DF8E8
:10B6C800062001F0B9FB3220FCF703FD002111220E
:10B6D8001E20FAF7B1F8012160221E20FAF7ACF813
:10B6E8006420FCF7F6FC002402A8FFF713FF2746A6
:10B6F80026460A25022101221E20FAF79DF832204B
:10B70800FCF7E7FC02A8FFF705FFBDF90820BDF923
:10B718000A1014448A42A8BF0A46BDF90C300F44E7
:10B7280093421E44A8BF134613F5805F09DD3D4AC6
:10B73800013DD36883F01003D360DBD14FF00108DB
:10B7480001E04FF000081E2000211222FAF774F8D9
:10B758000A25022101221E20FAF76EF83220FCF792
:10B76800B8FC02A8FFF7D6FEBDF90820BDF90A10FB
:10B77800A41A8A42A8BF0A46BDF90C307F1A934220
:10B78800A6EB0306A8BF134613F5805F07DD254A1D
:10B79800013DD36883F01003D360DAD101E04FF0A4
:10B7A8000008204607F0E8FB01461F4807F0ECFCBC
:10B7B8001E4D20F000402860384607F0DDFB0146AA
:10B7C800194807F0E1FC20F000406860304607F0B7
:10B7D800D3FB0146164807F0D7FC20F00040A860CC
:10B7E800002170221E20FAF727F8012120221E20AE
:10B7F800FAF722F81E2002210022FAF71DF8642029
:10B80800FCF767FCB8F1000F04D14FF07E532B60B2
:10B818006B60AB6004B0BDE8F08100BFA4020020FB
:10B8280000100240000C014000406F46200000203C
:10B8380001C05E46024640213C20F9F7FDBF0246A2
:10B8480080213C20F9F7F8BF012828BF01202DE905
:10B85800F04F0646142000FB06F3704F89B0F91824
:10B86800FC586F4B0A691C601E716E4BB1F808805A
:10B87800DD69B1F80AA02A43DA61A2884D6822F48A
:10B8880040721204120C4AEA0809A28003A9C5F8FA
:10B89800109002228DF80E0028460193ADF80C9006
:10B8A8008DF80F2001F0C8FA019B00971F464FF052
:10B8B800080BAA6818EA020F03D10A20FCF7FEFB5E
:10B8C800F7E70A20C5F81480FCF7F8FBC5F81080E4
:10B8D8000A20FCF7F3FBBBF1010BEAD1C5F814A071
:10B8E8000A20FCF7EBFBC5F814800A20FCF7E6FBFE
:10B8F800C5F810800A20FCF7E1FB0222C5F810A069
:10B90800284603A98DF80F201C228DF80E20ADF8CB
:10B918000C9001F091FA444A03A894423A690BBF8B
:10B9280042F4001242F480023A613A610BBF3A696C
:10B938003A6922F4001222F480023A61A38823F4BF
:10B9480040731B041B0CA38023889BB243F00103A4
:10B958002380A58803F08EFC0599344B25F03F051C
:10B96800B1FBF3F32D042D0C1D43ADB2A580228845
:10B97800002522F001021204120C22802C4A03A88E
:10B98800B1FBF2F100298AB208BF012242F400415A
:10B998004FF4967253434FF47A7293FBF2F30133E8
:10B9A8009BB22384A1832388009A9BB243F00103AE
:10B9B8002380238823F4816323F002031B041B0CD8
:10B9C80023804FF480432381142303FB0626737BD3
:10B9D80001248DF80C308DF80D508DF80E508DF82F
:10B9E8000F4006F085FB337B9DF80F208DF80C3057
:10B9F8008DF80D508DF80E501AB103A806F078FB9B
:10BA080008E05A0903F01F039C4002F12003094A89
:10BA180042F8234009B0BDE8F08F00BFF09D01084F
:10BA2800681D0020001002400054004040420F00F2
:10BA3800804F120000E100E0914B70B51A68908ABF
:10BA480080B2C1B2CE072ED5118821F40061090455
:10BA5800090C1180118889B241F48061118000219C
:10BA68005971997999B1D97911B9197AFF290ED1F2
:10BA78000121D971597A022901BF118889B241F48B
:10BA880000611180997A41F001011182E2E0997A0E
:10BA980001F0FE0111821A7AFF2A00F0DB80784A51
:10BAA800FF215171D6E08D073AD5BFF35F8F587AE1
:10BAB800C0B2012813D1997989B1D97979B111889E
:10BAC80021F480610904090C1180BFF35F8F118B89
:10BAD8001188D87289B241F4007111801BE0118B72
:10BAE800BFF35F8F587A664902280AD1887940B136
:10BAF800C97931B1118821F480610904090C1180D8
:10BB0800A2E0587A5E49032805D1887918B1C97925
:10BB1800002940F09980918889B241F4806198E0C9
:10BB28004C0757D50121D9729979002938D0D9798C
:10BB3800002935D0597A1088022959791ED920F45C
:10BB480080600004000C1080148ADD68C8B2E4B27A
:10BB580049B26C541188DC6889B241F400711180D3
:10BB68001968821C5A710A8A0130D2B240B2225432
:10BB78008A8892B242F480628A8026E080B240F4D9
:10BB880000701080148ADD68C8B2E4B249B26C54FF
:10BB9800128A411C49B2D2B203306A54587114E077
:10BBA800D979374809B9017C41B1118889B241F482
:10BBB800007111805A7901325A7106E0118889B2F0
:10BBC80041F4807111800122C27119680A88D20576
:10BBD800FCD43FE001F0400101F0FF04E1B15879E5
:10BBE800168ADD68C4B2611C40B2F6B22E54C9B2DE
:10BBF8005D7A597149B2C81C854201BF908820F40A
:10BC080080600004000C08BF90805A7A8A4221D1D3
:10BC18001B4A023454711DE006061BD5597948B2F7
:10BC2800451C0AD05C690131205CC9B21082587A7F
:10BC3800597149B288420DD106E0197A5C711182B6
:10BC4800997909B9597A29B9918821F48061090447
:10BC5800090C9180597A93F9050001318842084A04
:10BC68000CD10021D171D17A31B111688A8822F4BE
:10BC780040721204120C8A8000221A7670BD00BF2E
:10BC8800681D002010B5204C2368998A89B211F4E8
:10BC9800706F1CBF0122627611F4E06F2AD01A8BF4
:10BCA8009A88890522F480624FEA02424FEA1242DA
:10BCB8009A801FD41A8892051CD41A88D0050ED5EC
:10BCC8001A88D105FCD41A8892B242F400721A80FC
:10BCD8001A889205FCD42079FFF7B6FD0AE01A8885
:10BCE80092B242F400721A809A8822F440721204C6
:10BCF800120C9A802268938A23F470631B041B0C2D
:10BD080093820023237610BD681D002008B50848DB
:10BD18000AF087FFC0B209280246054B04DC01304F
:10BD28002021C0B29954F6E700221A5408BD00BF7A
:10BD38001927002008B507480AF073FFC0B2142875
:10BD4800044B04D8421C20211954D0B2F7E7002232
:10BD58001A5408BD192700202DE9F74FFCF792F96E
:10BD6800A64C804626686568A768861BF643451B6F
:10BD7800C71BED43FF43F60FED0FFF0F2EB93FB979
:10BD8800002D00F08782B9462CE04FF0000929E029
:10BD9800B14627E003EB8A0BBBF802301A050ED434
:10BDA80013F4805F1DBF964A9BF801101268954AEC
:10BDB800954B14BF52F82120126843F82A20BBF88B
:10BDC8000230D80516D499050AD5904B1B7813F084
:10BDD800040F0CBF8E4A8F4A8B4B126843F82A20F7
:10BDE80009F10109207B5FFA89FA8B4982450B68C2
:10BDF800D0D326E0894A5046594604F0FBFB884BCD
:10BE08001B885A0603D550465946864A16E05807F5
:10BE180003D550465946844A10E0190703D55046C1
:10BE28005946824A0AE09A0703D550465946804A3D
:10BE380004E0DB07D4D5504659467E4A04F0DAFBC5
:10BE4800CEE7DFF808E20093BEF906307822A3F5C2
:10BE58007A7353434FF47A7293FBF2F3F34603F287
:10BE68002B13019300225FFA82FE864517D2009BAE
:10BE780003EB820EBEF802E01EF4806F0DD040F294
:10BE8800671ADFF88491019B39F822E09E449EFBF3
:10BE9800FAFC0AFB1CEE29F822E00132E3E74DB375
:10BEA80008F5C333A0336360637B544A13BB9373B1
:10BEB800614B1B6813F0020F0AD0DFF894E19EF87B
:10BEC80000E0BEF1000F03D04FF0010E82F80EE043
:10BED800DA0506D5594BDB781BB1A37B43F0020387
:10BEE800A3734A4B1B7813F0050F02BFA37B43F0E3
:10BEF8000403A37394F80EE0BEF1000F03D13F4B87
:10BF08005B7B002B4FD094F80DC01CF0010FACF1F7
:10BF18000C031DD1BCF1030F07D8DFF8E8901EF021
:10BF2800040F3B4A08BF4A4600E0364AACF1040C0D
:10BF3800BCF1070F05D8DFF81CC11EF0010F18BFB0
:10BF48006246DBB2032B0ED81EF0020F3C4B06E014
:10BF5800DBB2032B06D82F4B2A4A1EF0020F18BF5C
:10BF68001A4600E0274A4FF0000C5FFA8CF3834230
:10BF78000DD20B6803EB8C035B881B0642BFD2F81B
:10BF88000090214B43F82C900CF1010CEDE785B1A2
:10BF9800BEF1000F08D0637B184A0133DBB2142BC3
:10BFA80006D1002304E025B1637B002BF3D100E028
:10BFB8005373002E52D0234A3223B2F90250B2F9F9
:10BFC8000020002DB8BF6D42002AB8BF524295FB31
:10BFD800F3F592FBF3F2EDB2D3B2AB4238BF2B4686
:10BFE800194A13B192FBF3F300E01346434423606C
:10BFF800E37B024A83BB01232FE000BF841D00209E
:10C00800141B0020FCB40108720E0020E730002049
:10C0180004B40108F4B30108181B0020189E010895
:10C028008C1A00201E9E0108249E01082A9E0108E1
:10C03800309E0108369E0108FC2C00209430002018
:10C048000CB40108CC110020400D0300382D00204D
:10C05800141A002014B401080023D3738F4D904B99
:10C068002D78E27BADB9002F00F00F818D4B267B38
:10C078001A788D4B02F0040293F800C08B4BD2B2B1
:10C08800D3F800E00B680021894D03EB86060F46C4
:10C09800B5E01AB9874A1A61002508E0864AFAE726
:10C0A8000A68AB00D6187688760604D40135EBB258
:10C0B8008342F5D3D7E7814EB6F90060192E25DD06
:10C0C80012F803E094F814C00EF00F09E145266950
:10C0D8000CDCDFF8CCC19CF815C0BCEB1E1FDEBF22
:10C0E800D6F800C0DFF8D8E143F80EC012F803E034
:10C0F80094F816C00EF00F09E14533DBDFF8A0C154
:10C108009CF815C0BCEB1E1F2CDC26E0193629DA7A
:10C1180012F803E094F814C00EF00F09E1452669FF
:10C128000CDCDFF87CC19CF817C0BCEB1E1FA2BF5B
:10C13800D6F800C0DFF888E143F80EC012F803E033
:10C1480094F816C00EF00F09E1450BDBDFF850C17B
:10C158009CF817C0BCEB1E1F04DBD6F800E0584E55
:10C1680043F806E0554EB6F90260192E1BDD12F8A9
:10C1780003C094F814E00CF00F09F14526690CDCB3
:10C18800DFF81C9199F81590B9EB1C1FDEBFD6F8A3
:10C198000090DFF82CC143F80C90D25C02F00F0C31
:10C1A800F4451EDD82E7193680DA12F803C094F8E8
:10C1B80016E00CF00F09F14526690CDBDFF8E0907A
:10C1C80099F81590B9EB1C1FDEBFD6F80090DFF880
:10C1D800F0C043F80C90D25C02F00F0CF445FFF667
:10C1E80065AF94F817E0BEEB121FA2BF3668344A59
:10C1F8009E505BE75888000504D404330435B342E5
:10C20800F8D122E04AB101EB0C0A06209AFBF0F9BA
:10C2180000FB19A001280DDC01E057B9012793F8AC
:10C2280001900EEB89003EF829A090F80290C078A2
:10C2380003E01746002081468246013125F802AC0A
:10C2480085F800906870C9B2D7E7174A1378013BA0
:10C2580013F0FF0308BF06231370124B1B785B070C
:10C2680041BFBBF906304FF47A72A3F57A7303EB3A
:10C27800C30348BF93FBF2F3124A46BF0133DBB254
:10C28800012392FBF3F34344A36003B0BDE8F04FEE
:10C2980000F0F4BC03B0BDE8F08F00BF230F00200E
:10C2A800841D0020E73000202C000020141B0020F3
:10C2B800740E002010B40108FCB40108CC11002051
:10C2C800720E0020400D0300026B0346C16810B5D2
:10C2D800406942B11A6C8C1A013A08BF0A46005DDF
:10C2E8001A64C0B210BD1A6A805C01328A4228BF43
:10C2F8000022C0B21A6210BD436B13B190F844001B
:10C308007047836A406A1B1A584258417047036B4A
:10C3180013B15B68016C01E0C369016A8B423CBFE1
:10C32800C2689B18581AC0B27047426A806A131ACA
:10C338005842584170474171704743799B070AD565
:10C34800436A8269D154436A01690133B3FBF1F24C
:10C3580001FB123343627047437913F001031FBF97
:10C36800C36803F1FF32C369006A1DBF181A104081
:10C37800C0B218467047437910B513F0010304465C
:10C388000DD0FFF7E9FF58B1236A6269E168D05C14
:10C398000133B3FBF1F201FB1233236210BD1846DF
:10C3A80010BDF0B5046D8279A389467923F4005352
:10C3B80012F0020F4FEA03434FEA13430CBF002168
:10C3C8004FF4005112F0040FA38114BF4FF4806E94
:10C3D8004FF0000E16F0010F8768054614BF0420C1
:10C3E8000020B307238A48BF40F008029BB223F419
:10C3F800405343EA01032382A18948BF90B289B21E
:10C4080021F4B05121F00C014EEA010140EA010289
:10C41800A281A38A87B023F440731B041B0CA38258
:10C4280001A802F027FF039B049E264A944218BFE6
:10C438001E46A389192272431BB2002BB4BF7E008B
:10C44800BE00B2FBF6F66427B6FBF7F0000101095F
:10C4580007FB1163A28912B2002AB7BFD9001A01DB
:10C468003231B1FBF7F2A7BF3232B2FBF7F302F079
:10C4780007021043A8BF03F00F03AA79A8BF184307
:10C4880080B212F0010F20812B6D06D00E498B422D
:10C4980002BF042001F54841086112F0080F9A8A8A
:10C4A8000BBF22F0080292B2120442F0080208BF41
:10C4B800120C9A829A8992B242F400529A8107B079
:10C4C800F0BD00BF0038014000440040417168E7FA
:10C4D800816066E703460A4690F84602D96A9B7966
:10C4E80000F0DCBC38B5A0F513746379A579DB07D7
:10C4F80046D594F8383205F00105F3B1226B10687F
:10C50800838DC3F34E03838494F83C3223B1B4F88B
:10C5180042320133A4F84232917A6A0000F01DFBDE
:10C52800012384F83B32002384F8393284F83A3204
:10C5380084F83832A4F8403238BD94F83B322046AB
:10C54800012B04BF94F8393284F83A3200F0F0FA3B
:10C5580094F83B22236B3AB9012284F83B221868ED
:10C56800997A05FA02F207E0002284F83B22954204
:10C578001868997A08BF0222BDE8384000F0EDBA81
:10C5880038BD10B5A0F5127494F83C22BAB9A36A64
:10C59800616A994228D0591CA069A162C35C2069CC
:10C5A800DBB25B0043F400738142A4F83E324FF0E3
:10C5B8000A0384F83D3228BFA262012312E094F9ED
:10C5C8003D327BB1B4F83E1220464B08A4F83E3207
:10C5D80001F0010100F0D4FA94F83D32013B84F8EF
:10C5E8003D3201E084F83C3294F83832002B50D1C7
:10C5F80094F839320133DBB2092B84F8393204D18B
:10C608002046BDE8104000F093BA0A2B41D194F8B7
:10C618003B322BB9B4F8403243F00103A4F840325E
:10C628006379D9071CD5B4F84002820501D4C30741
:10C6380005D4B4F844320133A4F8443210E0E36A74
:10C64800C0F347000BB198470AE0E3696269D05428
:10C65800E369E1680133B3FBF1F201FB1233E361F3
:10C66800012284F8382294F83B220023012A84F816
:10C6780039320ED1A27984F83B32236B12F0010FC4
:10C688001868997A0CBF02220022BDE8104000F019
:10C6980064BA10BD026D70B515880446ADB2A9061E
:10C6A80013D5036B8BB9C36A1BB1908880B29847C6
:10C6B8000BE0E169928840694E1CD2B2E6614254AF
:10C6C800E169E268914228BFE3612B0613D5636AEA
:10C6D800A26A9A42236D0AD0511CA069A162825CA9
:10C6E8009A802369994206D30023A36270BDDA6851
:10C6F80022F08002DA6070BD836A8169426B194456
:10C70800D160416A994297BF0169CB1ACB1A53602D
:10C7180096BF0023536083624FF0000380F84430D3
:10C72800136888BF816243F0010313607047436A4E
:10C738008269D154436A02690133934228BF0023B6
:10C748004362436B1BB11B68DB0705D4D4E7026D5A
:10C75800D36843F08003D36070472DE9F0431E4649
:10C76800944B8DB09842894690469DF8507051D1AF
:10C77800914B924A92491A60924AC3F808805A61CA
:10C7880002F580729A614FF48072DA601A618E4AFB
:10C7980018651A63A2F54842543ADA649A645963F0
:10C7A8008A4B9A6942F480429A615A6942F00102BE
:10C7B8005A6102238DF803303A074FF40073ADF83D
:10C7C800003001D51C230FE0B30706D51823804895
:10C7D80069468DF8023000F02FFBF5070AD54FF4B3
:10C7E8008063ADF800304823794869468DF80230F7
:10C7F80000F022FB0E238DF804300022012301A84B
:10C808008DF805308DF806208DF807306A4C05F054
:10C818006FFC4EE06F4B984240F0C7806E4B674A02
:10C82800C3F808801A604FF48072DA601A616B4AA4
:10C8380018655A6102F580729A61694A3C079A64E0
:10C84800DA64624BDA6942F40032DA615A6942F01A
:10C8580001025A614FF002038DF803304FF00403D0
:10C86800ADF8003001D51C230EE0B00706D518231B
:10C87800574869468DF8023000F0DEFAF10709D50D
:10C888000823ADF800304823514869468DF8023036
:10C8980000F0D2FA26238DF804300022012301A8E3
:10C8A8008DF805308DF806208DF8073005F020FC4E
:10C8B800494C0025012384F844302562E561A562CE
:10C8C8006562C4F82C906671C4F80880A771204688
:10C8D800FFF767FDF20731D5206B002826D0E36CFF
:10C8E800039501934FF480530A9380230693E368DA
:10C8F8000595049320230993636907950293089586
:10C908000B9502F03FFC01A9206B02F01DFC226B85
:10C91800216D136843F0010313608B8A9BB243F0C7
:10C9280040038B8253689BB2236407E04FF6DF72A3
:10C93800236D1A80DA6842F02002DA60B3072CD53A
:10C94800606B28B3A36C002501934FF480530A93BE
:10C958008023069323690295049310230393059576
:10C968000795089509950B9502F00CFC606B01A9D9
:10C9780002F0EAFB636B1A6842F002021A60226D49
:10C988005D605D60938A9BB243F08003938204E00C
:10C99800226DD36843F08003D360226D20469389CB
:10C9A8009BB243F40053938100E000200DB0BDE832
:10C9B800F08300BF00380140141D00203C9E010890
:10C9C800440002409C1D0020580002400010024014
:10C9D8000008014000440040C01C00209C1F0020AB
:10C9E8000444004010F80A3C0133DBB20A2B84BF30
:10C9F80010F8131C044A00F80A3C82BF002322F8EE
:10CA0800113000F80A3C7047E02F0020334A70B517
:10CA1800136C9068194440F68C23081A9842916068
:10CA2800D060516013463BD9127893F945101046EF
:10CA38008A420BD1111F082908D893F846101829E3
:10CA480001D8013103E083F8442002E0002183F893
:10CA5800461093F944402149A24219D191F8474020
:10CA6800B4B10C310024944206DA51F8046F1C4D1D
:10CA780025F814600134F6E70C2805D0184900247D
:10CA880021F810400130F7E71648017801310170AC
:10CA980083F84520002201211A7083F8471070BDE1
:10CAA80092F84710C9B140F2DA51A0F2EF248C4253
:10CAB80008D811780B2905D80B1D0131117042F8DF
:10CAC800230070BD002283F84720074B03F1300292
:10CAD800002143F8041F9342FAD170BDF4000020EE
:10CAE800E02F00201C06002000010020024A136CE1
:10CAF8000133194411647047F4000020024B53F8C5
:10CB080020301B6819807047802A0020074BA1F548
:10CB18007A7153F820301A681B8959434FF47A7395
:10CB280091FBF3F189B21180704700BF802A002081
:10CB380090F83B3210B57BB990F83A3290F8394208
:10CB4800A34209D2B0F8401201229A400A430133A5
:10CB5800A0F84022DBB2F3E710BD1FB50123ADF802
:10CB68000830ADF80410002301A9ADF80A30ADF87B
:10CB78000C30ADF8062002F0DEFB05B05DF804FBD2
:10CB88008379DB0748BFB1FA81F1D0F8343148BF67
:10CB980049095A681B8909B1136170475361704785
:10CBA8001FB50123ADF808300023ADF80C30ADF8FF
:10CBB8000A30094BADF804101B7801A9012B08BFF6
:10CBC8000323ADF8062008BFADF80C3002F0B3FB24
:10CBD80005B05DF804FB00BFF000002038B510F880
:10CBE8000E2C044650F8043C52B9012200F80E2CD1
:10CBF80020F80C1C997A18680222BDE83840CFE763
:10CC080030F80C2C20F80A1C891A89B220F8081C64
:10CC1800074A10F80F0C002522F8101004F80E5CD3
:10CC28001868997A2A46FFF7BBFF04F8065C38BDF6
:10CC3800E02F0020044B53F820301BB107289CBF7D
:10CC48001B681980704700BF1C020020084A13683F
:10CC58009B020BD5074B002119704FF6FE7306494E
:10CC6800086803400B604FF400135360704700BF1F
:10CC780000000240E63000206C0002402DE9F04739
:10CC8800664D2B686649581C0A788E4602F0FF06E6
:10CC98000AB10346F6E737462B60687BAB6895F820
:10CCA8000C80AA7B39B2202900F09C80DFF880C173
:10CCB8000CEB8103DC789B783CF82110C3F1FF036F
:10CCC8009BB2002B65D04FF03C0CB1FBFCF9C3F1D3
:10CCD800FF0363431B12B9F1050F5DD8DFE809F0C4
:10CCE800030B1A293A4AE01A4143B1FBFCF0DAB2C5
:10CCF8001044C0B251E0B1FBFCF00CFB101189B23A
:10CD0800DAB2C1F13C01E31A4B43B3FBFCFC204609
:10CD180094442CE0B1FBFCF00CFB1011E21A89B230
:10CD28004A43B2FBFCF25FFA83F84244D2B220468F
:10CD380032E0B1FBFCF90CFB191189B2E01AC1F120
:10CD48003C014843B0FBFCF05FFA83F84044C0B2B2
:10CD5800224621E0B1FBFCF80CFB1811D8B289B2CD
:10CD6800E31A01FB03F2B2FBFCFC224684445FFA9F
:10CD78008CF412E0B1FBFCF80CFB181189B2D8B2A4
:10CD8800C1F13C01E31A4B43B3FBFCF20244D2B2BB
:10CD980003E02246204600E044464FEA042C4CEAD1
:10CDA800004C4CEA020C17234FF0010808FA03F86C
:10CDB80006F1170118EA0C0FA1EB0301DFF87480E4
:10CDC80014BF4FF011094FF0090989B213F1FF336D
:10CDD80008F80190E8D218360137B6B2BFB2114B45
:10CDE800A0465FE7AB6001238EF8003040F22A339B
:10CDF800AA730D4AE9800D4985F80C806873AE80E6
:10CE0800536000238B840B889BB243F001030B8093
:10CE1800136843F001031360BDE8F0879C210020EC
:10CE2800E6300020A82100206C00024000040040E9
:10CE3800720E0020C5020020F0B5B1F800E0002312
:10CE48004EFA03F2D50725D58E784FEAD30CF406AF
:10CE580048BFCC7806F00F0203F0070748BF22430B
:10CE6800BF0050F82C500F24BC4025EA0404BA40F7
:10CE78002243282E40F82C2005D1C46801229A406C
:10CE880024EA020205E0482E04D1C46801229A402F
:10CE98002243C2600133102BD2D1F0BD2DE9F04FEF
:10CEA8001E464FF414734343554D85B005F11004E5
:10CEB80080469146E718A24610B92B44514A03E030
:10CEC800012805D1504A2B441A641032C3F8442172
:10CED8004FF4147303FB08F34C48EC180AEB0302F5
:10CEE80003F59C73343253442061E1636262A362A8
:10CEF80000224FF480714FF0010BD4F84431032025
:10CF0800E1612263E2622162A263626384F84C22D7
:10CF180084F848B284F84922A4F85222A4F854228A
:10CF2800C4F818906075A67584F8568258681B89ED
:10CF380004F5A0724FF0020CADF80C3003A91023D1
:10CF480001928DF80E308DF80FC0CDF800C0FFF7B4
:10CF580073FF236CDDF800C0597B58681B898DF876
:10CF68000E1003A9ADF80C308DF80FC0FFF764FF61
:10CF780059463846FFF704FE3220FBF7AAF8244B3F
:10CF8800019A1B68D2F804B01A46B2FBF9F1B1F560
:10CF9800803F03D3012AF8D95208F6E71D4A4FF417
:10CFA8001474B3FBF2F204FB08F8584689B2D2B203
:10CFB800FEF7DCF905EB0809174B08F512780AEBC0
:10CFC80008040022C9F8583258462146FEF716FAD6
:10CFD800D9F8405016F0010F0CBF02220022286831
:10CFE800A97AFFF7BAFD0D4B2846C9F85C32211D16
:10CFF8000022FEF703FA384605B0BDE8F08F00BFFF
:10D008009C2100205CB401087CB40108549E0108EE
:10D018005000002040420F008BC50008EDC40008F6
:10D028002DE9F7438E460546DFF8A092114699F898
:10D03800B0440068164698467246631C89F8B034B6
:10D04800FEF740F92B8901A9ADF8043018238DF8B3
:10D058000630686802238DF80730FFF7EDFEAB7ADB
:10D0680009F2B447240127442A6849460C2B00F2E8
:10D07800F680DFE813F00D00F400F400F40051002E
:10D08800F400F400F4008A00F400F400F400C20094
:10D09800138CDFF83CC223F001031B041B0C138420
:10D0A800138CB2F804E0108B624520F073004FEA4D
:10D0B80000404FEA10409BB21FFA8EFE40F070000D
:10D0C80014D00CF5006C624510D00CF5406C62452C
:10D0D8000CD00CF5806C624508D00CF5806C62456C
:10D0E80004D023F0020343F0030307E023F00E0308
:10D0F8002EF4407E43F003034EF4807EA2F804E051
:10D108001083A2F834801384138B23F008031B04C4
:10D118001B0C43F0080336E0138CDFF8B4C123F08E
:10D1280010031B041B0C1384138CB2F804E0108B3F
:10D13800624520F4E6404FEA00404FEA10409BB2B7
:10D148001FFA8EFE40F4E04008D00CF5006C6245F2
:10D1580004D023F0200343F0300307E023F0E0037A
:10D168002EF4406E43F030034EF4806EA2F804E0D3
:10D178001083A2F838801384138B23F400631B04F4
:10D188001B0C43F40063138369E0138CDFF840C180
:10D1980023F480731B041B0C1384138CB2F804E073
:10D1A800908B624520F073004FEA00404FEA104030
:10D1B8009BB21FFA8EFE40F0700008D00CF5006C90
:10D1C800624504D023F4007343F4407307E023F46A
:10D1D80060632EF4405E43F440734EF4805EA2F820
:10D1E80004E09083A2F83C801384938B23F0080317
:10D1F8001B041B0C43F0080330E0138CDFF8D0C08D
:10D2080023F480531B041B0C1384108CB2F804E025
:10D21800938B20F4005023F4E6431B0400041B0CFA
:10D22800000C62451FFA8EFE43F4E04340F4405080
:10D2380003D00CF5006C624503D12EF4804E4EF4F9
:10D24800804EA2F804E09383A2F840801084938B68
:10D2580023F400631B041B0C43F4006393832B7BB0
:10D2680043B1B2F844306FEA43436FEA53439BB289
:10D27800A2F8443013889BB243F001031380AB7AC1
:10D288000C2B19D8DFE803F0071818180B18181812
:10D298000F18181813000B1902F134000AE00B19C3
:10D2A80002F1380006E00B1902F13C0002E00B190C
:10D2B80002F14000C3F8B40438460C44A4F8BC6436
:10D2C800C4F8B82403B0BDE8F08300BF9C21002057
:10D2D800002C014010B5D420FEF7B1FA8020FEF7EB
:10D2E800AEFAA820FEF7ABFA3F20FEF7A8FAD32043
:10D2F800FEF7A5FA0020FEF7A2FA4020FEF79FFAF3
:10D308008D20FEF79CFA1420FEF799FAA120FEF76B
:10D3180096FAC820FEF793FADA20FEF790FA122060
:10D32800FEF78DFA8120FEF78AFACF20FEF787FAFA
:10D33800D920FEF784FAF120FEF781FADB20FEF708
:10D348007EFA4020FEF77BFAA420FEF778FAA620A2
:10D35800FEF775FAAF20FEF772FAA620FEF76FFA0D
:10D36800AE20FEF76CFA2020FEF769FA0020FEF7DF
:10D3780066FAB020FEF763FA4020FEF760FA002054
:10D38800FEF75DFA1020FEF75AFA4FF48064013C6C
:10D398000020A4B2FEF74EFA002CF8D18120FEF747
:10D3A8004EFAC820FEF74BFAAF20FEF748FA0120E4
:10D3B80010BD70B500EB8000094CA0F1A1059C38A8
:10D3C80025440444074B15F8010F1E787040FEF7FA
:10D3D80031FAA542F6D13046BDE87040FEF72ABAC8
:10D3E8006C9E0108E930002010B5441E14F8010FA6
:10D3F80010B1FFF7DEFFF9E710BD08B55038C0B22D
:10D40800FEF71DFA0020FEF71AFABDE808401020C2
:10D41800FEF715BA10B504465039C8B2FEF70FFA30
:10D4280004EB4400400000F00E00FEF708FA062066
:10D438006043BDE81040C0F303101030FEF7FFB999
:10D448000028114AB8BF404290FBF2F330B50F4CA8
:10D458003C2504FB030068430D4D90FBF2F22D6858
:10D468002D7B25B903EB830303EB830301E0C3EBB7
:10D47800031302EB830304FB02020B804FF47A735D
:10D4880092FBF3F24A8030BD80969800806967FF6E
:10D49800B8190020022803D0431E5842584170474B
:10D4A800064B1B681B7823B1054B1868C0F3C040B6
:10D4B8007047044B1878C0F380007047F0050020CF
:10D4C800E8100020E730002010B50A4C5E2801461D
:10D4D800206805D15D2102F0FCFD20683E2105E0B1
:10D4E8005D2903D102F0F5FD20683D21BDE810401B
:10D4F80002F0EFBD1027002010B50446C0B2FFF7B8
:10D50800E3FFC4F30720BDE81040DDE7024B5E21CE
:10D51800186802F0DEBD00BF1027002038B50546A8
:10D52800054C5E21206802F0D4FD20682946BDE83C
:10D53800384002F0CEBD00BF1027002013B50446C6
:10D5480001A90068FFF77CFF1320FFF7E7FFBDF98B
:10D558000400FFF7D1FF1B20FFF7E0FFBDF906002D
:10D56800FFF7CAFF2320FFF7D9FF2368002BB4BFBA
:10D5780053204E20FFF7C0FF01A96068FFF760FF46
:10D588001220FFF7CBFFBDF90400FFF7B5FF1A2003
:10D59800FFF7C4FFBDF90600FFF7AEFF2220FFF733
:10D5A800BDFF6368002BB4BF57204520FFF7A4FFD9
:10D5B80002B010BD674B73B51878FFF76BFF664D67
:10D5C80004462B78834220D0C8B1644B1B68E3B172
:10D5D80093F9000002230093614B04211B68002289
:10D5E8005B78003318BF012301934FF41653FAF701
:10D5F800D0FD5C4B186040B101232B7005E0594EFB
:10D608003068FAF725FB34602C70574B574D187863
:10D61800FFF740FF2B780446834218D088B1544B5B
:10D628001B68A3B10022012493F9000008214FF4DC
:10D63800964300940192FAF7ACFD4E4B186028B956
:10D6480005E04C4E3068FAF703FB34602C704A4B07
:10D658004A4D1878FFF71EFF2B78044683422E4662
:10D6680043D0002838D0464B1A68002A3DD0D379D9
:10D6780092F90000002B4FF00202424C08BF02232F
:10D688000092002254F8233001921021FAF781FD0C
:10D698003D4B0546186040B33C4C94F84A30022B89
:10D6A8000BD094F89620022A01D14C3405E023B11E
:10D6B800002A04F14C0418BF0024354B1C6044B107
:10D6C800204600214C2209F068FA0223256084F8DC
:10D6D8004A300123337008E02B4E306803F078FE9F
:10D6E8003068FAF7B5FA34602C702A4B2A4D18784E
:10D6F800FFF7D0FE2B780446834229D000B3274B8E
:10D708001B682BB3264A93F900001268032352784A
:10D718002021002A0CBF08220922009301924FF40D
:10D7280061430022FAF735FD1E4B186080B11E4A8E
:10D73800012313702B701D4B1A681D4B1A6007E0EC
:10D74800184E3068FAF784FA174B34601C702C7046
:10D7580002B070BDF8050020AC110020F4050020CF
:10D76800B819002010270020F9050020D81900203A
:10D778005C1A00204C1A002004060020621A0020BF
:10D788000006002034A10108641A0020182800208F
:10D79800681A002010060020781A00200C060020C5
:10D7A800080600207C1A0020801A0020202D002066
:10D7B800841A0020642928BF6421F8B501FB00F50C
:10D7C800642495FBF4F40646E4B20027FBB2A342B6
:10D7D80004D29F20FFF7EDFD0137F7E7B4420BD2E3
:10D7E800142195FBF1F5C4EB8410663DC4EB800071
:10D7F8002844C0B2FFF7DDFD0134E4B2B44201D2DF
:10D808009A20F7E7F8BD2DE9F743FAF73BFC924C6D
:10D818006368C31A002BC0F2688300F5433303F52D
:10D82800A07363608D4B1D78237AC5F38005EB1ACE
:10D8380018BF012325724DB1002B00F05683884B89
:10D848005A789A7001225A701A702BE0844A2BB1C8
:10D85800D37843F00203D37093785370D67806F0E8
:10D86800020101F0FF0339B97D498968411A00298D
:10D8780003DB06F0010300E0012303F00107784908
:10D8880017707BB1F2070DD50A7905230132D2B2A0
:10D89800B2FBF3F303EB8303D31A724ADBB20B71C7
:10D8A800D35C4B706E4EDFF8088233787BB3F37825
:10D8B80023F00203F3706C4B0344AE20B360FDF712
:10D8C800BEFF08B1FFF706FD88F80000002800F049
:10D8D8000C83B020FDF7B3FF4020FDF7B0FF002018
:10D8E800FDF7ADFF1020FDF7AAFF4FF48067013F59
:10D8F8000020BFB2FDF79EFF002FF8D13846FFF792
:10D908007CFD7278594B53F82200FFF76DFD98F8AB
:10D918000030002B00F0E9827378062B00F2B28207
:10D92800DFE813F00700B002180078006A018701E9
:10D93800EC014F494F4A504B5048FCF782FB0120FD
:10D94800FFF75BFD4D48FFF74FFD0220FFF755FD40
:10D958004B48ACE14B4F3B689B0735D5DFF854810A
:10D968000A23B8F80010DFF85091B1FBF3F203FB7B
:10D97800121399F8001092B29BB200913F484249A5
:10D98800FCF75FFBFEF7D6F90120FFF736FD3B48B1
:10D99800FFF72AFD3D4B99F800201868B8F80030C9
:10D9A800067902FB163164234B43C17802208E1B93
:10D9B8005643B3FBF6F6F6B2FFF71FFD31461520C6
:10D9C800FFF7F8FE032600E001263B681F0540F13B
:10D9D80059822F4B2F491F68642397FBF3F209687C
:10D9E80003FB1273009125482B49FCF72AFBFEF72D
:10D9F800A1F93046FFF701FD2048FFF7F5FC01F0DB
:10DA0800DFFE0746701CFFF7F8FC15203946FFF7C4
:10DA1800D1FE37E20120214FFFF7EFFC2048FFF746
:10DA2800E3FC3B68980749D51E4A1448B2F902102E
:10DA3800B2F900300091B2F904201B4901921B4A47
:10DA4800FCF7FFFAFEF776F90220FFF7D6FC0B4841
:10DA5800FFF7CAFC032632E010270020E730002039
:10DA6800D41A002069C00108404B4C0010A10108DD
:10DA78006EC0010877C001087DB60108192700208B
:10DA88007EC00108FC2C00208CC00108B0190020C1
:10DA9800BC190020C0190020A4C00108C419002026
:10DAA800B9C00108B6110020CFC00108DEC00108C6
:10DAB8003D020020B41900204400002002263B68E3
:10DAC800D9071AD57B4A7C48B2F90210B2F900305E
:10DAD8000091B2F9042079490192794AFCF7B1FA28
:10DAE80006F10108FEF726F93046FFF786FC5FFAD3
:10DAF80088F87148FFF778FC46463B681A0718D53E
:10DB0800704A6D48B2F90210B2F900300091B2F9CA
:10DB180004206A4901926C4AFCF793FA771CFEF7D5
:10DB280009F93046FFF769FCFFB26348FFF75CFC70
:10DB38003E46664A6149B2F90030B2F902205E48B1
:10DB48000092634ADFF8B091B2F90020771C019285
:10DB5800604AFCF776FAFEF7EDF83046FFF74DFC21
:10DB68005548FFF741FC5449D9F80000FCF704F97F
:10DB7800514809F056F8FFB2C1B2092909D84B1C1F
:10DB8800DBB2214420224A720021E2189172194620
:10DB9800F3E7DFF82481D9F804004144FCF7ECF8F6
:10DBA800FEF7C8F83846FFF728FC4046FFF71CFC8C
:10DBB8004146D9F80800FCF7DFF8404609F031F88B
:10DBC8000236F6B2C7B2092F09D87B1CDBB227444C
:10DBD80020227A720021E21891721F46F3E73E4B29
:10DBE800B3F9000005F0C8F908EB0701FCF7C4F821
:10DBF800FEF7A0F8304657E00026384F3B78B3428E
:10DC080040F240810E2E00F03D8170080130FFF790
:10DC1800F4FB304604F0D8FC3B78B34206D9202008
:10DC2800FFF7C7FB701CC0B204F0CEFC0236F6B298
:10DC3800E3E72B4E2B4996F8B0271F48FCF701FA6B
:10DC48000120FFF7DAFB1C48FFF7CEFB264B2749DC
:10DC58001F7819483A46FCF7F4F90220FFF7CDFB84
:10DC68001548FFF7C1FB0C2303FB0766204996F80C
:10DC7800B32796F8B2371048FCF7E3F9FEF75AF8DD
:10DC88000320FFF7BAFB0C48FFF7AEFB96F8B8176E
:10DC980096F8B62796F8B737074800911549FCF764
:10DCA800D0F9FEF747F80420FFF7A7FB0248FFF773
:10DCB8009BFBE7E00811002019270020CFC00108CE
:10DCC800E2C001080E1100202DD00108F42C00201C
:10DCD800C4110020E6C001086C080020B428002008
:10DCE800D4110020EAC00108A82C0020F6C00108C1
:10DCF80007C1010818C10108600800207C4B1B6897
:10DD08001B0640F1BB80236A616A7A4A8B421CBFBA
:10DD1800536292F828304FF001011CBF013303F021
:10DD280003034FF0000018BF82F82830FFF772FB9A
:10DD380094F82830704A0026D05CFFF73AFB02209E
:10DD48000121FFF767FB6D4B3620F35C0136C3EB0F
:10DD5800C30393FBF0F0C0B2062828BF0620603842
:10DD6800C0B2FFF726FB102EEDD1654B65491B7835
:10DD7800654813F0020F654B1A7814BF59234E23D8
:10DD8800FCF75FF9FDF7D6FF0220FFF736FB5E4888
:10DD9800FFF72AFB5E495F4B4E680A685A4892FBB8
:10DDA800F3F25D4996FBF3F3FCF74BF9FDF7C2FF7D
:10DDB8000320FFF722FB5448FFF716FB574B58493F
:10DDC8001A885148FCF73DF9FDF7A0FF0420FFF73A
:10DDD80014FB4D48FFF708FB524B53491A884A4831
:10DDE800FCF72FF9FDF792FF04210A20FFF712FB39
:10DDF8004548FFF7F9FA4D49E26A4348FCF721F92B
:10DE08004B4EFDF783FF0520FFF7F7FA3E48FFF773
:10DE1800EBFA7268B36847493B48FCF712F9FDF71B
:10DE280075FF05210A20FFF7F5FA3748FFF7DCFAF6
:10DE38003369F2684049D21A3348FCF702F9FDF712
:10DE480065FF0620FFF7D9FA2F48FFF7CDFAB26829
:10DE58003A492D48FCF7F5F8FDF758FF06210A2046
:10DE6800FFF7D8FA2848FFF7BFFA354915222648A0
:10DE780008F002FFFDF74AFF072015E7F37843F0A3
:10DE88000203F370002D30D12E4B002193F820307F
:10DE98001220052B97BF2C4A3F259B181D7FFFF7A3
:10DEA800B9FA2846FFF785FA13200021FFF7B2FADE
:10DEB800264B1B78002B264B18BF72201B7808BFF7
:10DEC8002120002B18BF5220FFF773FA14200021DD
:10DED800FFF7A0FA94F83050074B585D013505F06C
:10DEE8000305FFF766FA84F8305003B0BDE8F08305
:10DEF800FC2C0020102700202AC1010899110020BD
:10DF0800C81900202FC1010819270020CE190020A8
:10DF1800D01900208096980040C10108CA19002035
:10DF28004DC101085011002055C101085CC101080C
:10DF38009C07002063C101086CC1010873C1010876
:10DF4800B00200209430002010A10108230F002007
:10DF5800880F0020064B1B7803F0040303F0FF0032
:10DF68001BB1044B1888C0F3C01000F001007047C3
:10DF7800E73000208C1A00202DE9F04F89B0059376
:10DF8800BE4B0026B3F90290B3F90030B9F1000F87
:10DF9800B8BFC9F10009002BB8BF5B429945B8BFAB
:10DFA80099468046B2463446B9F5FA7F0491039201
:10DFB800A8BF4FF4FA79019000960296B04D2B88CD
:10DFC800990754D0AD4B610033F91420AD4B33F9A8
:10DFD800143003EB4202039B5B429A4203DB039B30
:10DFE8009342A8BF1346A84A8F5E059ADB1B32F9F5
:10DFF80014001F18FFF7AEFF90B1A44B384613F872
:10E0080004A004F0B9FFA24905F0BEF80146504645
:10E0180004F0E2F89E4905F003F805F0C7F9074651
:10E0280098F8083064227B4393FBF2F398F81C209D
:10E038006FF0040A0AFB02FA534504DB02EB820A7A
:10E048009A45A8BF9A4642F21072924B53F82400A0
:10E0580038449042A8BF10468F4A9042B8BF104635
:10E0680043F8240098F812305843031302932D887C
:10E0780005F00303012B38D0804B884933F914305D
:10E08800A6000093019B51F8247093F801E0844B9B
:10E0980033F9140080EAE073A3EBE073B3F5206F63
:10E0A80016DC009A50235A4392FBFEF3042290FB9D
:10E0B800F2F0181A0744B7F57A5F7A4BA8BF4FF405
:10E0C8007A579F42ACBF41F8247041F8243002E0EF
:10E0D800002341F824308B597D2693FBF6F6019BEB
:10E0E800DB7A7343402693FBF6F6AA0712D5009A0B
:10E0F80009FB06F509FB02F70298C9F5FA7303FB59
:10E108000A7703FB00534FF4FA7297FBF2F193FB83
:10E11800F2F505E0EB0755BF354651460099029DDB
:10E128005F4B042733F914305F4A93FBF7F3A25C83
:10E138006FF04F07534393FBF7F398F851204FEADA
:10E14800440BCF1872B13846069204F015FF5749B0
:10E15800574B01EBC401069A1B68FBF747FD05F016
:10E1680025F907464E4B534A3BF803003BF902108A
:10E1780003B25B1A042193FBF1F102F1040E5EF87D
:10E1880024302BF802000C3252F8240042F82430D4
:10E1980098F8502018444FEA840C08444EF824108C
:10E1A80082B1CDF81CC0069204F0E6FE4249404B0D
:10E1B80001EBC401069A1B68FBF718FD05F0F6F899
:10E1C800DDF81CC03D4BDFF810E11B5D7A195843A0
:10E1D800202390FBF3F3D21A2BF80E20384A5B4227
:10E1E8004CF80230019B3748374901334CF801504D
:10E1F8004CF80070019375460CB90124DEE61F4BFC
:10E208000427B3F90440049B244E9B79D6F808E010
:10E218000F335B006343224C5B11B4F90440002BBD
:10E2280094FBF7F7A3EB0707B8BF5B42322B98F8CC
:10E238000D400BDC04FB07E4244BA342A8BF234694
:10E24800234CA342ACBFB360B46001E00023B360C9
:10E2580098F8034004FB07F31E4C9B112478032C09
:10E268003DD9B8F84E40B4F5FA7F38D26742BB4280
:10E2780034DBA342A8BF234631E000BFCC11002005
:10E288008C1A0020E0300020F42C002068A101083E
:10E298000000204144270020F0D8FFFFE02900209B
:10E2A8000811002080C1FFFF682A0020C42900202F
:10E2B800DC2900204C270020102A00207C2A00207E
:10E2C800482A0020302A00203C2A0020FEFFFF0FA9
:10E2D800020000F07F2A0020282A00203B46B4686C
:10E2E8006FF0FF0644F34F34B4F5807FA8BF4FF4B6
:10E2F8008074B442B8BF344683601E190023AE80D0
:10E308008C60936009B0BDE8F08F2DE9F04F87B0BD
:10E318000393B44B81461D88029105F00205ADB206
:10E32800019295B1B04BB3F90250B3F90030002D0A
:10E33800B8BF6D42002BB8BF5B429D42B8BF1D46B7
:10E34800B5F5007FA8BF4FF40075CB460026A64B55
:10E35800A64933F91620A64B4FEA460A33F9163078
:10E36800520083EAE374A4EBE374B4F5206F4FEA38
:10E37800860851F8260011DC042493FBF4F3D31A21
:10E388000344B3F57A5F9B48A8BF4FF47A5383429E
:10E39800ACBF41F8263041F8260002E0002341F8DE
:10E3A800263051F808709BF80B30FF119BF801409C
:10E3B8005F438C4B54431B88BF119B074FEAA4143F
:10E3C80056D08D4B3AF903301A44019B5B429A426E
:10E3D80003DB019B9342A8BF1346884A3AF90220FF
:10E3E8009B1A039A32F916201A440492FFF7B2FDD9
:10E3F800049A98B1824B10469B5D049304F0BCFDCF
:10E40800804904F0C1FE049B0146184603F0E4FE6F
:10E418007C4904F005FE04F0C9FF024642F2107080
:10E42800794958F8013013448342A8BF0346774816
:10E438008342B8BF034648F8013099F8081099F8A4
:10E448001C004A4300EB8000D21141428A4203DBA0
:10E458008242A8BF0246114699F81220641A534313
:10E468001B13FF1A6F436C4303EB672701EB64240C
:10E478005F4B04223AF9033093FBF2F2644B9B5D45
:10E48800534399F85120A4EBA31472B12046049287
:10E4980004F072FD5F49604B01EBC601049A1B68EA
:10E4A800FBF7A4FB04F082FF044651495B4B3AF8A2
:10E4B80001003AF903E002B2CEEB02024FF0040E7B
:10E4C80092FBFEF22AF803009E440C3358F80EC063
:10E4D80058F8030048F80E206044104499F850207A
:10E4E80048F803C08C467AB10591049204F044FDC3
:10E4F8004B49494B01EBC601049A1B68FBF776FBB5
:10E5080004F054FFDDF814C0464BDFF834E19B5D9E
:10E51800E21943435B11D21A2AF80E2042484349B4
:10E52800434A5B4248F8004048F8017048F8023016
:10E538000BF1010B74460EB9012608E72A4B042794
:10E54800B3F90450029B294E9B79D6F808E00F33A3
:10E558005B006B43BCF904505B1195FBF7F7002B8C
:10E56800A3EB0707B8BF5B42322B99F80D500BDCC1
:10E5780005FB07E52F4BAB42A8BF2B462E4DAB4200
:10E58800ACBFB360B56001E00023B36099F80350F5
:10E5980005FB07F3294D9B112D78032D0CD9B9F8EC
:10E5A8004E50B5F5FA7F07D26F42BB4203DBAB4250
:10E5B800A8BF2B4600E03B46B5686FF0FF0645F361
:10E5C8004F35B5F5807FA8BF4FF48075B542B8BF09
:10E5D800354683605E190023A6808D60936007B07E
:10E5E800BDE8F08F8C1A0020CC110020E029002013
:10E5F8000811002080C1FFFFE0300020F42C00202B
:10E6080068A101080000204144270020F0D8FFFF3E
:10E61800682A0020C4290020DC2900206027002067
:10E62800102A00207C2A0020302A00203C2A0020C2
:10E63800482A0020FEFFFF0F020000F07F2A00207A
:10E64800282A00202DE9F04F89B00593AE4B00270A
:10E65800B3F90280B3F90030B8F1000FB8BFC8F1C0
:10E668000008002BB8BF5B429845B8BF9846824661
:10E67800B946BB463C46B8F5FA7F0492A8BF4FF4AA
:10E68800FA7802900397A14D2B88990757D0022C4E
:10E6980055D09D4B610033F914209D4B33F914304C
:10E6A80003EB4202049B5B429A4203DB049B9342C6
:10E6B800A8BF1346974A8E5E059A9B1B32F9140031
:10E6C8001E18FFF747FC90B1934B304613F804B07F
:10E6D80004F052FC914904F057FD0146584603F0F6
:10E6E8007BFD8E4904F09CFC04F060FE06469AF817
:10E6F80008306422734393FBF2F39AF81C206FF0FE
:10E70800040101FB02FB5B4505DB02EB820293423D
:10E71800A8BF13469B4642F21072814B53F824005F
:10E7280030449042A8BF10467E4A9042B8BF104677
:10E7380043F824009AF812305843031303932988A6
:10E7480001F00303012B01D1022C3DD16E4B764D14
:10E7580033F91490029BA00093F801E0734B55F82D
:10E76800247033F9146086EAE673A3EBE673B3F515
:10E77800206F1CDC022C14D0502303FB09F292FBFF
:10E78800FEF3042296FBF2F69E1B3744B7F57A5F38
:10E79800674BA8BF4FF47A579F42ACBF2F502B50FE
:10E7A80007E089EAE973A3EBE973642BE4DD00234E
:10E7B8002B505D4B7D27C35893FBF7F7029BDB7A01
:10E7C8007B43402793FBF7F78A0713D5022C11D018
:10E7D80008FB07F508FB09F60398C8F5FA7303FB6D
:10E7E8000B6603FB00534FF4FA7296FBF2F193FBAE
:10E7F800F2F508E0CB0704D5022C02D0039D594658
:10E8080001E03D46494663000193484B042633F92D
:10E818001430484A93FBF6F3A25C6FF04F0653435B
:10E8280093FBF6F39AF85120CE18E2B1022C069227
:10E8380030460BD104F0A0FB069A530803D09A4245
:10E84800A8BF1A4600E001223B4905E004F094FB0A
:10E858003A49069A01EBC401394B1B68FBF7C6F924
:10E8680004F0A4FD0646314B019A0198D15A354B64
:10E878000AB2C05E4FEA840C121A042092FBF0F22E
:10E888000198C15203F10801143351F824E053F8F8
:10E89800240041F82420704410449AF8502043F88A
:10E8A80024E082B1CDF81CC0069204F065FB26492D
:10E8B800234B01EBC401069A1B68FBF797F904F098
:10E8C80075FDDDF81CC0214B214A1B5D0199584399
:10E8D800202390FBF3F073191B1A8B521D4B4042F7
:10E8E8004CF803601C4B01344CF803501B4B032CB1
:10E8F8004CF80300029B03F1010302937FF4C3AEBB
:10E9080009B0BDE8F08F00BFCC1100208C1A0020A0
:10E91800E0300020F42C002068A10108000020410C
:10E9280044270020F0D8FFFFE0290020081100202C
:10E9380080C1FFFF682A0020D4290020C4290020B4
:10E94800DC29002074270020102A00207C2A0020BF
:10E95800282A0020302A00203C2A0020482A0020AB
:10E968002DE9F04F89B005939D4B80461B880C46D6
:10E978009B0702924DD540F2E631129B994AD889FD
:10E98800B2F900301B1A03F2F3158D4203D8002B9D
:10E99800B8BF5B4201E04FF4FA73B2F90220101AD3
:10E9A80040F2E63200F2F311914203D80028B8BFD2
:10E9B800404201E04FF4FA7098F84C503DB3984249
:10E9C800B8BF1846C0F5FA7004F0D6FA864904F0C4
:10E9D800DBFB4FF07E5104F019FA0646642090FBE9
:10E9E800F5F004F0C9FA0146304604F019FB4FF07F
:10E9F8007E5104F00DFA0021074604F0AFFC30B94F
:10EA080038464FF07E5104F0C7FC20B101E00027E2
:10EA180001E04FF07E57E31C0393CDF800800024FB
:10EA2800039B022C13F8015F704E039309D1B6F9CA
:10EA380004000A35684304F09FFA6D4904F0A4FB0A
:10EA480074E036F9140004F097FA8146029804F04D
:10EA58008FFA654904F098FB0146484604F0E0FA4D
:10EA6800644B814633F9140004F086FA014648469F
:10EA780004F0CEF9029B8146584204F07DFA8346A1
:10EA8800484659464FEA440A04F068FC48B90298D7
:10EA980004F072FA83464846594604F07DFC00B9F2
:10EAA800CB46554B33F90A0004F066FA014658463E
:10EAB80004F0ACF9059B814633F9140004F05CFAC4
:10EAC8000146484604F0A4F94C4904F05DFB814630
:10EAD800FFF740FA28B14A4B4946185D03F07CFB22
:10EAE80081463F4BB3F800B01BF0010F05D04846F4
:10EAF800D8F8441004F094FA18E036F90A001435EE
:10EB0800684304F039FA3A4904F03EFB1BF0020F5F
:10EB180005460CD0D8F84810484604F081FA394622
:10EB280004F07EFA0146284604F072F905466300AF
:10EB38000493344B344E33F9140004F01DFA334B6C
:10EB4800196E04F06DFA0146284604F05FF9009B3F
:10EB58008246196A04F064FA2D4B0546185D04F0E4
:10EB68000BFA0146284604F05BFA2A4904F00CFB2C
:10EB780098F85120814692B1022C09D1530803D04C
:10EB88009A42A8BF1A4600E001224846224902E0FC
:10EB9800224901EBC4013368FBF728F88146336842
:10EBA80050461946019304F03BFA009BDFF878B011
:10EBB800D96A04F035FA114904F032FA5BF82410E6
:10EBC80004F026F91649A500064604F0C7FB68BB01
:10EBD8003046144904F0E0FB48B3124E27E000BF6A
:10EBE8008C1A0020382D00200000FA43CC11002098
:10EBF80000004842E0300020F42C002000002041B2
:10EC080068A1010808110020DC2900204427002001
:10EC1800C02900200000C842D4290020C4290020AF
:10EC280000007AC300007A435C2A0020444E4BF867
:10EC38000560DFF83CB1504655F80B1004F0E6F8D3
:10EC480045F80BA0069001994FF07E5004F09CFA0D
:10EC5800069B0146184604F0E3F982460BF10C03C3
:10EC6800EA580BF1180B104655F80B10079306924B
:10EC780004F0CEF8514604F0CBF8069A079B45F805
:10EC88000B2098F85020014645F803A032B12D49D1
:10EC9800019B01EBC401FAF7A9FF014608462A497E
:10ECA80004F072FA009B996B04F0BAF9274B82467C
:10ECB800185D04F061F90146504604F0B1F92449A1
:10ECC80004F062FA2349824604F048FB38B95046FA
:10ECD800214904F061FB20B1DFF87CA001E0DFF8F6
:10ECE80074A03146484604F093F8514604F090F871
:10ECF80008F060F9194BB0F57A7FA8BF4FF47A7025
:10ED08009842B8BF1846049A154B0134D052484669
:10ED180004F04CFB134B5851304604F047FB124BA0
:10ED28005851504604F042FB104B032C5851009B9D
:10ED380003F1040300937FF473AE09B0BDE8F08FCC
:10ED480000007AC3102A002000004040C02900209B
:10ED58000000C842000096C30000964318FCFFFF5D
:10ED6800282A0020302A00203C2A0020482A002097
:10ED7800A8270020044B00221A605A60034B002287
:10ED88001A605A60704700BF44270020542A0020A8
:10ED980010B50C4C0123E3704FF48060022384F813
:10EDA8002030FBF7E7FA084A084BD2F888201B689E
:10EDB8005278642101FB0233636123880133238085
:10EDC80010BD00BF9430002044270020202D0020D3
:10EDD800084BDA68D10709D4DA68520708D4DB6827
:10EDE80013F0100F14BF0320042070470120704750
:10EDF800022070470020024070470120704770478A
:10EE080003788B4286BF024B33F81100002070470D
:10EE1800D027002008B50021062207F0BEFE0120F9
:10EE280008BD08B50021062207F0B7FE012008BD7D
:10EE380070B50546F9F726F9324CA369A061C31AE3
:10EE4800B3F5FA5FE36182BF002384F8203084F8C9
:10EE5800213094F820302BB9A12D02BF294A012175
:10EE680082F8211094F82110264A31B1D118EDB258
:10EE7800013381F8225082F8203094F8205094F819
:10EE88004330AB423CD11F4B93F84430052B02D0A2
:10EE9800062B03D02FE0002003F0C8FE94F823309F
:10EEA8001E2B28D100200246C1B26B1E99421ADAE5
:10EEB800214491F822300821DBB283EA0206F607E2
:10EEC80044BF83F01803C3F3460301F1FF3154BF75
:10EED8005B0843F0800311F0FF01C2F34702ECD155
:10EEE80001301A46E0E7234493F822309A4202D1CF
:10EEF800032003F09BFE002384F8213084F820309F
:10EF080070BD00BFD027002010B50446B0F900003E
:10EF180003F0E8F8B4F9020003F0E4F8B4F90400E7
:10EF2800BDE8104003F0DEB810B50446006803F0F1
:10EF3800D9F8606803F0D6F8A068BDE8104003F07F
:10EF4800D1B82DE9F74F0120F8F770FF002488B3F6
:10EF5800012C2FD84FF04C0909FB04FA174E06EB89
:10EF68000A0808F19007BD7815B10134E4B2EEE75C
:10EF780090F9003090F804E01846114B03228DE810
:10EF8800240001212A4653F82E30F9F702F9834666
:10EF980060B106F14800504429464A4607F0FDFD95
:10EFA80001231C44C8F848B0BB70E4B20120F8F74C
:10EFB80023FFCCE703B0BDE8F08F00BFD0270020C7
:10EFC80034A101080021222210B5104807F0E5FD00
:10EFD8000F4B002219460F480424105C013283F8B5
:10EFE800F60183F8FB4105200024042A83F8FA017E
:10EFF80083F8FD4183F8FC0103F10803EBD10123F9
:10F00800A1F8F831522381F8F43110BDC81300205B
:10F01800D4110020A8C1010870B50646441E14F892
:10F02800011F89B1094D284607F0EDFD0028F6D0EB
:10F0380005F1080398423FBF054B401BC018A31BAE
:10F0480038BF80F88A31EAE770BD00BF3AD00108BE
:10F05800D411002007B51C4B03F1E402C3F8E020EB
:10F068001A4A92F892215AB1012A14D1032183F83D
:10F07800E610072183F8E82083F8E7100C2208E05F
:10F08800022183F8E610032183F8E82083F8E710CB
:10F09800072283F8E4200E4A0E4B40201A60F8F746
:10F0A800C5FE70B10122002390F9000040218DE8CF
:10F0B8000C00094A4FF4E133F9F76BF8003018BF38
:10F0C800012003B05DF804FBD0270020D4110020F4
:10F0D800F129010830000020A12A0108012000219F
:10F0E80002F0C4B9174AF0B5164692F8E930D2F8DA
:10F0F800ECE0032B10D85C1C0EEBC3039D1CE4B2A0
:10F1080008D09A88D10705D5104203D008E001310C
:10F11800042907D12346ECE786F8E9300020F0BD42
:10F128009F7800210C2202FB01F3064D05F1F00C3B
:10F138001CF803209742EAD12B4485F8E940D3F81C
:10F14800F400F0BDD02700208A6810B50C6A036867
:10F1580014430A6923F4FF4314434A6923F07003F4
:10F1680014438A691443CA6914434A6A14438A6A6D
:10F17800224313430360CB6843600B6883604B688A
:10F18800C36010BD4FF6FE7302681340036000238E
:10F19800036043608360C360284B984201D1284ACA
:10F1A80027E0284B984201D1254A2AE0264B98426D
:10F1B80001D1234A2DE0254B984201D1204A30E065
:10F1C800234B984201D11E4A33E0224B984204D186
:10F1D8001B4A536843F470032EE01F4B984204D136
:10F1E800174A536843F0706326E01C4B984204D1D9
:10F1F8001B4A536843F00F031EE01A4B984204D190
:10F20800174A536843F0F00316E0174B984204D1AD
:10F21800134A536843F470630EE0144B984204D1C8
:10F228000F4A536843F4704306E0114B984204D1E7
:10F238000B4A536843F47023536070470800024038
:10F24800000002401C00024030000240440002401E
:10F25800580002406C00024080000240080402404E
:10F26800000402401C0402403004024044040240EE
:10F2780058040240224A10B5536803F00C03042BCB
:10F2880003D0082B04D01F4B14E01F4B5B6811E020
:10F2980053685168C3F38343C90303F1020301D4DC
:10F2A8001A4906E0516811F4003F1749496818BF28
:10F2B80049084B4303605368154CC3F303132344B5
:10F2C80093F820100368CB4043605168C1F30221D2
:10F2D800214491F8201023FA01F181605168C1F3AB
:10F2E800C221214491F82010CB40C3605268C2F378
:10F2F8008132224492F83020B3FBF2F3036110BD4F
:10F308000010024000127A003000002000093D0081
:10F3180034A1010810B50446FFF75AFD012806D1AB
:10F328001CB1FFF755FD013CF8E7052010BD002C86
:10F3380008BF052010BD0A88F0B54B888E88B1F843
:10F3480008E0CC88002A3AD1028C43F0010322F06D
:10F3580001021204120C0284058B078CADB225F051
:10F36800F30545EA0E1189B241EA06027A49BFB2AD
:10F37800884212D001F5006188420ED0B0F1804F6A
:10F388000BD0A1F59831884207D001F580618842F9
:10F3980003D001F58061884202D127F0020701E01D
:10F3A80027F00A071F4302830784038B23F00C030B
:10F3B8001B041B0C0383038B9BB21C4344E0042AED
:10F3C80044D1028C22F010021204120C0284018B28
:10F3D800058C21F440721205120D42EA0E325E4984
:10F3E80092B242EA06228842ADB292B212D001F538
:10F3F800006188420ED0B0F1804F0BD0A1F5983152
:10F40800884207D001F58061884203D001F5806108
:10F41800884207D125F0200141EA03139BB243F04B
:10F42800100304E025F0A00143F010030B4302830E
:10F438000384038B23F440631B041B0C0383038B9B
:10F448009BB243EA0424A4B20483F0BD082A028CC8
:10F458003ED122F480721204120C0284828B3E4D3B
:10F4680092B222F0F307018C47EA0E1292B2A84238
:10F4780089B242EA060212D005F50065A8420ED00C
:10F48800B0F1804F0BD0A5F59835A84207D005F507
:10F498008065A84203D005F58065A84207D121F40C
:10F4A800007141EA03239BB243F4807304E021F422
:10F4B800206143F480730B4382830384838B23F09E
:10F4C8000C031B041B0C8383838B9BB21C4341E0FE
:10F4D80022F480521204120C0284858B018C25F4CC
:10F4E80040752D052D0D45EA062545EA0E321A4DC3
:10F4F80089B2A84292B212D005F50065A8420ED092
:10F50800B0F1804F0BD0A5F59835A84207D005F586
:10F518008065A84203D005F58065A84207D121F48B
:10F52800005141EA03339BB243F4805305E047F6A8
:10F53800FF5543F480530D402B4382830384838B10
:10F5480023F440631B041B0C8383838B9BB243EA25
:10F558000424A4B28483F0BD002C0140CA78F0B51D
:10F56800D40648BF8C780D8802F00F0348BF2343A8
:10F5780015F0FF0F1DD0016800240126A64006EAF9
:10F588000507B74211D14FEA840E0F2606FA0EF688
:10F5980021EA0601282A03FA0EF641EA060101D1FA
:10F5A800476102E0482A08BF07610134082CE4D10A
:10F5B8000160FF2D1FD94168002404F108070126C6
:10F5C800BE4006EA0507B74211D14FEA840E0F265E
:10F5D80006FA0EF621EA0601282A03FA0EF641EA8F
:10F5E800060101D1476102E0482A08BF07610134DA
:10F5F800082CE2D14160F0BD0F4B1A6842F00102BD
:10F608001A6059680D4A0A405A601A6822F08472D2
:10F6180022F480321A601A6822F480221A605A682A
:10F6280022F4FE025A604FF41F029A60044B4FF016
:10F6380000629A60704700BF001002400000FFF8A7
:10F6480000ED00E02DE9F8435B4C0368013AC4F88B
:10F65800203183880D46A4F82431072A42D8DFE8F0
:10F6680002F0040A101822292F35B4F820310B8033
:10F67800B4F8223113E0B4F822310B80B4F8203109
:10F6880005E0B4F820315B420B80B4F822315B42CC
:10F6980005E0B4F822315B420B80B4F820316B806E
:10F6A800B4F824311DE0B4F820315B420B80B4F883
:10F6B800223112E0B4F822310B80B4F820310CE08A
:10F6C800B4F820310B80B4F8223105E0B4F82231C7
:10F6D8005B420B80B4F820315B426B80B4F8243174
:10F6E8005B42AB80354B1B7A002B62D1B5F9000029
:10F6F80003F042FC8046B5F9020003F03DFC0746E2
:10F70800B5F9040003F038FCD4F828110646404641
:10F7180003F086FCD4F834118146384603F080FCA7
:10F728000146484603F074FBD4F840118146304640
:10F7380003F076FC0146484603F06AFB07F03AFC02
:10F74800D4F82C112880404603F06AFCD4F838110C
:10F758008146384603F064FC0146484603F058FBEE
:10F76800D4F844118146304603F05AFC0146484615
:10F7780003F04EFB07F01EFCD4F8301168804046B9
:10F7880003F04EFCD4F83C118046384603F048FCA0
:10F798000146404603F03CFBD4F848110746304682
:10F7A80003F03EFC0146384603F032FB07F002FC4A
:10F7B800A880BDE8F88300BFD027002030000020D3
:10F7C80038B50F4B1B689C890E4B186880F31000E6
:10F7D800201A03F0D1FB0C4903F022FC0546204611
:10F7E80003F0CAFB0146284603F0CEFC03F0DEFD19
:10F7F8006428A8BF642020EAE070C0B238BD00BF0A
:10F80800B0190020C01900200000C84244F6FB715E
:10F81800084B1A68137803EB431300FB0313507863
:10F82800C0EB0030B3FBF0F39078B3FBF0F080B29C
:10F83800704700BFB019002008B50A480A2290F89E
:10F848004D3100EB4303B3F85C1100F5B47089B295
:10F8580020F8041C00F040FC80B2FFF7D7FF024BF1
:10F86800188008BDD0270020B41900202DE9F04FDA
:10F8780089B00593A04B80461B880492980737D51A
:10F8880040F2E632129B9D48DC89B0F900301B1B20
:10F8980003F2F315954203D8002BB8BF5B4201E091
:10F8A8004FF4FA73B0F9022040F2E630121B02F26C
:10F8B800F314844203D8002AB8BF524201E04FF43F
:10F8C800FA729342B8BF13460522C3F5FA7393FB45
:10F8D800F2F30A22643B534398F81C20D210534396
:10F8E800642293FBF2F3134423EAE373DBB200E0F0
:10F8F8006423C1460193CB1C03930024039B022C71
:10F9080013F8016F7E4F03934FEA440A05D1B7F904
:10F9180004301B365E4376114AE07A4B37F91420DF
:10F9280033F9143003EB4202049B5B429A4203DB37
:10F93800049B9342A8BF1346734A32F90A50059AAA
:10F948005B1B32F9145003EB050BFEF703FB88B180
:10F958006E4A5846155D03F00FFB6D4903F014FC21
:10F968000146284602F038FC694903F059FB03F0C8
:10F978001DFD8346604A1288D10714D437F90A500E
:10F988001B366E4393074FEA261611D598F8125086
:10F998009DF9042005FB0BF35343642293FBF2F318
:10F9A80006EB231604E098F8085005FB0BF52E111A
:10F9B800584B042533F90A30574F93FBF5F5751B5F
:10F9C80099F80160E35D6E435E430293642396FBFE
:10F9D800F3F698F851B0F611BBF1000F1BD0022CCA
:10F9E80030460CD103F0C8FA5FEA5B0304D05B45EC
:10F9F800A8BF5B461A4600E00122484905E003F02B
:10FA0800BBFA5A46391D01EBC401FB69FAF7EEF857
:10FA180003F0CCFC0646424B99F80B7019883E4B14
:10FA280001FB05F203F1200E5EF82400D21207FB59
:10FA380002073C4AB7F5001FA8BF4FF400179742CA
:10FA480003F12C00B8BF174650F8242040F8245082
:10FA58004FF6FF700909B0FBF1F1AA1A4A4303F106
:10FA6800380103F144054EF8247051F824E055F8A4
:10FA7800240045F824E098F85050921170444FEA59
:10FA8800840C7F13104441F824208DB1CDF818C0A0
:10FA9800079303F071FA079B2A4603F1500101EB23
:10FAA800C401DB69FAF7A2F803F080FCDDF818C09E
:10FAB80099F81530F2195843029B0134434318460C
:10FAC800642390FBF3F0184B0012024423F80A2039
:10FAD80003F108024CF80260032C03F1140203F14D
:10FAE80020034CF802704CF8030009F101097FF477
:10FAF80005AF09B0BDE8F08F8C1A0020382D002022
:10FB0800CC110020E0300020F42C002068A101086E
:10FB18000000204108110020C0290020D42900201D
:10FB2800E41000200000E0FF282A00202DE9F04F13
:10FB3800054690F850008DB008910592099318B1C8
:10FB48003228A8BF322000E0012003F015FA014650
:10FB5800AA4803F019FBAA4B04461888002808BFD6
:10FB6800012003F009FAA749069003F059FA019019
:10FB78000199204603F04CF90146019803F004FB73
:10FB8800A14B07901B889A0724D5A049B1F90030EA
:10FB9800B1F9020083EAE37280EAE071A2EBE37252
:10FBA800A1EBE07191420C46B8BF1446B4F5E17F71
:10FBB80012DA914203DD0028D8BF404203E0002B4F
:10FBC800CCBF1846584203F0D7F9914903F0DCFA44
:10FBD800064603E0002601E04FF07E564FF000098C
:10FBE800CA4603950024630004938A4B33F9140032
:10FBF80003F0C2F9884903F013FA03F0D7FB03F0C6
:10FC0800BBF9864903F00CFA804B029033F91400D3
:10FC180003F0B2F97C4B07461B889B077ED0014650
:10FC280003F0F6F87E4B804633F9140003F0A4F98C
:10FC38000146404603F0ECF803F0B8FB059B5B4235
:10FC4800984203DB059B8342A8BF0346754A049983
:10FC5800885E099A1B1A32F91400184403F08CF9CB
:10FC68008046FEF777F970B16F4B40466F4914F83C
:10FC7800039003F089FA0146484602F0ADFA6B4951
:10FC880003F0CEF98046287F03F072F9684903F043
:10FC9800C7F98246287A03F06BF90146404603F01B
:10FCA800BFF9644903F0BCF903F080FB81460AF10F
:10FCB800004003F07BFB814505DB504603F076FBF3
:10FCC8004845A8BF484603F057F9DFF88C910199D9
:10FCD8008246404603F0A4F959F8241003F098F836
:10FCE80055494FEA840B804603F038FB38B9404643
:10FCF800524903F051FB20B1DFF8408101E0DFF801
:10FD0800388149F80B80A87C03F032F90146404657
:10FD180003F086F94A4903F083F981463A4BB3F870
:10FD280000B01BF0010F40F099803A4B049ADFF8BD
:10FD38002081D35E002BB8BF5B42B3F5206F4FEA3A
:10FD480084030A9303DD002348F824302AE03D4960
:10FD5800384603F065F9039B0B90587803F008F9CF
:10FD68000B9A0146104603F00FFA029903F04EF879
:10FD7800019903F055F958F8241003F049F832496D
:10FD8800804603F0EBFA38B94046304903F004FBEB
:10FD980020B1DFF8B88001E0DFF8AC802C4A0A9B7C
:10FDA80042F80380039BD87A03F0E2F8284B53F813
:10FDB800241003F035F9274903F032F91BF0020F3C
:10FDC80080464DD03846514603F020F8014630466B
:10FDD80003F026F90146504603F01AF8494607464B
:10FDE800404603F013F80146304603F019F901467E
:10FDF800484603F00DF8804632E000BF83F9223E02
:10FE0800E4100020BD3786358C1A0020CC11002064
:10FE18000000E143081100200000A03ECDCC4C407A
:10FE2800E0300020F42C002068A1010800002041E7
:10FE38000000A0406F12033C0000F0C10000F04138
:10FE48000AD7A33D0000A043000040C30000404380
:10FE58005C2A00200AD7233C542A0020C84657466B
:10FE6800DFF83CB20BF1A803185D03F085F80146F2
:10FE7800029803F0D5F8894903F0D2F801463846CC
:10FE880002F0C4FF95F85120034642B10BF104017A
:10FE9800DBF81C3001EBC401F9F7A8FE0346804FDC
:10FEA800029807F1AC0B5BF824100A9302F0AEFF3E
:10FEB800019903F069F9029B07F1B4024BF8243069
:10FEC80052F824B00292594602F0A0FF0146079862
:10FED80003F0A6F80146584602F09AFF029A8346B4
:10FEE80042F8240007F1BC02105D03F045F8014612
:10FEF800584603F095F86B4903F092F883460A9B3D
:10FF08004146184602F084FF594602F07FFF07F089
:10FF180051F8049B07F16802D0520A9B07F170025E
:10FF28001846029203F042FA029A07F17C0342F85B
:10FF380024004046029303F039FA029B07F188082F
:10FF480043F824000BF1004003F030FA039B48F813
:10FF58002400013303930CB9012444E6089A524B58
:10FF68009479B3F90430640028345C434F4B64112E
:10FF7800B3F9040003F000F84FF07A5103F050F899
:10FF880007F018F8201A02F0F7FF002CB8BF6442F7
:10FF9800322C064602DD0023BB6224E0069803F0FB
:10FFA80005FA20F0030002F0E7FF8046687B02F0C4
:10FFB800DFFF0146304603F033F83D49044640462A
:10FFC80003F0E2F80146204603F02AF803F0EEF9C0
:10FFD800BB6A1844374B9842A8BF1846364B98421C
:10FFE800ACBFB862BB62BB6A6FF0FF005B13B3F5CE
:08FFF800807FA8BF4FF4807365
:020000040801F1
:100000009842B8BF184602F0BBFF8046304603F066
:10001000D1F9EB785843801102F0B2FF97F8BF3066
:100020000446032B11D9B5F84E60B6F5FA7F0CD211
:1000300003F0C0F97342984203DBB0420346A8BF05
:100040003346184602F09CFF044695F8512062B1F1
:10005000530803D09A42A8BF1A4600E00122204666
:100060001849FB69F9F7C6FD04464146204602F0EF
:10007000D3FE03F09FF900B202F082FF06F09EFF6C
:10008000A7F86C00204603F095F9B867404603F0E6
:1000900091F90023C7F88400C7F890300DB0BDE88F
:1000A000F08F00BFA69B443BC0290020F7CC9238BC
:1000B000CC1100200811002000803B45FEFFFF0FFF
:1000C000020000F0D42900200368DB6818470368A9
:1000D0009B68184703685B68184703681B681847E4
:1000E000B0F902302DE9F74F93421CBF0023037093
:1000F00090F800A004460E469146BAF1000F40F079
:10010000AB80104602F03CFF864902F08DFF864925
:1001100002F08AFF4FF07C5102F086FF06F0AEFF3E
:100120000146054602F080FF80498346284602F0DA
:100130007BFF034658461946019302F06DFE4FF0CF
:100140007E5102F069FE01464FF07E5003F020F828
:100150002946804602F068FF294602F065FF0746FF
:100160000146606002F058FEE7604FF07E57294676
:10017000A0602761284602F04FFE294602F054FF96
:100180004FF0804102F046FE0146404602F04CFF2F
:10019000019B60611946584602F03CFE394602F068
:1001A0003BFE0146404602F03FFF40F2DC53A046D2
:1001B0002746554663651023A4F852301823A061E2
:1001C000A4F850304FF09741D8F8100002F02CFFFF
:1001D0000021824603F0C6F828B150464FF07C510A
:1001E00002F018FE04E050464FF07C5102F014FE7D
:1001F00003F042F9C7E90E014FF09741D8F8040027
:1002000002F012FF0021824603F0ACF828B15046FC
:100210004FF07C5102F0FEFD04E050464FF07C515F
:1002200002F0FAFD03F028F90135032DC7E90801B2
:1002300008F1040807F10807C4D1A6F2DC531B0437
:100240002367E3676367C4F88030A367C4F884302A
:100250000123A4F802902370D4F85490B4F952808A
:10026000C9EB0606636A06FA08F67343276A4FEA83
:10027000E67B206F07FB0B332667A7FB0667E26F61
:100280001F44636CD4F840C053434FEAE27B0CFB3D
:100290000B3ED4F88010C4F88020ACFB02237344DA
:1002A000B61A67EB0307E36AA26A43434FEAE07BAF
:1002B00002FB0B3EA2FB00237344B6185F41E36CC4
:1002C000656F4B436067A06C4FEAE17B00FB0B332B
:1002D000C4F88410A0FB01011944636B361A05FBB6
:1002E00003F3206B4FEAE57B00FB0B3367EB010761
:1002F000A0FB0501801919447941B4F95020A56784
:1003000002F076FD08F1FF3201239340E067C01848
:1003100041EBE371424602F06BFD484403B0BDE897
:10032000F08F00BF6F12833ADB0F4940F404B53FF2
:100330002DE9F8430024254BE0B293F8BF60B042AA
:100340000DD203EB8003224AD3F8C03032F81010EC
:100350001BB10B2801D8DB6898470134EBE71D4B34
:100360001B685B032FD500242346E2B2B2422AD297
:10037000DFF858904FEA840809F1C00757F82420A5
:1003800055689D4217D02846FBF71EF8EFF31283FD
:10039000502282F312882821AA8C01FB009092B28D
:1003A0000132C0F81421AA8ADBB292B242F00102F3
:1003B000AA8283F3118857F8083000221B680134A1
:1003C0001A802B46D1E7BDE8F88300BFC029002082
:1003D00028110020FC2C002008B50E4B1B6813F4DC
:1003E000805F0D4B14BFD3F89021D3F8942193F87C
:1003F000BF1092880023D8B2884204D2074820F860
:1004000013200133F7E7FFF793FFBDE808403220E0
:10041000F7F763BEFC2C0020C02900202811002023
:100420000A4B30B51A680A4B02F48052D3F8904157
:10043000D3F8945100230AB1A18800E0A9880548A7
:1004400020F8131001330C2BF5D130BDFC2C00200B
:10045000C0290020AA2C002070B5124D002421468E
:1004600005F29910702285F8984106F09AFB214612
:10047000D5F80C320B4A0B4493F9020088B11E6880
:1004800002F299140E5108199C88073184809B79D7
:100490007029837192F8983103F1010382F8983141
:1004A000E6D170BDC0290020094B1A680E2303FB5A
:1004B0000020437AFF2B07D0064A12789A4203D9CC
:1004C000054A32F8130000E0808800B2704700BF90
:1004D0001C1B0020B4280020382D00202DE9F74FE8
:1004E000304C0546D4F810723846F9F765FE0646DA
:1004F0003846F9F7EEFDD4F8147281463846F9F71C
:100500005BFE01903846F9F7E4FDD5F804A00746F4
:100510003146504602F088FDD5F8088083464946AA
:10052000404602F081FD0146584602F073FC019BF3
:1005300029688346184602F077FD4946054650462D
:1005400002F072FD394602F06FFD0146284602F0C6
:1005500063FC39460546404602F066FD314602F02E
:1005600063FD0146284602F057FC0146584606F056
:10057000FDFD0D4902F058FD0C4902F009FED4F8CA
:10058000181202F049FC0A4902F002FE06F016FDBC
:1005900083B21A0444BF00F5B47083B218B203B03A
:1005A000BDE8F08FC02900200000E144DB0F494086
:1005B0000000204101380A4B042804D8DFE800F08D
:1005C0000507090B0D00074A08E0074A06E0074A3D
:1005D00004E0074A02E0074A00E0074A1A60704751
:1005E000480000204DE6000875F8000869E9000899
:1005F00013E3000881DF000835FB000810B54B88C5
:10060000DC0641BF2F4B14791B6853F8244044BFCC
:100610002D4B43F820404B889B0641BF294B547912
:100620001B6853F8244044BF274B43F820404B88B5
:100630001C070ED5254B0C781B78B3EB141FA1BFFC
:10064000204BD4781B6853F82440A4BF1E4B43F8BA
:1006500020404B889B070ED51D4B0C781B78B3EBC5
:10066000141FDFBF174B54781B6853F82440DCBFBE
:10067000154B43F820404B88DC070FD5154C0B7801
:10068000247803F00F03A342DFBF0E4B14781B68DE
:1006900053F82440DCBF0C4B43F820404B885B07E9
:1006A0000FD50B780C4903F00F0309788B42A1BFDB
:1006B000044B92781B6853F82220A4BF024B43F8E6
:1006C000202010BD141B0020720E00209B1D002056
:1006D000991D0020981D00209A1D0020254A002306
:1006E000F0B515681C461A462348244903700B7060
:1006F0002E1976884EB92F5D3FB9037000230A701A
:100700004B7007781C461A460CE0360548BF01328C
:1007100004F1040403F1010348BFD2B2802CDBB220
:10072000E6D1EAE7E0B2B8420CD215F82400013471
:1007300006099E4200F00F00A8BF731C9042A8BF9C
:10074000421CEFE78A704B70C2F3470102F00102CE
:100750000A444C1E0A490B480A70C3F3470203F0CF
:100760000103134404700849501E084A08701370AE
:10077000F0BD00BF181B0020901D0020DC2B0020C6
:100780009A1D0020981D00209B1D0020991D00200F
:10079000924B2DE9F04FDA68914D1A612A6891B0B9
:1007A000DA60904A0295136843F0200313608E4B81
:1007B0001A78012A0CBF002201221A708B4B1A787A
:1007C000910740F14D838A490978042940F2488312
:1007D0008849097801F0040101F0FF0011B922F005
:1007E00001021A701B78DB0702D408B1FAF7D2FCB9
:1007F0008149CA78531C052293FBF2F202EB820274
:100800009A1A7E4BCA701F7892000023DFF810827C
:10081000DFF8109258F82310794C91FBF9FE04F19F
:10082000080040F823E0774844F8231000FB0E113D
:1008300042F2107091FBF0F004F1100680B226F83D
:1008400013004FF0140C04F114060CFB036C04F1BC
:100850003C0A5AF823605CF802504CF80210761BF0
:10086000314405264AF8231091FBF6F109FB0E11DD
:100870004434012F44F823104FEA830B444605D13A
:100880000238B0F5797F98BF4BF808100BB90123F7
:10089000BCE7594E029BB2461868336DC01A02F08D
:1008A0006BFB594902F074FC029B4FF07E511B68B0
:1008B0000746336502F056FD08B94FF07E574B4BA3
:1008C000CAF854701B78514E13F00103504D12D0EA
:1008D0000DAA00924F4B0EAA01920CCB94E8030094
:1008E000FAF76EFB0D9A6421B2FBF1F20E9B328097
:1008F00093FBF1F300E033802B809AF858303E4DA3
:10090000002B35D0696D4FF07E5002F041FC074658
:10091000EB6D2068C01A02F033FB394602F084FB0D
:1009200002F048FD2B6E86B2606836B2C01A02F043
:1009300027FB394B196802F077FB394602F074FB4C
:1009400002F038FDB5F9662000B28118B5F96420CF
:100950000220B31891FBF0F193FBF0F389B29BB244
:10096000A5F86A10A5F86830A5F86610A5F86430F7
:1009700001238AF85830294B61681B88206803F0EE
:1009800030031D4E264DCAF86010CAF85C00002BDB
:1009900000F0668206F17403009306F17803019378
:1009A000F26E336FFAF70CFB6B68306FC01A02F00F
:1009B000E7FA194B196802F037FB02F0FBFCF36E03
:1009C0002A68C6F880009B1AF3670C4B1B78012B32
:1009D0002AD0022B00F0E68042E200BF9C070020F4
:1009E000202D0020C419002052110020C819002019
:1009F000CE190020E7300020DC2B0020FC0F002067
:100A0000E02B0020806967FF00007A44421A002032
:100A1000441A0020541100203C0000208C1A0020B1
:100A2000D019002080969800D6F88430D6F8A040DF
:100A30000293D6F8943004F100400393D6F898302E
:100A4000776D059302F0B6FC8146204602F0B2FCB9
:100A5000D6F89C30BB4C0493BB4B06901B684FF000
:100A6000000B0793B94E4FEA4B0356F82B80A6F1C3
:100A70001402404632F81B50089302F081FA0299A2
:100A800002F0D2FA02F096FC401B1FFA80FA2836D8
:100A900026F81BA00FFA8AFA504602F071FA039961
:100AA00002F0C2FA02F086FC86B20AEB080002F0FD
:100AB00067FA059902F0B8FA394602F0B5FA2168EA
:100AC00002F0AAF902F076FC484504DB069B984246
:100AD000A8BF184600E0484602F052FA206002F033
:100AE00069FC079B304486B2987802F045FA984931
:100AF00002F09AFA01464FF07E5002F049FB394667
:100B000002F08AF90146384602F042FB099060681B
:100B1000D4F808A0C0EB080002F032FA394602F01F
:100B200037FB514602F076F9099A0146104602F069
:100B30007BFA0146504602F06FF93135ADB2622DB5
:100B400001462061C4F80480A0600ED9049802F028
:100B50006BFA02F02FFC7F4AB0F5FA6FA8BF4FF492
:100B6000FA609042B8BF104600E0002040F6B8326C
:100B7000064436B29642A8BF1646774A089B96426C
:100B8000B8BF1646754A54F8140B9E52142202FB45
:100B90000BF273495050BBF1000F40F061814FF0F0
:100BA000010B5FE7684BB6F8A8401F68736F3D897B
:100BB00002935B089D4228BF1D4623B29D4202DC82
:100BC0001FFA85F90AE06749706D02F02DFA02F00C
:100BD000F1FB20441FFA80F9A6F8A890DAF87860B3
:100BE000DAF8AC40341B2046FAF72CFA41F29313A2
:100BF0000028D8BF40429842CCBF0020012078B3E3
:100C0000204602F0BDF9584902F00EFAF9F761FAF0
:100C10000446029802F0B0F90146204602F004FAB8
:100C200002F0C8FB40F6B83380B2AAF8B00000B2B8
:100C30009842A8BF1846484B9842ACBF3018F018ED
:100C400048F6A043984203DDA0F50C40A03804E02C
:100C50000028BCBF00F50C40A030CAF8B40001E089
:100C6000CAF8B460DAF8B4300026C3F50C50283066
:100C7000039302F085F93C4902F0D6F90446F9F7EE
:100C80009BFA0F902046F9F724FADAF8B830DAF830
:100C9000C4400593DAF8BC300E9004F1004008938C
:100CA00002F088FB0490204602F084FBDAF8C030A2
:100CB000DAF854802A4C09900793730048460A9347
:100CC00002F05EF90EAB53F8261002F0ADF9DFF832
:100CD000A0A005463AF9160002F052F9014628464E
:100CE00002F098F802F066FB05B2204BB5F57A7F6A
:100CF000A8BF4FF47A759D42B8BF1D460AF13C0A61
:100D0000A8B22AF8160000B202F03AF90599824614
:100D100002F08AF902F04EFB089983B2504606931E
:100D200002F082F9414602F07FF9216802F074F87E
:100D300002F040FB049B98421CDB099B9842A8BF31
:100D4000184618E03810002000100020582C002011
:100D5000DB0FC94030F8FFFF48F4FFFF0A10002006
:100D6000601000200000C842D302373918FCFFFF92
:100D7000442C0020049802F003F920608346B878E0
:100D800002F0FAF8384902F04FF901464FF07E5070
:100D900002F0FEF9414602F03FF80146404602F0FB
:100DA000F7F90B906068D4F808A0281A02F0E8F868
:100DB000414602F0EDF9514602F02CF8DDF82CC066
:100DC0000146604602F030F90146504602F024F830
:100DD000656001462061A060079802F025F902F0E5
:100DE000E9FA069B1434034458469A4602F0E2FAA4
:100DF00040F6B832504400B29042A8BF10461B4A99
:100E00000A9B9042B8BF1046194A1A4998521422B8
:100E1000724342F801B00EB901264EE73B792BB17F
:100E2000039A642392FBF3F3134A13803B88029ADC
:100E3000124C9A420DD9D4F8AC30A06FC01AFAF710
:100E400001F942F2107380EAE072A2EBE0729A427A
:100E500006DD0B4B01221A70B4F8C820064B1A802D
:100E600011B0BDE8F08F00BFDB0FC94048F4FFFFB1
:100E70000A10002038100020F80F0020DC2B002082
:100E8000FC0F0020F0B5974D87B02B78023B082B64
:100E900000F29581DFE813F009002E004E00630098
:100EA0007B008D0009016E0179018F4B8F4C1A6810
:100EB000636864339A4240F2828100268C4B8D4AEB
:100EC0001B789E420ADA2368884FD05C30B101F06B
:100ED0005DF83B68013601333B60EFE72168834BE7
:100EE000525C002A40F06B811A604FF0FF325A606A
:100EF000032354E1262300937F4B492003F10C0286
:100F0000019302925021A3F10A020233F8F724FD63
:100F1000002840F05481794B4FF0FF311B6813F0EB
:100F20008002724B03D083E80300042337E11A6088
:100F300059602AE0724A0223002100930191029134
:100F4000482002F10803F8F707FD002840F0378138
:100F5000664B4FF0FF3218605A6005231FE10723EC
:100F60000093684B472003F10C0201930292002189
:100F7000A3F108020433F8F7EFFC002840F01F81CA
:100F80005A4B4FF0FF3218605A60062307E15E4A61
:100F900005230021009301910291532002F10803DF
:100FA000F8F7DAFC002840F00A81504B186007235C
:100FB000F5E04E4C236813B96360012323604C4B6A
:100FC0001A7863681344402BA8BF4023132B636037
:100FD00040F3F580454B1B680D2B00F2E780DFE8FE
:100FE00003F060070B0E121923282D3134404B51AA
:100FF000464800F0A9FF51E0454846493FE04648D1
:101000004649474A48E0474B474893F8D61793F874
:10101000D72741E0434B0C2193F8B027434801FB0D
:10102000023393F8B2172AE03E4B4148B3F844111B
:1010300025E03C4B3F48B3F8461120E03E4B3F488B
:1010400019691CE03E483F4B18E03F4B1B68D80431
:1010500004D5344B3D4893F87C1110E00C232360F9
:101060001FE0304B3A4893F8801193F8812193F8B0
:101070007F3100F079FF11E03648374B198800F0D6
:1010800073FF0BE01D4B1B6819050AD5254B334830
:10109000B3F88411B3F9822100F066FF6368181A6F
:1010A000606023680133236089E02D4B1B689A013F
:1010B00014D52C4B1B888BB92B4B0E201B6804A915
:1010C00004932A4B1B680593F8F72AF9284B4FF431
:1010D00080521A8009232B70F8F79CF9F8F702F96F
:1010E0006DE000BF5C2D0020202D00201C2F002073
:1010F000540000206CA10108D6A10108FC2C00209E
:1011000094A30108ACA30108F8A30108ACC101082D
:10111000C9C101087DB60108E1C1010868B601082E
:1011200074B60108D4110020F8C101080CC20108EE
:1011300019C201082BC20108942700203DC20108F2
:1011400050C201081A000020042F00205DC20108CF
:101150006DC2010889C20108002F002097C2010852
:10116000E8100020102F00200C2F0020CC30002091
:10117000242F0020134B1B78002BADD0124B1B6883
:101180009B01A9D408232B70A8E7104B1A68104BB9
:101190005B68C8339A4204D900F0AEFE01232B707D
:1011A0000DE000F0C3FE0028F6D108E000F0BEFE1E
:1011B00028B1084B4FF480521A800923EFE707B09B
:1011C000F0BD00BF082F0020E8100020202D0020D7
:1011D0001C2F0020242F002007B5064B0649009342
:1011E000064B074A01930748074BF8F743FF03B044
:1011F0005DF804FB74B601087EC001087DB60108E5
:1012000077C00108B7C3010868B6010808B50378BC
:1012100033B90C4B0C481978BDE80840F8F72ABFE1
:1012200005F058FD02280CD8064B0C221870074B0D
:1012300002FB0030064B0230186000F0C7FB054887
:10124000E5E708BDA82C0020D7C3010884190020B9
:101250004C1100202FB6010808B503783BB90B4BA1
:101260000B4893F8B017BDE80840F8F703BF05F046
:1012700031FD022808D8054B83F8B007F9F7C0F80C
:10128000F9F764F90348E8E708BD00BFD41100206E
:10129000DBC301082FB6010838B5037803BB214B27
:1012A0001B6801330F2B07D81F490C2202FB0312C6
:1012B00095681C462DBB00E01C4601340F2C01DD57
:1012C000002400E005D818490C2202FB041295689E
:1012D000BDB99C42F1D11548BDE83840F8F7CABE07
:1012E00005F0F8FC0F28044605D80F4A0C2303FB31
:1012F00000239D682DB92146BDE838400C48F8F719
:10130000B9BE084B1C60F6F775FE21462A4609480F
:10131000F8F7B0FE0C235C43034B185DBDE8384082
:10132000F6F77ABE4000002020A40108E8C30108B7
:10133000FEC3010816C4010873B5037813B9F6F7A4
:10134000D5F93DE01F4901AA05F025FD002401461D
:101350002646254699B134B1012C08D1084605F03E
:10136000B9FC064603E0084605F0B4FC05461549FD
:10137000002001AA05F00FFD01340146EAE70B2D1C
:1013800002D911480C220BE0022C10D1A6F57A7379
:10139000B3F57A7F07D90D484FF47A714FF4FA62AA
:1013A000F6F721F90CE00A4B03EB45035E80084B8E
:1013B000084803EB45032946B3F90220F8F75AFE23
:1013C00002B070BD52BA010890B80108B5BD01085D
:1013D000A82C00202DC4010838B50D4C0546236803
:1013E000834206D1F6F738FC204600214C2205F056
:1013F000D8FBE36CAB4209D12846F6F72DFCBDE8DB
:101400003840044800214C2205F0CBBB38BD00BF5A
:101410001828002064280020034B1A68D379591C2F
:101420001344D171187A70476C1A002010B5FFF779
:10143000F3FF84B2FFF7F0FF04EB002080B210BD91
:1014400010B5FFF7F3FF0446FFF7F0FF04EB004091
:1014500010BD10B50446054B21461868FEF73DFE49
:10146000034B1B6898796040987110BD701A00207A
:101470006C1A002038B504460D462420FFF7E9FF1A
:101480004D20FFF7E6FF002C084C14BF21203E2022
:10149000FFF7DFFF2368002228469A71FFF7D9FF84
:1014A000236893F84900BDE83840D2E76C1A002061
:1014B00001460020DEE710B50446C0B2FFF7C9FFC1
:1014C000200ABDE81040C4E710B5044680B2FFF71B
:1014D000F2FF200CBDE81040EDE737B58288836845
:1014E000044610060D4641BF29494FF4CC7091F8CF
:1014F000B01700FB0133D10542BF26490C20097803
:1015000002F03F0248BF00FB0133042A12D006D884
:10151000012A0DD0022A2FD193F900102DE0102AB4
:101520000AD0202A0AD0082A26D1B3F9001024E0D4
:10153000197822E0198820E019681EE069461868C9
:10154000F8F71EFC01461448F8F794FDF5B1E06881
:1015500001F016FD6946F8F713FC01460F48F8F74D
:1015600089FD206901F00CFD6946F8F709FC014688
:101570000A48F8F77FFD09E000210948F8F77AFDED
:1015800025B10848E1682269F8F774FD03B030BD61
:10159000D4110020A82C00206BB9010864B90108FF
:1015A00059C101083CC40108024B0146D869FEF745
:1015B00094BD00BFA82C002010B5441E14F8011FD4
:1015C00021B1034BD869FEF788FDF7E710BD00BFD6
:1015D000A82C0020F7B52A492A4B08782A4D1C6808
:1015E0002A4B05EB80001A88D0F8C010284B2948F8
:1015F0001B7800914FF47A71B4FBF1F1F8F73AFDE2
:10160000254B26481968264B0026B1FBF3F1F8F765
:1016100031FD244B1F68F3B205EB8302D2F8D010E2
:10162000E9B101249C403C4217D0220715D01E4A44
:101630000B20D25C00FB0323134A1C4802EB8303FC
:10164000D3F8F020F8F716FD022C06D1184B93F8CA
:10165000281011B11748F8F70DFD0136DBE71648E1
:10166000FFF7AAFF154B16481A88164B92B2198835
:1016700040F2DC7303B0BDE8F040F8F7FBBC00BFFC
:10168000141A0020202D002020A40108B4190020E5
:101690004400002043C401085000002086C4010813
:1016A00040420F00C41900204C00002096C40108DD
:1016B000A82C00209EC40108E6C40108E610002002
:1016C000A2C40108E41000202DE9F0410024804666
:1016D00025460F4E4146A759384605F0E3FA58B162
:1016E00039460C48F8F7C6FC30190021FFF7F5FE23
:1016F0000948FFF761FF013540F6BC4314349C42B2
:10170000E7D11DB9BDE8F041044855E7BDE8F081D7
:10171000C0A50108D4B90108E6C40108E7B801086A
:101720002DE9F74F824605F080FA054628B10128D9
:1017300019D19AF800302A2B15D15948FFF73CFFF0
:101740000024584E5848A159F8F794FC30192946FE
:10175000FFF7C3FE5548FFF72FFF40F6BC43143494
:101760009C42EED198E050463D2105F050FA002809
:1017700000F08D8003461D4613F8012D202AFAD073
:10178000441C204605F0A6FA81462046F8F762FA86
:101790000746CAEB05054FF0000B142404FB0BF4BD
:1017A000DFF8208108F5D073E6580193304605F044
:1017B0003CFA8446314662465046CDF800C005F0FA
:1017C0003DFADDF800C0019B002856D1EAB262451F
:1017D00053D11D194444D4F8AC0101F0D1FB0146AA
:1017E000384601F0D3FD002845D0D4F8B00101F00F
:1017F000C7FB0146384601F0BFFD00283BD0B4F8D6
:10180000A4319A0658BF4F46142202FB0B881C06CF
:1018100048BF2748D8F8A82142BF90F8B0074FF436
:10182000CC7404FB0022D80542BF22480C24007867
:1018300003F03F0348BF04FB0022042B39460BD0C2
:1018400004D8013B012B0CD817700AE0102B05D0EF
:10185000202B05D0082B04D1118002E0176000E096
:10186000176031461448F8F705FC2846002103B0FC
:10187000BDE8F04F31E6114805E00BF1010BBBF17B
:10188000A30F8AD10E4803B0BDE8F04F94E650464E
:1018900003B0BDE8F04F17E703B0BDE8F08F00BF1D
:1018A000D4C40108C0A50108D4B90108E6C40108E0
:1018B000D4110020A82C0020E9C40108F4C40108B8
:1018C000E7B8010820A4010870B50546284605F0D0
:1018D000ACF9064658B9194B19485A79194BBDE865
:1018E000704003EB8203D3F8581EF8F7C3BB2846B9
:1018F0001549324605F0A2F960B91448FFF75CFEBD
:10190000134C54F8041F19B11248F8F7B3FBF8E769
:10191000114805E00024114B53F8241019B9104860
:10192000BDE8704048E62846324605F087F90134A4
:101930000028F0D1014B0B4D5C71C7E7D41100209A
:1019400014C5010820A4010882B9010820C50108B6
:1019500078B201087EB90108E6C401087CB201082A
:10196000E7B801082FB6010808B50748FFF724FEBD
:10197000064BD869F6F75DFCFEF72EFDF8F716FD6D
:10198000034A044BDA6008BD33C50108A82C0020C7
:101990000400FA0500ED00E008B50548FFF70CFE6D
:1019A00000F05AF8F8F72CFDBDE80840DCE700BF6E
:1019B0003FC5010808B50448FFF7FEFDF8F720FD14
:1019C000BDE80840D0E700BF55C5010810B50E4C72
:1019D0002068F6F77DFA20680022047A02FB02F301
:1019E000193B634303F6C4135343192193FBF1F3EB
:1019F000064921F812300132072AEFD1BDE8104024
:101A00000349F6F71DBA00BF4C11002088100020D2
:101A1000181300200E4B1A78692A16D140F2DC7296
:101A20005988914211D11A79BE2A0ED193F8D9273B
:101A30000020EF2A0BD113F8012B5040054A9342A6
:101A4000F9D1B0FA80F04009704700207047704724
:101A500000F80308DCFF03082DE9F74FEA4C0021EA
:101A600040F2DC72204605F09CF8E84B04F53A722F
:101A70001A60E74B00221A70E64B04F2B27119604B
:101A800069232370032363714FF48073A3604FF4C1
:101A90001673A4F86631FA23A4F86831BC23A4F8BD
:101AA00064314FF4FA73A4F86E31012384F8623183
:101AB00084F87E3184F88631052384F8273240F299
:101AC000DC53A4F8983140F24C43A4F89A3140F228
:101AD0006C73A4F89C3140F27533A4F89E3140F643
:101AE0004303A4F8A0312346202184F86A116E2113
:101AF00084F87C110A2184F87D112B2184F87F1150
:101B0000212184F88011232184F881114FF4C871B8
:101B1000A4F88211032ACCBF0121002102F10102A5
:101B200083F8A21114BF1E217521122A83F8A31174
:101B300003F10203EED140F27E41A4F8441140F2D9
:101B40003A71A4F8461140F27E51A4F84C1140F2CB
:101B5000EA5140F2DC50A4F84E1140F2B4514FF477
:101B6000FA63A4F8C831A4F8CC31A4F8D031A4F8B1
:101B7000D431052384F8E231C82301264FF47A7763
:101B80004FF0320BA4F8E631DFF880924FF4C873BF
:101B90004FF01E0A1922A4F8EA31A4F84A01A4F869
:101BA0005011A4F8C671A4F8CA71A4F8CE71A4F8B3
:101BB000D27184F8E46184F8E56184F8E861A4F8FE
:101BC0004871A4F852B184F895A184F8E3210092F9
:101BD0000190A4F8543184F8E16184F8EE61A4F82E
:101BE00056B184F8F161FDF7F1F9D9F80030009AA7
:101BF00000254FF00F0E2674E673A573A58183F8B8
